:020000040800F2
:10500000C8480020D5500008D5D8000823CB000898
:105010000000000000000000000000000000000090
:1050200000000000000000000000000005E500088E
:105030000000000000000000D7D80008D5FA0008E2
:10504000E7500008E7500008E7500008E750000864
:10505000E7500008797B0008E7500008837B0008D0
:1050600000000000E7500008397A0008497A00087B
:10507000E7500008D5CF0008350E0108E7500008BA
:10508000E7500008E7500008E75000080000000063
:10509000E7500008E7500008E7500008E750000814
:1050A000E7500008E7500008E7500008150E010817
:1050B000250E0108E7500008000000000000000075
:1050C0000348854600F00EFD00480047F929010815
:1050D000C84800200448804704480047FEE7FEE730
:1050E000FEE7FEE7FEE7FEE799FB0008C150000877
:1050F00030B50B46014600202022012409E00D4670
:10510000D5409D4205D31D469540491B25469540F7
:1051100040191546521E002DF1DC30BD70B500243B
:105120002546002801DA01244042002901DA012540
:105130004942FFF7DDFFAC4200D04042002C00D0D6
:10514000494270BDF0B51FB40646002082B0054646
:105150004024019100901BE0019922460F46304601
:1051600000F020F8049A059B801A994110D310464C
:105170001946224600F018FB361A8F410197224645
:1051800001200021009F00F00FFB38184D410090D6
:105190002046641E0028DFDC019B00982946324629
:1051A00007B0F0BD10B5202A04DB0846203AD040F5
:1051B000002110BD0B46D340D0402024A21A9140BC
:1051C0000843194610BD03460B439B0703D009E073
:1051D00008C9121F08C0042AFAD203E00B78037032
:1051E000401C491C521EF9D27047D2B201E0027035
:1051F000401C491EFBD270470022F6E710B513464B
:105200000A4604461946FFF7F0FF204610BD421E2D
:105210005378521C002BFBD10B781370491C521C85
:10522000002BF9D1704730B505462A460B46107859
:105230001C78521C5B1C002801D0A042F7D0002C27
:1052400003D0002802D06D1CEFE7284630BDCAB25B
:10525000401E4178401C8A4202D00029F9D100202A
:105260007047421C0178401C0029FBD1801A70470E
:1052700010B5002200E0521C835C8C5CA34201D17B
:10528000002BF8D1D8B2E1B2401A10BD30B50446B7
:105290000020034600E05B1C934203D2E05CCD5C3F
:1052A000401BF8D030BD03460A780270401C491CF0
:1052B000002AF9D11846704730B50546002003464C
:1052C00000E05B1C934205D2EC5CC85C201A01D163
:1052D000002CF6D130BD70B506460CF025FA0468F6
:1052E00005460A220021304600F004FB2C6070BD08
:1052F00070B502464A40D50F40004A00ED0740080D
:105300005208002814D0002A12D0C40DD30D410237
:105310000120C0055202490A520AE41A091812185B
:105320007D34914201D3641C00E04900002C01DA75
:10533000002070BD0023914201D3891A0343400825
:1053400049000028F7D100290AD0914202D1012159
:10535000C90705E0914201D2012101E00121C943C1
:10536000E005C018401900F0FDFA70BDF0B5074621
:105370000846584087B0C00F049048000E465900B8
:1053800040084908BC1A884105D2384631461E46B5
:1053900017460B4602465800400810434CD0300DCB
:1053A000039040055900400D490D0590401A0290A8
:1053B000402872DA18030121000B09050843019007
:1053C00004980092002805D001995242002088419B
:1053D00000920190029840210A1A0199009800F069
:1053E000E3F905460C466B4607CB00F0EDF9C01912
:1053F0007141039A0E0D0023D71756401A467A4082
:10540000164344D0049A002A2DD0029A012A039A06
:1054100015DC1205C01A914101263605001C7141A8
:10542000D20F059ED2070093019202962A46234688
:1054300000F0E6FA07B0F0BD38463146FAE7160547
:10544000224A0F46B218C01AB74101210905001CB3
:105450004F4100187F41114618187941E20F10435F
:105460006D19644113E0E2076D0815436408C20733
:105470001443039A01261205C01A91413605001CF7
:105480007141CE07400830434908C01851412A46AF
:10549000234600F0A8FACDE7FFE704980122400078
:1054A000C117121A00238B4104983146C417381AC9
:1054B000A141EEE730B40124E407634030BC55E776
:1054C00030B40124E407614030BC4FE70000E0FF46
:1054D000F0B51FB488B00B99099800244840099989
:1054E000C00F490049080991C0070B990090490075
:1054F00049080B9109990898A64608431CD00B99B6
:105500000A98084318D0099801244000420D480029
:10551000410D099824050003000B204309900B98C6
:105520000003000B20430B9050181C494018002228
:1055300001901446104605E0002001460DB0F0BD74
:10554000032801DA034600E003239C46C11A0AAE91
:105550000AE05F0008ADED5B4F00F75B7D4300277D
:10556000AA187C41491C5B1E6145F2DD410004AB79
:105570005A522104120C0A43240C401C0828DFDB79
:10558000019802900099704601910090059B049A41
:105590000799069800F034FAD0E700000DFCFFFFF1
:1055A000F0B50C465C4085B0E40FE40703944C0072
:1055B0000026640859009446490802460296224390
:1055C00021D062460A431ED06200570D4A000E03E6
:1055D0002303550D012402462C492405781B1B0B7F
:1055E000360B401823432643614600901C46501A50
:1055F000B44103D30098401C009002E09218009838
:105600005B41002803DA0020014605B0F0BD002010
:10561000012109050746864611E064461D46141B14
:10562000B54106D36546521BB341744607430C434C
:10563000A646CD0740084908284392185B41054615
:105640000D43EAD11046184313D060461946504026
:105650007140084306D06046101AB34106D20122B9
:10566000002306E000220123DB0702E00122D243EF
:105670005310009874460105381C6141029C039D3B
:105680000019694100F0AFF9BFE70000FD03000019
:1056900010B500229623114600F06CF910BD0000F1
:1056A0000EB505490291002100910A460B46019171
:1056B00000F0A6F903B000BD330400004100400231
:1056C0000122400AD205090E80187F2901DA002044
:1056D0007047962903DC9622511AC84070479639C4
:1056E000884070474A0009030123090B1B05194331
:1056F000094B10B5520D9A4201DA002010BD064B3D
:1057000034339A4203DC9A1AFFF74CFD10BD03496B
:105710005118884010BD0000FF030000CDFBFFFFC3
:10572000C20FD207400040080BD0C10D0723DB0198
:10573000C91840020905400A1143C2084007114335
:10574000704700200146704710B5002904DB012492
:10575000E40740428C412146002B04DB1C46012318
:10576000DB075242A341994200D1904210BD000094
:10577000CB0FDB07490010B5490802460A4307D0A2
:105780000A0D07240903E401090B121B002A01DC9E
:10579000002010BDC900440F0C43C100E018D20521
:1057A000801800F0DFF810BD10B5202A04DB014698
:1057B000203A9140002010BD914020239C1A0346BE
:1057C000E3401943904010BD10B5202A06DBCB17EB
:1057D0000846203A1041C1170B4306E00B4613411F
:1057E000D0402024A21A91400843194610BD3A28FF
:1057F00000D23038202302469A43412A01D3104672
:105800003738884201D30020C04370474268002ADD
:1058100008D001680B78491C002B03D0521E06C02B
:10582000184670470121C160881E70474268002AEF
:105830000BD0C3680168002B07D183688B4204D06A
:10584000491E521C06C0002070470020C04370470C
:105850000FB400B589B00CA900910B990023CB605F
:10586000204B214A06930792042201921F4A02927A
:105870001F4A089202466B46002000F0E2F909B088
:1058800008BC04B0184770B586B006460020C04377
:105890000190002015460C4600910291049032467A
:1058A000694604A8FFF7D4FF024604982118002D8A
:1058B00005D0002801D0084600E020462860049862
:1058C00000280DD0002A02DD0098884208D0081B6D
:1058D0000190009432466946029404A8FFF7B8FF8D
:1058E00006B070BD0D5800082D580008FFFFFF7F5F
:1058F000115B0008F7B5009C0F4600262578641C54
:10590000002D05D000F000F90068405DC007F5D11A
:105910002B2D02D02D2D18D0641E39462046029A18
:1059200000F0BAFA002F04D03968A14201D10099E1
:1059300039607105022400290BDA4042002803DD9A
:105940000BF0F2FE0460A007FEBD012080020643BA
:10595000E3E70028F8DA0BF0E7FE04600048FEBD3C
:10596000FFFFFF7F002904DA401C490001D14008F5
:105970004000704770B40024050C05D110240004C9
:1059800002D1002921D01124050E01D100020834D2
:10599000050F01D10001241D850F01D18000A41C39
:1059A000002801DB4000641C002908D020252E1BA4
:1059B0000D46F540A14000D00121294308430106CE
:1059C0001B1B000ADB1D02D5002070BC7047DB05E5
:1059D000181880180029F8DA401C4900F5D170BC6D
:1059E00040084000704710B5002B08DA0024401C26
:1059F000614192185B411A4301D14008400010BD3B
:105A0000F0B51FB482B005460C0003D008460BF079
:105A10002DFE02E00BF02AFE2030024600902146C7
:105A20002846FFF7C1FE049B059A04460F4618431B
:105A30001143084314D0184610431BD0009840214E
:105A40000A1A18460599FFF7ADFB05460E46009A5F
:105A500005990498FFF7A8FE084305D0012004E04B
:105A60002046394607B0F0BD0020C11705430E435C
:105A70002C43374300990E986305401A7905E40AD0
:105A800000220C43FD0A0A3002D500200146E9E756
:105A90000105101969410C9C0D9D00196941FFF722
:105AA000A2FFDFE74A0009030123090B1B05194385
:105AB0000A4B10B5520D9A4202DA0020014610BD81
:105AC000064B34339A4203DC9A1AFFF76BFB10BD86
:105AD000034BD218FFF768FE10BD0000FF03000063
:105AE000CDFBFFFF064C0125064E05E0E36807CC21
:105AF0002B430C3C98471034B442F7D3FFF7E4FA39
:105B0000084001082840010800487047783401081F
:105B100010B50446FFF7F8FF0068005DC007C00F2E
:105B200010BD0000FFB5087889B01546FF2805D0E4
:105B3000491C2D2804D00022002407E000240BE09B
:105B40000122F9E70A235C430419491C0878FF285D
:105B5000F8D1002A00D06442002004902A7801463F
:105B60002D2A01D02B2A0FD16D1C2D2A02D0002204
:105B7000049209E00122FBE700260A2233466D1C4D
:105B800000F0DDF9381871412F78FF2FF4D10C9A0D
:105B9000A218069202460A4304D0FF23069A9133C4
:105BA000DA4205DA002109980A4606C00DB0F0BDB8
:105BB0000024B74AB54D2646079200F0FDF9029041
:105BC00006980391002801DA474200E007463905AC
:105BD0000020AF4A001C51410191009012E0F807EB
:105BE00007D022462B4630460799FFF771FC064640
:105BF000079122462B4610461946FFF769FC0446DA
:105C00000D467F10002FEAD10698019B0028009ACC
:105C10000399029806DAFFF7C3FC3246079BFFF7A9
:105C2000BFFC05E0FFF754FC3246079BFFF750FC32
:105C3000049A002A02D00122D2075140099A03C2D5
:105C4000B4E7FFB591B0002009900025ED432E2068
:105C50009E685C681F460190B9696D1C1298884760
:105C60000090396A88470028F6D10098401C0AD075
:105C70000D20C0018443002E12DD00982B2809D08E
:105C80002D280DD103E00020C04315B0F0BD012048
:105C900080020443B9696D1C12988847761E0090F3
:105CA00003A9600501D52D2000E02B206A46107362
:105CB000491C0CA80F9102900AE0B9696D1C12985A
:105CC000884700900120400204431398761E056027
:105CD000002E02DD00983028EFD00199009888420C
:105CE00046D18020044308E00998401E0990012015
:105CF000400204431399681C0860B9696D1C761E44
:105D00001298884700903028EED031E001998842FF
:105D100005D1200603D480200443761E1EE000989F
:105D20000BF0A4FE002826D001204002044307A95E
:105D30000F980331761E88420BD200980F993038A5
:105D400008700F98401C0F90200607D50998401E38
:105D500003E0200602D40998401C0990A00502D552
:105D60001399681C0860B9696D1C129888470090E7
:105D7000002ECBDC59E0002E57DD0098652801D0BD
:105D8000452852D1A00550D5032000028443B969AB
:105D90006D1C761E129888470090002E0CDD2B2873
:105DA00004D02D2808D1FF2001300443B9696D1CAF
:105DB00012988847761E0090E00501D52D2100E05D
:105DC0002B21029801700298401C0290019025E05E
:105DD0000120400204430EA902980131761E884238
:105DE0000ED20098029930380006000E087003D1D8
:105DF0000299019881420AD90298401C029006E05B
:105E0000E00501D5234801E0224840420990B969E4
:105E10006D1C12988847009013980560002E04DDD1
:105E200000980BF023FE0028D2D1F9691298884718
:105E30000F99FF200870029903AA087000200A90A9
:105E40000B900CA90AA8099BFFF76CFEA00502D4D1
:105E50000120C04319E72420044209D0E00713D1F0
:105E600038680B9A0A99031D3B60006806C00BE076
:105E70000B990A98FFF77CFC0146E00704D13868CB
:105E8000021D3A60006801602846FEE600001440EA
:105E90000000F03FF1D8FFFFF7B582B0029C002769
:105EA0002078641C15460197302802D0002D15D0AB
:105EB00015E020780127641C782804D0582802D0E7
:105EC000002D09D00BE0002D01D0102D07D10027A7
:105ED00010252078641C02E0082500E00A25002631
:105EE000009610E00099012769430818020C294622
:105EF00080B2714300908E183804864201D301208D
:105F000001902078641C2946FFF771FC0028E9DA2B
:105F10000398002805D0002F01D0641E00E0029CE9
:105F200004600198002806D00BF0FEFB02210160FE
:105F3000C81E05B0F0BD009930040843F9E7F0B57C
:105F40001FB486B000200090019002900698069938
:105F500080B204900798090C0204001411430790C2
:105F60000027089D099806913E463C4603900398F9
:105F7000A9B20204000C039004982D0C1543484369
:105F800000212246FFF710FCC719714110340E465C
:105F9000402CECDB3846029AFFF706FC009A019B86
:105FA00080180090594102980191103002904028C9
:105FB000CCDB00980BB0F0BD0EB5054A0292002272
:105FC000009213460192FFF71BFD03B000BD0000D5
:105FD0003304000070B58C180578401C6B075B0F0C
:105FE00001D10378401C2A1106D10278401C03E03D
:105FF00006780E70401C491C5B1EF9D12B0705D496
:106000000023521E0DD40B70491CFAE70378401C84
:10601000CB1A921C03E01D780D70491C5B1C521EAC
:10602000F9D5A142D8D3002070BD000038B5044690
:10603000064805490068FFF75BF8604300E0401E32
:1060400000900028FBD138BD40420F00A400002082
:10605000F8B50446006881688907890F012902D1D3
:106060000168C90727D18168144A1026114001250B
:10607000002913D18168294381600120FFF7D6FFF1
:1060800003F040F8074611E003F03CF8C01B0A2873
:106090000CD920680068C043C00707D0606D30434A
:1060A0006065A06D2843A0650120F8BD20680068E8
:1060B000C043C007E8D10020F8BD000017000080F1
:1060C000F7B58EB00D4630224A4901A8FFF77BF89C
:1060D0000E98494C8068372D416B09680D91E7692E
:1060E0001DD019DC444A0C23D26900215A4301AB6C
:1060F000D618042D2BD008DC002D18D0012D20D06F
:10610000022D24D0032D38D121E00E2D57D00F2D94
:1061100064D0362D31D102E0383D072D2DD81098AE
:10612000002F4FD0012F51D0022F5CD152E0E161FE
:106130002162019A029904F0C3FE206A401C206289
:1061400051E004F0E1FE0D9806F00AF94BE02A4A0E
:10615000D7697F1C042D0DD0B268022D10D0022506
:106160002A4217D0E7612162042F0BD32149002274
:10617000503917E0327A5207F4D4012011B0F0BD43
:106180000125EDE70C214F43F918DA59496804F06D
:1061900097FE28E0206A401C2062032806D3154998
:1061A0000022A0390E9805F0E9F91CE00E200090BD
:1061B000124A00210E9B0D9805F0C6F913E09A587B
:1061C0007168E4E703C807F043FB0CE003C807F07D
:1061D00055FB08E003C807F02FFB04E0002007F0A0
:1061E000DDFA012801D00020C8E702490022B039B9
:1061F0000348D8E778310108C000002010270000CC
:1062000060100020FEB5074680680A46416B384C96
:106210000968019100250E26A378032A61D007DCC6
:106220003449002A0CD0012A12D0022A06D115E0E6
:10623000042A28D00E2A40D00F2A4DD00120FEBDBE
:10624000032061610AF0CAFEA570E56025612BE0BC
:1062500004F05AFE019806F083F842E0012B0DD0BD
:106260002561E168491CE1601ED0E12162690903F2
:106270008A4229D10121A1701FA221E0032061617E
:106280000AF0ACFE10E02069E560401C20610528A2
:1062900007D00A2808D91D490022384605F06EF9B2
:1062A0001FE0E1210903E9E77D223B46D2000021FE
:1062B0000096019805F048F913E0012B04D014A2D0
:1062C000154904F0FDFD0CE00321002007F076FAEB
:1062D0000E4900222031E0E7002007F05FFA012894
:1062E00001D00020FEBD0949002210390B48D5E736
:1062F000C000002000C2010041542B4950523D31E2
:1063000031353230303B26570D0A0000D8300108B5
:10631000415445300D0A0000881300006010002031
:1063200038B504468068164B022915D004DC0029D4
:1063300008D0012904D10CE003290DD00A2911D07D
:10634000012038BD516819600EA2114904F0B8FD52
:1063500014E004F0D9FD11E000222046196805F090
:106360000DF90BE00020009003CA6B4609A206F06D
:10637000C5F9022802D1009807F09EFA002038BD26
:106380004C01002041542B4353510D0A00000000E2
:10639000881300002B4353513A2025642C252A0DE5
:1063A0000A0000001CB500230093C26B52680192E2
:1063B000C06B42685168044A936051606A46024962
:1063C00005F0DCF800201CBD5001002010B504468B
:1063D00007F06AFA012802D00020C04310BD204611
:1063E000FFF7E0FF002010BD10B5044680680029CB
:1063F00007D001290AD002290BD0032909D0012096
:1064000010BD09A20B4904F05BFD0BE004F07CFD1C
:1064100008E00221084607F0D1F90022064920468B
:1064200005F0ACF8002010BD41542B4346554E3DBD
:10643000300D0A00881300001831010800B5E1B0E2
:10644000FF21813168460BF0FBF8684604F048FFF5
:10645000002061B000BD000010B594B00021684676
:10646000417202210172234803904802049022489D
:106470000590642006900820079002A903200AF0E6
:1064800033FD0024E443002820D11C4805F07CFFA4
:1064900000281BD11A4809901A480A9039200B90FD
:1064A00019480C9019480D9019480E9012488021F7
:1064B00064300F9080301190104810911291139019
:1064C00009A9144804F04CFD002802D0204614B05D
:1064D00010BD01210F48019100900F4B0FA21149EF
:1064E000074804F0F1FF1049054805F025F80020A1
:1064F000EDE70000640A0020640E0020B8000020D0
:1065000060100020E02D0108F9720008BD74000839
:1065100061730008C80F0020A82F010841495237B5
:1065200038304500A83001083D64000810B5054921
:106530000869002803D0898A012202F0DCFD0020CE
:1065400010BD00004810002010B50549086900285A
:1065500003D0898A002202F0CEFD002010BD000089
:1065600048100020C3000348C15018188280002042
:10657000704700004810002010B505490868002841
:1065800003D08988002202F0B6FD002010BD000073
:106590004810002010B505490868002803D08988F4
:1065A000012202F0A8FD002010BD000048100020CC
:1065B00010B503468068154C002907D001290CD07E
:1065C00002290DD0092918D0012010BD0021A16396
:1065D0000FA2124904F074FC15E004F095FC12E0DF
:1065E000A06B012805D00E490022184604F0C6FF12
:1065F00009E00B4900223031F7E7044B03CA383376
:1066000008A206F07BF8002010BD0000C0000020AA
:1066100041542B43474154543F0D0A008813000056
:10662000283101082B43474154543A202564000087
:10663000F0B599B00C460646202110A8FEF7DCFD07
:10664000B5683C22686B5649076801A8FEF7BBFD98
:1066500007F076F8052253A10090FEF72DFE0028E2
:106660001CD0052251A10098FEF726FE002815D067
:10667000052250A10098FEF71FFE002810D0052229
:106680004EA10098FEF718FE002807D005224DA164
:106690000098FEF711FE002804D008E04BA202E0AB
:1066A0004CA200E04DA2202110A806F01AF9002209
:1066B0004C4801A9032C3DD006DC002C0BD0012C4A
:1066C00015D0022C69D119E0042C17D00E2C5ED005
:1066D0000F2C62D158E00263426304462846019AB7
:1066E000029904F0EDFB606B401C60634CE02846AF
:1066F00004F00AFC384605F033FE45E0042C04D0D3
:10670000022C0FD0032C15D02BE0036B0C245C4320
:106710006418247A640740D5426314E020490022BB
:10672000603925E0036B0C2463435B181B7ADB079D
:1067300007D116E0036B0C2463435B181B7A9B079D
:106740000FD54263036B5B1C0363052BE6D20C2061
:106750004343CA585818416810AB284604F0B0FBB0
:1067600012E0416B491C4163032905D31E490022F5
:10677000304604F003FF07E00E20009033461B4A2A
:106780000021384604F0E0FE002019B0F0BD006B97
:106790000C2250430A584018DDE70120F5E70000BD
:1067A000A831010834363030300000003436303043
:1067B00032000000343630303100000034363030E2
:1067C000360000003436303033000000434D4E4573
:1067D00054000000554E494E4554000043544E4568
:1067E00054000000C0000020A8300108102700005D
:1067F00010B58268002912D0012910D00F2901D0CC
:10680000012010BD07490B78012B03D0104600F082
:10681000F5FD04E000220A70034904F0AFFE0020F9
:1068200010BD0000C00000202831010808B50F2964
:1068300025D006DC002922D0012908D0042904D162
:1068400008E01A290BD0272916D0012008BD08F02E
:1068500085FE14E000220B4904F090FE0FE00020BA
:10686000009003CA6B4608A205F048FF012806D134
:10687000009808F053FF02E0094901200870002049
:1068800008BD0000B83001082B51495552433A2049
:1068900022636C6F736564222C25640D0A0000006E
:1068A000C000002010B58068002907D0012905D05C
:1068B0000F2901D0012010BD00F082FD002010BD85
:1068C00010B5002909D0012907D0042901D00120E1
:1068D00010BD0022024904F051FE002010BD00004E
:1068E000B830010810B504468068324B9AB00229CE
:1068F00016D004DC002909D0012904D10DE00329B8
:106900000ED00B2912D001201AB010BD51681960A9
:1069100029A22E4904F0D4FA4AE004F0F5FA47E03F
:1069200000222046196804F029FE41E000201446A8
:10693000189016901390149015900790129003CC15
:1069400018AB23A2083C05F0D9FE012830D11898D5
:1069500000282DD112AB069307AA15A914A803ABE2
:1069600007C310AA13A816A900920191029003CCA4
:106970000EAB1BA205F0C2FE092819D110980BF02E
:1069800029FC099108900E980BF024FC0B910A90B9
:1069900068461699018608A8139981741499C174E0
:1069A00015990175079941751299817506F0E2FEF6
:1069B0000020A9E78C01002041542B434950475344
:1069C0004D4C4F433D312C310D0A0000881300001F
:1069D0002B43495047534D4C4F433A202564000008
:1069E0002B43495047534D4C4F433A20252A2C25E1
:1069F000702C25702C25642F25642F25642C25648C
:106A00003A25643A25640D0A000000001CB50023F5
:106A10000093C26B52680192C06B42685168044A8D
:106A2000936051606A46024904F0A8FD00201CBD35
:106A30009001002010B5044606F094FE012802D013
:106A40000020C04310BD2046FFF7E0FF002010BD2E
:106A500010B504468068002907D001290AD0022910
:106A60000BD0032909D0012010BD09A20B4904F065
:106A700027FA0BE004F048FA08E00321022006F0B0
:106A80009DFE00220649204604F078FD002010BD3E
:106A900041542B4346554E3D310D0A0088130000EA
:106AA0002831010810B50446002905D001291DD060
:106AB0000F2908D0012010BDFFF75EFD0221002044
:106AC00006F07CFE12E0002006F068FE012803D1EB
:106AD0000221002006F072FE002006F067FE012869
:106AE00004D100220249204604F048FD002010BDD8
:106AF000D8300108F7B582B002980E268468274D79
:106B0000606B00290068019008D0012915D00E297A
:106B100016D032293FD0012005B0F0BD0027E76232
:106B20002169204688470028FAD0E7626F70FFF796
:106B300023FD00961A4A029B23E005F011FC2AE08F
:106B400068787D24E400002806D0012809D00228B6
:106B50000FD003281FD119E001206870FFF71AFD3C
:106B600003E002206870FFF7E1FC00962246029BDA
:106B700007E003206870FFF7E7FC1922029B0096EC
:106B800052010021019804F0DFFC04E000220549D5
:106B9000029804F0F3FC0020BEE70000C0000020D3
:106BA000B80B0000E830010800B585B0002923D0FB
:106BB000012921D0042904D0352907D0012005B0AE
:106BC00000BD00220D4904F0D9FC15E00020029020
:106BD0000390049003A904A80191009003CA02AB9A
:106BE00007A205F08BFD032806D102AB07CB08F006
:106BF00067FE029808F006FE0020E0E7B8300108C2
:106C00002B524543454956452C25642C25643A0DA5
:106C10000A256500002903D0012901D00120704711
:106C20000020704770B5054684680B000AF04DFDE2
:106C300005040D1111111C0006F090FD03460BA276
:106C40000C49204604F03CF90CE0204604F05CF9C5
:106C500008E0104606F0EEFD07480022416828468D
:106C600004F08CFC002070BD012070BD25730D0A5E
:106C70000000000088130000FC000020FEB58668BC
:106C80000346706B3F4F00680190012500203C795E
:106C900007294DD006DC00290CD001290DD002298E
:106CA00006D111E008294AD00E2951D00F2960D011
:106CB0000120FEBD3871B8624FE0304604F024F97F
:106CC000019805F04DFB5AE02E4A916A526A491C20
:106CD000002C02D0012C0ED051E07871012A07D08F
:106CE000052A05D0B962642919D90022264912E083
:106CF0003D71B86235E07871012A04D0052A02D0CE
:106D0000B962F8620BE0F86A401CF862032806D307
:106D10001D4900228031184604F030FC2FE00E207F
:106D20007D22009012010021019804F00DFC26E064
:106D3000002C24D1134B03CA243314A205E0012CE8
:106D40001DD1104B03CA243314A205F0D7FC16E062
:106D5000002C02D0012C04D011E078627D7113A2C6
:106D600002E078627D7114A21649304604F0A8F85A
:106D700005E07879002802D1304600F021FB0020A0
:106D8000FEBD0000C0000020B83001082B43524572
:106D9000473A20252A2C2564000000002B43475247
:106DA00045473A20252A2C256400000041542B43F6
:106DB0005245473F0D0A000041542B434752454777
:106DC0003F0D0A00881300007FB505468068214CFE
:106DD00037292BD00CDC02291FD004DC002912D06B
:106DE00001290DD116E0032917D0362908D11DE05D
:106DF00038291BD0392919D03A2917D03B2915D069
:106E0000012004B070BD1346A26013A2174904F01C
:106E100057F81DE004F078F81AE0A06808F07EFC4E
:106E200000221349284604F0A9FB11E0002003903A
:106E300001A8009003CA03AB0EA205F05FFC022874
:106E400006D10FA1029A0198FEF736FA0028E4D085
:106E50000020D6E73401002041542B434950434CD5
:106E60004F53453D25640D0A0000000030750000B9
:106E70005831010825642C2025700D0A00000000FF
:106E8000434C4F5345204F4B00000000F7B584B0F2
:106E9000049800268568474C686B36290068039083
:106EA00010D00CDC02297ED004DC002915D0012989
:106EB0007DD134E0032939D00E2978D16EE03739FD
:106EC000042974D801A80396009003CA03AB3AA220
:106ED00005F014FC022866D134E01046226008F068
:106EE000E5FB0746206808F0D1FB0646206808F05D
:106EF00007FC012811D033A06946C1C132A23A492A
:106F00002846236803F0DCFF0E200090374A00215A
:106F1000049B039804F018FB45E035A0ECE72846F5
:106F200003F0F2FF039805F01BFA3CE0206808F03C
:106F300013FC6068401C606003282FD300222D4999
:106F400066602DE02068039988422CD12AA1029A1C
:106F50000198FEF7B1F900280ED02BA1029A0198F2
:106F6000FEF7AAF9002807D02AA1029A0198FEF795
:106F7000A3F9002805D016E06660206808F006FC3A
:106F80000CE0206808F0E8FB6068401C60600328A3
:106F900004D303206060206808F066FB21490022CA
:106FA000049804F0EBFA002007B0F0BDFFE70120E1
:106FB000FAE700003401002025642C2025700D0A1A
:106FC000000000005544500041542B434950535495
:106FD0004152543D25642C222573222C22257322F4
:106FE0002C25750D0A0000008813000020BF020048
:106FF00054435000A8300108414C524541445920A7
:10700000434F4E4E45435400434F4E4E454354204C
:107010004F4B0000434F4E4E454354204641494C90
:1070200000000000583101087FB506468568002041
:10703000374C362910D00CDC022964D004DC00293E
:1070400015D0012962D126E0032929D010295DD16C
:107050002AE03739042959D8039001A8009003CABF
:1070600003AB2CA205F04AFB02284CD12BE01046C2
:10707000E26008F029FB002845D005F0E1FC206122
:10708000002840D04068009025A22A492846E3689D
:1070900003F016FF37E02061284603F035FF32E0A9
:1070A000E06808F03BFB29E003F0B6FF012803D1BC
:1070B000206903C804F060F920691F490CC82846FC
:1070C00003F02AFF1FE0E068039988421BD11BA14F
:1070D000029A0198FEF7F0F8002807D019A1029A49
:1070E0000198FEF7E9F80028DAD00CE0E06808F033
:1070F000EBFA002807D0216905F076FC002214493C
:10710000304604F03BFA002004B070BD0120FBE7DC
:107110003401002025642C2025700D0A0000000099
:1071200041542B43495053454E443D25642C25750D
:107130000D0A000088130000204E000053454E4405
:10714000204F4B0053454E44204641494C0000001F
:1071500058310108F8B50546002405F045F92046E8
:1071600008F0C0FA03281AD0204608F0BBFA042819
:107170001DD0204608F0B6FA052814D0641C032C54
:10718000EDDB1C4F03217869401CFDF7C7FF0C465F
:107190000026084608F0A6FA06280DD01EE00421B5
:1071A000204608F015FC22461349E86B12E012490C
:1071B00022461039E86B0DE0204608F085FA0028D9
:1071C0000CD005F03DFC002808D00B497C6122461C
:1071D0001031E86B04F0D2F90020F8BD0321601CE7
:1071E000FDF79CFF761C0C46032ED2DB0020C0432B
:1071F000F8BD00003401002004320108F8B58568AC
:10720000274E6A6B0B001468264AD7780AF05DFA9D
:1072100010090D1417212323232323232338232587
:107220003B230020D07090611EE0284603F06CFEE6
:10723000204605F095F82BE000221B491DE00E21A9
:1072400003467D220091D2000021204604F07CF903
:107250001EE0012FF0D00120F8BD012FECD0916984
:107260000A2907D2491C916110A23146284603F031
:1072700027FE0DE00C490022103104F07FF907E0F1
:107280000120D07004E0002006F088FA012801D027
:107290000020F8BD0449002240390748EDE700000E
:1072A00088130000C00000200831010841542B431E
:1072B00050494E3F0D0A00006010002010B50446F2
:1072C000022006F06BFA012802D00020C04310BD56
:1072D000084A00231360E06B416851604968183226
:1072E0009360516003491A46183104F047F90020B1
:1072F00010BD0000FC00002010B5032009F0A2FD25
:1073000010BD000005480649406804E0884201D1EC
:107310000120704740680028F8D1704760100020B5
:107320004831010810B50446022006F03FFA012852
:1073300002D00020C04310BD084A00231360E06B58
:1073400041685160496828329360516003491A4688
:10735000283104F013F9002010BD0000FC000020CB
:1073600070B50D4614461146284605F0ADF90128C2
:107370000DD1285D00280AD1002C04D0281920380E
:10738000C07F0A2809D0294605A003F0CDFF224678
:107390002946032009F0DCFE70BD294604A0F4E76D
:1073A0005B41542053656E645D2025730D0A000017
:1073B0005B41542053656E645D202573000000001E
:1073C00010B5044600F05CF8002815D02046FEF702
:1073D000FDFF002810D0204600F03EF900280BD019
:1073E0002046FFF76BFF002806D02046FFF79AFFE4
:1073F000002801D00020C04310BD000070B5054634
:1074000004F0F2FF0446284600F03AF800281BD0AA
:107410002846FFF79FFE002816D02846FEF7D6FF25
:10742000002811D02846FFF705FB00280CD0104893
:10743000104A8168611A914207D9846000220E497E
:107440000E4804F09BF8002070BD284600F004F9B7
:107450000028F9D02846FFF731FF0028F4D028464D
:10746000FFF760FF0028EFD00020C04370BD000090
:10747000C0000020102700006831010860100020C3
:1074800010B5002006F092F9012803D10321002055
:1074900006F094F9002006F081F9012802D00020BE
:1074A000C04310BD00220349034804F067F80020E0
:1074B00010BD0000C830010860100020FEB5044671
:1074C000002668460670002C12D0E06800280FD015
:1074D000606A00280CD02746A06A4D4D203700284E
:1074E00006D078E0E268694620469047002802D03E
:1074F0000020C043FEBD68460178E06A626A431C12
:10750000E3621154E16A606A4654E06A09280BD1CB
:10751000092240A0616AFDF7B9FE002804D10120CC
:10752000287001F0EFFDE8602878012803D00228D8
:1075300001D0032809D101F0E5FDE968401A384976
:1075400088424DD82878012809D0C0B20A2822D014
:10755000684600780D2823D00A2824D026E031A1DF
:10756000606AFDF760FE0290002834D0019601ABFE
:107570002DA2E16A606A05F0C1F8022830D10198B5
:1075800000282DD0626A0299891A0818C01CA860C8
:107590000A2028701FE0E16AA86881421BD11FE021
:1075A0000120387405E0387C012806D0387C022898
:1075B00005D0E06A01280ED109E002203874E06AA3
:1075C000022801D03E740BE0E6623E7403E0606A7C
:1075D00000783E2804D0A06AE16A401E814281D32F
:1075E000E16A606A05F070F801280CD1E06A0028B1
:1075F00005D0616A08182038C07F0A2806D00EA07E
:10760000616A03F091FE2E700020FEBD0EA0F8E727
:10761000A80000202B524543454956452C00000048
:10762000DC0500003A0000002B5245434549564511
:107630002C252A2C25643A005B4154205265637640
:107640005D2025730D0A00005B415420526563766E
:107650005D2025730000000010B5044606F0E2F836
:10766000012802D00020C04310BD084A0023136047
:10767000E06B41685160496808329360516003498A
:107680001A46083103F07AFF002010BDFC000020EC
:10769000F1B54948494984B00A7802724978417283
:1076A0000121C71D464CF971217D0173617D417334
:1076B0000026354668460BF036F804206946320E3F
:1076C0002D02154332020E5C1643401EF7D5A6620A
:1076D000E562E17814204143FF220498913250433F
:1076E00008187D21C90040180104C817891968418C
:1076F0000206080A1043E0610BF047F8E069002534
:1077000041084900080E0902216360632A48E36AC0
:107710002130A26A0BF0F2FA2748636B2530226B06
:107720000BF0ECFA24482749213089890181264849
:1077300021490078387021207872029800220007D1
:10774000000FF874C91D26200BF012F90021262025
:107750000BF020F901200BF071F8A0701B4801F02C
:107760009DFEE08164216170FF30913080B2012183
:10777000C9032082884201D3401A2082134801F0B5
:107780008DFEA081124E0AE0104801F087FE80B203
:10779000A081218A884202D38919884206D3002118
:1077A0000F200AF081FFA0610006EDD50948217A7B
:1077B000455405B0F0BD0000FD39002090000020C8
:1077C000500300201036002094000020F006002016
:1077D000983A0000303B002010B5064C2079401C40
:1077E000C0B22071642804D90020207100F082FE0C
:1077F000607010BD0000002010B500231A4603E0A1
:10780000845CE3189BB2521C8A42F9D3D84380B2FD
:1078100010BD0000F1B50024084E094D09E06000DC
:10782000811902226846FDF731FD002804D0641C4E
:10783000A4B2687A8442F2D32046F8BD583B0020B7
:10784000500300200148407870470000B401002038
:1078500000B587B01C216846FDF7CEFC01216846C3
:107860004170022101700D480190C8010290C000D2
:107870000490402005906946002009F035FB074838
:107880000749203801610749C161074981610749FA
:107890004161074804F040FC07B000BD402B0020C8
:1078A000D9790008CD790008097A0008177A00080C
:1078B000A02500207CB5444C607800280AD0002523
:1078C00001280AD00126022833D0032804D16846B3
:1078D000057060E004F094FB7CBD6846057001A96A
:1078E0000220019509F0EEFA7D26F6000AE06846CE
:1078F000007803280DD0656033460122694601985F
:1079000003F09BF96946002009F09CFA0028EED0AC
:107910007CBD6068002808D004F066FD6168401AEC
:10792000C828E9D900206070E6E704F05DFD6060DA
:10793000E2E76846057001A90220019509F0C2FA44
:1079400008E06846007803280BD0A56068460078F8
:1079500009F0EAFC6946002009F074FA0028F0D02A
:107960007CBDA068002809D004F03EFDA168401A43
:10797000C828EBD9A67000206070E7E704F034FD5A
:10798000A060E3E76846007803280BD0E56068460E
:10799000007809F0C9FC6946002009F053FA002874
:1079A000F0D07CBDE068002809D004F01DFDE1683E
:1079B000401AC828EBD9A67000206070E7E704F0F1
:1079C00013FDE060E3E70000B401002010B50146BC
:1079D000002009F037FA10BD0FB400B5FFB082B037
:1079E000012183AB49026846829A09F029FE684664
:1079F000FDF737FC02466946002009F0A9FB7FB07D
:107A000002B008BC04B0184701B501226946002045
:107A100009F09EFB08BD10B50446FDF722FC0246A6
:107A20002146002009F094FB10BD00000149487078
:107A300000207047B401002010B5024801F050F852
:107A400010BD0000040A002010B5034801F048F8FA
:107A5000024801F045F810BDBC090020740900205F
:107A600030B5446C1C252C400125A540046C656094
:107A7000046863608368102B036803D09960006812
:107A8000C26030BD9A600068C16030BD7D2100B524
:107A9000C900484300F001F800BD002140E000BFEC
:107AA00000BF00BF00BF00BF00BF00BF00BF00BFDE
:107AB00000BF00BF00BF00BF00BF00BF00BF00BFCE
:107AC00000BF00BF00BF00BF00BF00BF00BF00BFBE
:107AD00000BF00BF00BF00BF00BF00BF00BF00BFAE
:107AE00000BF00BF00BF00BF00BF00BF00BF00BF9E
:107AF00000BF00BF00BF00BF00BF00BF00BF00BF8E
:107B000000BF00BF00BF00BF00BF00BF00BF00BF7D
:107B100000BF00BF00BF00BF00BF00BF00BF491CC7
:107B20008142BCD37047000010B506F0F9F920205F
:107B300007F05EFF01200AF00BFD002007F058FF60
:107B40000A480AF0A9FB012109480AF025FE094864
:107B50000AF034FE00200AF069FE7D20C0000AF021
:107B600037FE00200AF0E7FD10BD000040030020B2
:107B700000D023248380000010B5012001F0CCF94F
:107B800010BD10B50120400201F0C6F901208002AD
:107B900001F0C2F90120400301F0BEF910BD72B638
:107BA000FEE7000010B5084900224A6107494B680A
:107BB0004C1523434B604B68082423434B60C0099A
:107BC000C001026010BD00004C0A002000200240ED
:107BD0007FB500240D460646039401F0CBF8E80972
:107BE000029003A901960094684601F05BF80749EA
:107BF000002806D00120088001F090F8002004B091
:107C000070BD0C8001F08AF80120F8E7E001002047
:107C100010B5002302E0C45CCC545B1C9342FAD341
:107C200010BD000010B5214A00219069C30520480D
:107C300004D54169022319434161911593699B055C
:107C400005D54369012423434361630219439369C2
:107C50005B0505D54369082423434361E3011943C8
:107C600093691B0505D543690424234343616302DB
:107C7000194393699B0405D5436910242343436149
:107C80006302194393699B0304D5446920231C4371
:107C9000446119439369DB0305D5436940242343B9
:107CA0004361A0020143916110BD00000020024029
:107CB0004C0A002070B5054601F024FA0646184C1F
:107CC0000AE0681C08D0002D04D001F01BFA801BCC
:107CD000A84201D9032070BDA069C007F1D1A069F5
:107CE000800701D50220A061A069C00511D4A06958
:107CF00080050ED4A06940050BD4A069000508D406
:107D0000A069800405D4A069800302D4A069C003DF
:107D100003D5FFF787FF012070BD002070BD000074
:107D200000200240F8B51746002605460C4601F033
:107D300021F80BE029460220226800F0FDFF0849E7
:107D40000028488004D1241D2D1D361DBE42F1D3CC
:107D500000F0E4FFBE4201D20020F8BD0120F8BDD2
:107D6000E00100200FB4F8B504460D460026002CB3
:107D700004D1401EF8BC08BC04B01847E06A0028D3
:107D800000D1F7E709A80090E76A29462046009B42
:107D9000089AB8470646002000903046EAE7FFB54B
:107DA00004460D46002100260023214600BF11E0B5
:107DB000D8001150D80080184660D80086185B1C87
:107DC00068684F68B84204D103980660002004B088
:107DD000F0BD49680029EBD1481EF8E7F8B5054623
:107DE000002600272E0CAFB20848046809E020885E
:107DF000B04205D100223946204603F001FB02E0E3
:107E00006469002CF3D100BFF8BD0000C803002056
:107E100070B502210B4801F069F90B490B4D0028A0
:107E200005D001200870A88A401CA88270BD0024DB
:107E3000074E0C703078022801D101F0A5FB347098
:107E4000AC8270BD000400500A0200200000002037
:107E50003A03002010B5827F5118C9B281771829E2
:107E600014D318398177417F0122491CCCB2447761
:107E7000017F0B0009F029FC0D0A080B08190819ED
:107E800008081908191E0A001F2C10D810BD817E81
:107E90008B070321002B03D01C2CF7D9427702E07B
:107EA0001D2CFBD810BD017710BD1E2CFCD94277CC
:107EB000491CF8E71F2CF7D942770277418B491C00
:107EC000418310BD10B5054B64220549054802F0F9
:107ED000B4FE9620FFF7DAFD10BD0000B80B0000DD
:107EE0002C0000206408002010B586B003AA009280
:107EF00001AB0FA204F002FC0024E443022811D1DC
:107F00000499039804F091FBC3B20198012102780F
:107F100003E00198405C4240491C02988842F8D82E
:107F20009A4202D0204606B010BD0020FBE70000B8
:107F30002425702A25700D0A0000000010B588B0B5
:107F400000F066FA164C0122A188206801F0D3F8EF
:107F50000A2000F095FEA1880022206801F0CBF8ED
:107F60000A2000F08DFEA1880122206801F0C3F8EC
:107F7000002069464870022008700A4901914102B8
:107F8000029109490391042104910590694608F082
:107F9000ABFF20468821103004F026FB08B010BD4E
:107FA000B8230020B81F0020AC010020F3B52C48F6
:107FB00095B001270770282108A8FDF71DF9294C65
:107FC0002948A178FDF718F916991598FFF78CFF45
:107FD000BD1E002807D112AB24A21699159804F0F3
:107FE0008DFB0F2802D0284617B0F0BD1298FDF780
:107FF00072F9C0B26070159A169900255618203E85
:10800000002828D02369002B03D00A4600201599A8
:108010009847112121480902016021480770F5772E
:10802000B5772048E178007805901F4803950495BE
:10803000069101781D486A46808823C2FF211CA250
:1080400001310948159B04F04CFCE178491CE170B2
:10805000A0700020C8E71148056011480570DEE7F0
:1080600006000020A00100207824002024252A2CCE
:10807000252A2C252A2C252A2C252A2C252A2C2574
:10808000702C252A2C252A2C252A2C252A2C252A19
:108090002C252A2C252A2C252A2A00002000002005
:1080A000090200200A0200200100002010360020F2
:1080B00025732C25582C253032782C25782C2564D6
:1080C0002C25642C25642C25640D0A00F3B50025AD
:1080D0004468ED43066883B0092C0AD322462E215A
:1080E000304604F071FC070003D0B81B019004284F
:1080F00002D0284605B0F0BD0221304604F009FC4C
:10810000FDF7CEFA054600910221B01C04F001FCF7
:10811000FDF7C6FA029001980E46241A641E214605
:10812000781C04F0F6FBFDF7BBFA0E4F04E00022CA
:108130003B46FDF735FA641E002CF8D102460B468B
:1081400031460298FDF712F90022074BFDF728FA95
:108150002A46009BFDF70AF9049AD160906000203E
:10816000C8E700000000244000004E40F3B50025A1
:108170004468ED43066883B00A2C0AD322462E21B8
:10818000304604F021FC070003D0B81B01900528FD
:1081900002D0284605B0F0BD0321304604F0B9FBFB
:1081A000FDF77EFA054600910221F01C04F0B1FBB8
:1081B000FDF776FA029001980E46241A641E2146B5
:1081C000781C04F0A6FBFDF76BFA0E4F04E00022CA
:1081D0003B46FDF7E5F9641E002CF8D102460B463C
:1081E00031460298FDF7C2F80022074BFDF7D8F997
:1081F0002A46009BFDF7BAF8049A516110610020ED
:10820000C8E700000000244000004E40F3B59BB0DA
:108210000F465E4C1B98FFF767FE0026F6430025CD
:10822000002801D02576A0E010AB079313AA0EA971
:1082300015A804AB07C319AB03930CAA17A90AA886
:108240006B4607C308AB52A239461B9804F056FA96
:108250000D2872D10B980A9901286ED1087841280F
:1082600006D02576207E012805D000201DB0F0BD67
:1082700001202076F6E7089F2E213846099A04F05F
:10828000A3FB002871D0C01B06286ED102213846FE
:1082900004F03FFBA0770221B81C04F03AFBE07722
:1082A0000221381D04F035FB202108551198109F3C
:1082B00006285AD10221384604F02BFB60770221B0
:1082C000B81C04F026FB20770221381D04F021FBA6
:1082D0007D21090140186083214617A8FFF7F6FEAB
:1082E000002842D1214619A8FFF740FF00283CD1C1
:1082F0000F9F0E990A2F38D2002F0FD03A4603A8AD
:10830000FCF761FF03A8C55509F064FF2B4A2C4B0D
:10831000FDF7DEF8FDF7E6F9208000E0258028462D
:10832000149F139D002F0DD03A462E21284604F0AD
:108330004BFB002802D0411B01E016E039462846DD
:1083400004F0E7FA60800D980C9901280DD80028F8
:1083500007D00878532804D10122E068D2075040A2
:10836000E06016981599012801D930467EE700286B
:1083700007D00878572804D101226069D2075040FD
:10838000606108212046FFF765FD6EE7502400205C
:1083900024252A2C25702C25702C25702C25702C3A
:1083A00025702C25702C25702C25702C25702C25E3
:1083B0002A2C252A2C252A2A000000006F1283C0AF
:1083C000CAA1FD3FC3000248C150181882807047FF
:1083D000B823002008B500206946087003E068460D
:1083E000007800F023F86946022008F02BFD0028F1
:1083F000F5D008BD10B50549002008700122052000
:108400001103000700F077FE10BD0000A00100205E
:1084100010B505490120087001030520002200075E
:1084200000F069FE10BD0000A001002070B5224DD3
:1084300000262C462B78611C8034002B08D0224665
:108440005268022B0CD0032B09D10A2813D030E03C
:10845000242804D102222A7070540120606070BD6B
:1084600050546168491C61607E2922D20D28F6D1E2
:108470000320287070BD50546068401C60604654F2
:108480000EA1681CFCF7CFFE002808D0681C6168AC
:10849000FFF78CFD681C6168FCF7AEFE09E009A1DE
:1084A000681CFCF7C0FE002803D0681C6168FFF759
:1084B000ADFE2E7070BD0000C82300204747412C40
:1084C00000000000524D432C0000000010B5084889
:1084D00000F05CFA0A21064800F0F4F9044800F0C4
:1084E000DFF8800503D5024800F0DCF880B210BD4B
:1084F00084060020F8B5FFF7E9FFFDF7C9F8274E1D
:108500003146FCF7F5FE264C2649002520618842BD
:108510003EDB2078244F002815D02570FFF7D6FFCA
:10852000FDF7B6F83146FCF7E3FE2061FDF7F8F8F9
:1085300000223B46FCF7BEFF00221C4BFCF7C8FFA5
:10854000FDF716F9A0602069FDF7EAF800223B4626
:10855000FCF7B0FF164A174BFCF7BAFF06460F466A
:10856000A068FDF7DDF8124A134B5242FCF7B0FF4A
:1085700032463B46FCF7FAFEFDF7FAF80F49A060D9
:10858000884201DDA16004E0FF21C905C84200D393
:10859000A560A068FDF792F8C0B2F8BD00401B448A
:1085A000CC0100200000604000000C4000E064406E
:1085B0003333333333B33040CCCCEC3F0000C842CC
:1085C00010B50F4CA07800280FD1012149020D48A9
:1085D00000F08CFD002808D10B480078002804D159
:1085E000A079002802D00020607110BD6079401C85
:1085F000C0B260710528F8D900F0C6FF10BD0000B8
:1086000000000020000400503A030020F8B50646A0
:108610000D464036317C01290DD0012131740168AD
:108620008A68520709D5416D202211434165002017
:1086300030740120F8BD0220F8BD174B6A68D805D8
:1086400047109A42154C8A6A2B6812D05B035B0B69
:108650001A438A622968490305D5A1680143A160CC
:108660000A20FDF7E3FC2868800312D5A068384390
:108670000EE05B035B0B9A438A622968490302D5CB
:10868000A1688143A1602868800302D5A068B8432F
:10869000A06000203074F8BD0110000000270140E8
:1086A000406D70470068006C7047000070B50400B2
:1086B00006D0606D264600254036002802D006E030
:1086C000012070BDA5653574204600F0D3F8606DBB
:1086D000C00603D421688868400705D5606D102165
:1086E000084360653574EBE7606DFF22013290430B
:1086F00002221043606588688207920F5B48012A56
:1087000002D10A68D2072BD1032362689B079A42E1
:1087100005D05B429A4202D05B009A4209D10A69B5
:10872000920092080A6121680A6963681A430A6123
:108730000CE00A69920092080A6181680F22920493
:108740009143816081686268114381602168CA68D1
:1087500018239A43CA602168CA68A3681A43CA608A
:10876000816801225206914381608168A28E52067F
:108770001143816020688168C90004D481680122A6
:108780001207114381602068C168394A1140C160F5
:108790002069E168022825D00020014320462030CE
:1087A0000278037B52035B001A431143226B11438F
:1087B000A26992031143E269D20311432268D3688C
:1087C0001943D160616A0A46FF3AC23A05D0A26AEB
:1087D00011432268D3681943D16042780121012AEC
:1087E00002D00BE00420D8E70078002823D0606D89
:1087F000202210436065A06D0843A065E06B01284E
:1088000020681FD00169C90703D0016949084900E0
:10881000016120684169C908C90041612068416956
:10882000A26B11434161A565606D80088000401C0A
:108830006065002070BD2068C26801231B041A43D4
:10884000C260DBE70269FF239B009A430261206854
:108850000269236CA66C1A43636C33431A430261AA
:10886000206802690A430261D3E700000027014043
:108870001902FEFF10B586B0044614216846FCF7C5
:10888000BBFC0E492068884216D10D48416B421549
:1088900011434163C16A01221143C162C06A694642
:1088A00010400590022000900320019000200290CB
:1088B0000520000700F03CFB06B010BD002401407D
:1088C00000100240F8B504464069254640350E4682
:1088D00008280BD02068C068C00709D0606D20212F
:1088E00008436065002028740120F8BD082700E0D7
:1088F0000C2700F007FC009015E0701C13D0002E30
:1089000005D000F0FFFB0099401AB0420BD9206857
:108910000068384207D1606D04210843606500207B
:1089200028740320F8BD206800683842E5D0606DE7
:1089300001214902084360652068C16809058A0F62
:108940000C21002A1BD12022125D002A17D10268B7
:10895000120714D5826853070122002B08DB4368F5
:108960008B434360606D130298431043606506E0DB
:10897000606D202318436065A06D1043A065A06959
:10898000002801D1206801600020F8BD70B50446C0
:10899000216800208968490721D425464035297C73
:1089A00001291CD001212974E169012904D0204644
:1089B000FDF74EFB002811D1616D0A4A1140FF22DC
:1089C0000132114361650021A165297422681C21CF
:1089D000116021688A6804231A438A6070BD0220EE
:1089E00070BD0000FEF1FFFF30B5014620314A792D
:1089F0000023022A04D00422C2630B71012030BD7F
:108A0000026814680E25AC43146002681468640898
:108A100064001460446C1C22144001221546006C52
:108A2000A54045604A7118460B7130BD70B50024F1
:108A3000014620314A79022A03D00421C16301246E
:108A400018E0026813680E25AB43136002681368D0
:108A50005B085B001360436C1C2213400122154627
:108A60009D40036C5D604A7100220A71816B002990
:108A700000D08847204670BD70B5040029D020681A
:108A80000168490849000160134825681421281825
:108A9000FCF72EFB800060641048206400202860F2
:108AA000626C1C210A4001239340226C53600B4AE4
:108AB0008032936A656C0D400F21A9408B4393620D
:108AC000E06220636063A063E06320346071207122
:108AD00070BD012070BD0000F8FFFDBF0000024026
:108AE000F0B4016C0D6801680C68466C1C2304220C
:108AF0001E401746B7402F420ED067070CD50C68B2
:108B0000A40602D40C6894430C60416C19408A405E
:108B1000016C4A60016B1AE00227B74002462F4001
:108B20002032002F17D0A70715D50C68A40605D44E
:108B30000C680A25AC430C6001215171446C022180
:108B40001C40036CA140596000211171C16A0029C9
:108B500018D0F0BC08470827B7402F4212D024078E
:108B600010D50C680E25AC430C60446C01211C40F0
:108B70000B46A340046C6360C16351710021117105
:108B8000416BE4E7F0BC704770B504003CD01F486F
:108B9000256814212818FCF7ABFA800060641C4893
:108BA000206402212046203002464171296819487C
:108BB000E3680140A068666918432369334318439A
:108BC000A3691843E3691843236A184308432860DC
:108BD0000121A0688903884210D00D488030836A43
:108BE000656C1C210D400F26AE40B3438362656C5B
:108BF00063680D40816AAB400B4383620020E063F1
:108C000001215171107170BD012070BDF8FFFDBFD1
:108C1000000002400F80FFFFF8B504468C4620306C
:108C200001790025012909D0012606714179002723
:108C3000012905D0077102252846F8BD0220F8BD9C
:108C400002214171E7632068016849084900016019
:108C500061462046FEF704FF206B0028206801686B
:108C600001D00E2205E004229143016020680168D2
:108C70000A22114301602068016831430160DBE78B
:108C800070B5044600F03EFA0546601C02D0044868
:108C90000078241800F036FA401BA042FAD370BDC9
:108CA00098000020F8B51A4E0546307C0F46012882
:108CB00007D0012030741748FEF7FCFF010002D0F6
:108CC00021E00220F8BD0020C04338606C6814E049
:108CD0002046FEF767FF0F48FEF7ECFF01460E48FF
:108CE000426808239A434260426843159A434260AF
:108CF000002901D03C6006E08034A8686A68C001A1
:108D00008018A042E4D8002030740846F8BD000066
:108D10004C0A002050C30000002002400548416872
:108D20000222114341604168012211434160002049
:108D30007047000000200240F8B50C4C1646207C1D
:108D40000F46012808D0012020740948FEF7B2FF21
:108D50000025002802D006E00220F8BD65613E60D3
:108D60000348FEF7A7FF2574F8BD00004C0A002059
:108D700050C3000011484168C9070BD0EFF31081C0
:108D800072B60F4AC2600F4AC26081F31088416810
:108D9000C9070ED1416889070DD5EFF3108172B66E
:108DA000094A0261094A026181F31088406880071C
:108DB00001D50120704700207047000000200240CC
:108DC000EFCDAB8905040302BFAE9D8C16151413BD
:108DD000F0B5002262E0012393401C460C405CD0B9
:108DE0009608304DB6007519AF68AC4695072E0F42
:108DF0000F25B540AE463D4005273F07B84201D19B
:108E0000002719E0284FB84201D1012714E0274F6D
:108E1000B84201D102270FE0254FB84201D1032704
:108E20000AE0244FB84201D1042705E0224FB8429E
:108E300001D1052700E00627B740AF4212D11F4DF0
:108E40002E68A6432E606E68A6436E60EE68A64349
:108E5000EE60AE68A643AE606546AD687446A54355
:108E60006446A560056856000324B44025430560A8
:108E7000D508AD002D182E6AAC465507EF0E0F250C
:108E8000BD40AE4365462E62C568A543C5604568D2
:108E90009D4345608368A3438360521C0B46D340C7
:108EA00099D1F0BD000001400004005000080050BE
:108EB000000C005000100050001C00500004014045
:108EC00070B501229202054651100801114C9542DD
:108ED00003D1E089401CE08170BD8D4207D106F0CE
:108EE000FFFD04F06BFB208A401C208205E08542D8
:108EF00003D1608A401C608270BD012DFCD106F058
:108F0000EFFDA078012801D100F03EFB0020A081F8
:108F100070BD00000000002010B504494A690242FB
:108F200002D04861FFF7CCFF10BD000000040140F3
:108F3000F8B5002303240125C2E032462E469E40A8
:108F4000B446324079D00E79B607B60F012E01D063
:108F5000022E17D186682746B6465E00B7400096B7
:108F60007646BE43B646CF68009EB7407646374346
:108F7000876046686746BE430F79FF06FF0F9F4034
:108F8000374347600E79F643B6070ED0C6682746CA
:108F9000B4465E00B646B7406646BE43B4468F68E8
:108FA0007646B74066463743C7600E79B607B60FB8
:108FB000022E14D1DE08B60036180096366A5F0716
:108FC000B446FE0E0F27B646B7406646BE43B446CB
:108FD0000F697646B74066463743009E376206689B
:108FE0002746B4465E00B646B7406646BE430F7994
:108FF000B446BF07BF0F7646B740664637430760A3
:109000004E68B603B60F5AD0304F7E6B2E437E6348
:109010009F082F4EBF00BE190096B6680F27B446B2
:109020009E07360FB646B7406646BE4305273F0744
:10903000B446B84202D100271AE040E0254FB842BA
:1090400001D1012714E0244FB84201D102270FE0DB
:10905000224FB84201D103270AE0214FB84201D183
:10906000042705E01F4FB84201D1052700E006277D
:109070007646B74066463743009EB7601A4EB668DC
:109080004F689643FF0200D51643174FBE60FE6837
:109090004F689643BF0200D51643134FFE607E68AB
:1090A0004F689643BF0300D516430F4F7E603E685E
:1090B0004F689643FF0300D516430B4A16605B1CAE
:1090C0000A681646DA4000D037E7F8BD00100240C3
:1090D000000001400004005000080050000C005047
:1090E00000100050001C00500004014000690840BE
:1090F00000D001207047002A01D081617047816251
:109100007047000001488068704700009800002008
:1091100070B504000FD02168154808602168154813
:10912000086003CC41602068083C21688860FFF734
:10913000E9FF05460CE0012070BDFFF7E3FF401B8F
:109140002A2805D92068C068400701D0032070BDD7
:109150002068C0684007F0D120680269E1688A424F
:1091600001D0016101E004490160002070BD0000F0
:10917000CCCC000055550000AAAA000000680249A6
:109180000160002070470000AAAA00000248816820
:1091900002788918816070479800002010B508484F
:1091A00000240168402211430160032000F00AF806
:1091B000002801D0012401E000F0BAF9204610BDDA
:1091C0000020024070B504460D4D7D202978C00076
:1091D000FBF78EFF01460B480068FBF789FF01F0A3
:1091E000CDF8002809D1042C07D200222146401EC8
:1091F00000F0C6F900206C6070BD012070BD000059
:1092000098000020A400002070477047F8B506F0D1
:1092100067FCFFF7D5F904F01FFC01214902304833
:10922000FFF764FF012600252E4C002810D0208B6C
:10923000401C80B220832178884201D9E67100E089
:10924000E571E1218901884204D900F09DF901E02E
:109250002583E571012149022148FFF747FF224F8D
:10926000002810D0387800280DD1207A401CC0B2D8
:109270002072022807D92572A56265622562E56120
:1092800005F0A0F905E0E369226A616AA06A05F0C9
:109290007BF9FEF7BDFD6089401C6081608B401C3E
:1092A0006083A089401CA08106F026F9FEF794FA9D
:1092B000A0891E2801D9667200E065720121490269
:1092C0000748FFF713FF002808D13878002805D198
:1092D000A56265622562E56105F074F9F8BD0000DC
:1092E0000004005000000020080200207047704772
:1092F000704710B5044600680168C943C90708D122
:109300008168C943C90704D1012141602046FFF7A4
:109310007DFF20680168C943890708D48168C94373
:10932000890704D4022141602046FFF76DFF2068C1
:109330000168C943490708D48168C943490704D46F
:1093400004214160204600F0F1F820680168C9431B
:10935000090708D48168C943090704D4082141607A
:109360002046FFF7C3FF20680168C943C90608D437
:109370008168C943C90604D4102141602046FFF723
:1093800044FF20680168C943890608D48168C9433D
:10939000890604D4202141602046FFF7A9FF2068F8
:1093A0000168C943490608D48168C943490604D401
:1093B000402141602046FFF79AFF10BDF8B5040038
:1093C00005D025462035A87B002802D006E00120E4
:1093D000F8BD00206873204600F048F80220A8730A
:1093E0002068C26884466368012B04D00120A16A0A
:1093F000C005814201D11E20824319486169814222
:1094000001D0184802401848A66802401846304368
:10941000676A266A3E433043A66A30431043002BF6
:1094200018D0012B03D00122D205964203D1236923
:10943000E2681A4310430A4A914205D0A2691143D7
:10944000E2690243084610436146C8600120A873E0
:109450000020F8BD2369E2691A431043E3E70000E6
:10946000FFFF00003F1FFFFFFEF119FF10B500686E
:10947000084988420CD10848816BC20411438163BA
:10948000002211460D2000F07BF80D2000F06CF852
:1094900010BD0000007C0040001002400068C06960
:1094A00070470000F8B504460220254620351746CF
:1094B000A8731D480268C3041A4302602068C2688A
:1094C0009B121A43C260206802690126324302617E
:1094D000226810205060206881611021204603F02E
:1094E000F7FD03281FD021680820486020684761E5
:1094F0000821204603F0ECFD032814D0204603F099
:1095000071FDA87B03280ED02068816831438160FB
:109510002068016931430161206801690422114317
:109520000161AE730020F8BD0004014070470000E7
:109530000448416B012211434163816B02041143D2
:109540008163704700100240002809DBC106C90E84
:109550000120884003490860BFF34F8FBFF36F8F2E
:109560007047000080E100E0002805DBC106C90E5D
:1095700001208840014908607047000000E100E0D8
:1095800010B508F0AFF810BDBFF34F8F0449034882
:10959000C860BFF34F8F00BFFDE700000400FA056D
:1095A00000ED00E002480168821511430160704738
:1095B00000700040F0B5154A1368154D54152D6A1A
:1095C0002340ED07ED0F002B04D0002D02D01668CC
:1095D000A64316601668B608B600064316600D4826
:1095E000076904263743076101290DD040BF20BF1A
:1095F00020BF0169B1430161002B04D0002D02D0CE
:10960000106820431060F0BD30BFF2E700700040EA
:109610000000014000ED00E0F8B5044600780027A6
:10962000594D800674D5584E403EB06BC00004D4EE
:10963000B06BA9050843B063012754480168C90508
:1096400011D40168821511430160FFF75BFD0090A2
:1096500005E0FFF757FD0099401A642837D84B48BA
:109660000068C005F5D532680321090560680A4025
:109670000140914208D08103890F032904D1316848
:10968000890301D50120F8BD2A69032109040A4094
:1096900022D0084090421FD02078800631D528691A
:1096A0002A6988430121C9040A432A612A698A4335
:1096B0002A612861C0050FD5FFF724FD009008E05E
:1096C000FFF720FD0099411A3148814201D903205A
:1096D000F8BD28698005F3D52078800611D561682A
:1096E0008803800F032805D13268000582430140BA
:1096F0000A4332602869032261681204114008435A
:109700002861002F04D0B16B012000078143B163B1
:109710002078C00705D0E868A16880088000084369
:10972000E8602078800705D5E8680C218843E16867
:109730000843E8602078400706D5E86803218902DD
:10974000884321690843E8602078000706D5E86867
:1097500003210903884361690843E8602088C00544
:1097600006D5E868032109048843A1690843E86035
:109770002078000606D5E868032189048843E1695A
:109780000843E8600020F8BD40100240007000402F
:1097900088130000F8B50E46050038D05E48006812
:1097A000C007C00FB04214D25B4C20684008400094
:1097B00030432060FFF7A6FC074605E0FFF7A2FC58
:1097C000C11B564881427AD82068C007C00FB042FA
:1097D000F4D12878524C800705D5E068F021884301
:1097E000A9680843E0602878C00752D0686802285A
:1097F00006D0032807D0216801280AD0890504E093
:109800002168890301E021688901002903DB012027
:10981000F8BD4907F9E7E168890889000143E1607B
:10982000FFF770FC0746686802280AD0032814D0A6
:1098300001281ED029E0FFF765FCC11B3748814293
:109840003DD8E0680007800F0228F4D121E0FFF73F
:1098500059FCC11B3148814231D8E0680007800FB4
:109860000328F4D115E0FFF74DFCC11B2B488142C2
:1098700025D8E0680007800F0128F4D109E0FFF740
:1098800041FCC11B2548814219D8E0680007800FC0
:10989000F5D121480168C907C90FB14217D901683C
:1098A0004908490031430160FFF72CFC074608E0F6
:1098B00005E0FFF727FCC11B1848814201D90320AE
:1098C000F8BD15480068C007C00FB042F1D1287834
:1098D000400706D5E068072109028843E968084384
:1098E000E0602878000707D5E0680721C9028843AF
:1098F0002969C9000843E06000F03AF8E168094AC4
:109900000906090F515CC84007490860074800680C
:10991000FFF758FCF8BD000000200240881300004B
:1099200000100240BC2D0108A40000209C00002073
:10993000044805490068C968044A4905490F515C53
:10994000C8407047A400002000100240D52D010837
:10995000044805490068C968044A8904490F515CF4
:10996000C8407047A400002000100240D52D010817
:1099700070B51A4AD3681A490C2018408D00042883
:109980000CD04E00082810D00C2810D050680004CD
:10999000410F0120C003491C884070BD1068C006FB
:1099A00001D5084670BD284670BD304670BD98028E
:1099B0000C4C000F205C1B029C0FD368641CDB0363
:1099C00001D5314603E01268D20600D4294607F0DB
:1099D00064FE22460023FBF7B5FB70BD0010024079
:1099E00000093D00CC2D0108FEB505007ED0F74CE6
:1099F000E7680C20E668074001200004064028784C
:109A0000C00747D0082F05D00C2F0AD10120000431
:109A1000864206D1206880033CD568680028E5D0DE
:109A200038E0012069680004814203D121680143C4
:109A3000216011E0052301221B0492049942216850
:109A400002D111432160F1E7814321602168014087
:109A50000091206890432060686800280DD0FFF7CF
:109A600051FB009005E0FFF74DFB0099401A642878
:109A70007ED820688003F6D50CE0FFF743FB00900A
:109A800005E0FFF73FFB0099401A6428F0D82068F2
:109A90008003F6D4287880075DD5E868810604D570
:109AA000226820210A43226088430923042F0DD015
:109AB0000C2F01D1002E09D000283CD021689943F9
:109AC00001432160FFF71EFB064628E02168490795
:109AD00001D500288AD061681F22120291432A69A9
:109AE0001202114361602168994300E091E1014352
:109AF0002160FFF73DFFE16809060A0FB449895C60
:109B0000C840B4490860B4480068FFF75BFB002810
:109B100074D120E0FFF7F6FA801B0228A8D820684D
:109B20004007F7D560681F210902884329690902A7
:109B3000084360600FE02068400840002060FFF7A5
:109B4000E1FA064604E0FFF7DDFA801B02288FD811
:109B500020684007F7D42878C00661D5002F0DD0C3
:109B6000A86900284BD02068FF210131084300E09C
:109B7000C6E02060FFF7C6FA06462DE020688005A3
:109B800002D5A8690028A5D0606807214903884349
:109B9000296A084360606068297F0002000A09069C
:109BA00008436060286A410B0120C003491C8840BB
:109BB000E16809060A0F8649895CC8408549086042
:109BC00085480068FFF7FEFA002817D128E0FFF764
:109BD00099FA801B0228A1D820688005F7D5606813
:109BE000072149038843296A084360606068297F28
:109BF0000002000A09060843606011E0E1E0216804
:109C0000FF20013081432160FFF77CFA064604E023
:109C1000FFF778FA801B022872D820688005F7D4F5
:109C200028786E4E000724D568690028306910D066
:109C3000012108433061FFF765FA009005E0FFF766
:109C400061FA0099401A02285AD830698007F6D57F
:109C50000FE0400840003061FFF754FA009005E043
:109C6000FFF750FA0099401A022849D83069800756
:109C7000F6D42878400765D500200290A06BC0007C
:109C800006D4A06B012109070843A06301200290BC
:109C900053480168C90511D4016882151143016058
:109CA000FFF730FA009005E0FFF72CFA0099401A10
:109CB000642825D84A480068C005F5D5FF20AA6861
:109CC0000130824203D131690143316111E0012148
:109CD0008902002A07D005231B029A4203D1326968
:109CE0000A433261EFE73269824332613069884367
:109CF0003061A86800280FD0FFF704FA009007E051
:109D00005EE0FFF7FFF90099411A3648814257D8C3
:109D100030698005F5D50DE0FFF7F4F9009006E015
:109D2000FFF7F0F90099411A2E48814248D830696E
:109D30008005F5D40298002804D0A06B0121090702
:109D40008843A063686A002865D00C2F4CD0012698
:109D500036060228206805D0B0432060FFF7D2F90C
:109D600005462FE0B0432060FFF7CCF9074604E03A
:109D7000FFF7C8F9C01B022822D820688001F7D459
:109D8000E96AA86AE2680843296BFD231B049A4329
:109D900011430843E060206830432060FFF7B2F9C8
:109DA000054604E0FFF7AEF9401B022808D82068FA
:109DB0008001F7D52FE0FFF7A5F9401B022801D954
:109DC0000320FEBD20688001F5D424E0001002408D
:109DD000BC2D0108A40000209C000020401002407F
:109DE00000700040881300000128EAD0E0680121DB
:109DF0000904AA6A014091420BD10F218904EA6A41
:109E00000140914205D1032189050840296B884210
:109E100001D00120FEBD0020FEBD000070B5040091
:109E200005D0254620356878002802D006E00120BC
:109E300070BD00202870204600F046F802206870AF
:109E40002068C168C943C90637D5CA214162216863
:109E500053204862204604F029F8002827D12068C2
:109E60008168184A11408160216888686268A36926
:109E7000104322691A43104388602168E068086132
:109E8000206801692289120411430161204604F00F
:109E900030F800280BD12168CA6C92089200CA647D
:109EA0006269E16911432268D36C1943D164226865
:109EB000FF215162002801D070BD0020012169708E
:109EC00070BD0000BFFF8FFF00680549884205D1C3
:109ED00004480169012292041143016170470000A6
:109EE000002800404010024070B5044621680A482E
:109EF000C860FFF707F97D260546F60006E0FFF784
:109F000001F9401BB04201D9032070BD2068C06830
:109F10008006F4D5002070BD5FFF0100F8B5040095
:109F20000ED0FF27606A0537002500280AD025617A
:109F3000656126464036A562707C002807D00AE09D
:109F40000120F8BD6068B842F3D0E561F1E73574EF
:109F5000204600F03FF80221717420680268402317
:109F60009A4302602123A26860689B021A4038402D
:109F70001043E3688A021340184323690B40217D94
:109F80001843C907C90F0843A16993101940084332
:109F9000E169382319400843216A802319400843A6
:109FA000A16A93001940084321680860A069042150
:109FB000000C0840616A102319400843216848607A
:109FC0002068C1699143C1616565012070740020FA
:109FD000F8BD000010B586B0044614216846FBF7B2
:109FE0000BF910492068884219D10F48416B82143F
:109FF00011434163C16A01221143C162C06A002159
:10A0000010400590E0200090022001900320039072
:10A0100002910491052069460007FEF789FF06B00A
:10A0200010BD00000030014000100240FFB50546A1
:10A0300004464035287C002781B01646012809D007
:10A0400001202874FFF75EF80090687C012804D096
:10A05000022797E0022005B0F0BD0298002874D0D6
:10A06000002E72D00320687400206065029921637D
:10A07000A686E686A063A087E0876064206401224C
:10A08000A068D2034021904208D1206802688A4328
:10A090000260206802680B021A43026020680268AE
:10A0A000520602D402680A4302600121E068C90234
:10A0B0008842606828D1002801D0012E1ED1206B73
:10A0C00021680088C86006E020688168890709D592
:10A0D000216B0988C160206B801C2063E08E401ECC
:10A0E000E0860BE0FFF70EF80099411A04988142D0
:10A0F00002D3401C02D005E0002803D0E08E0028E7
:10A10000E2D128E003273BE0002801D0012E1FD137
:10A11000206B21680078087306E020688168890751
:10A1200009D5216B09780173206B401C2063E08EF8
:10A13000401EE0860CE0FEF7E5FF0099411A049806
:10A14000814203D3401C03D0DCE717E00028D9D0BC
:10A15000E08E0028E1D12046009A049904F018F915
:10A16000002801D020206065A068002803D1206865
:10A17000C16880680090606D002801D0012701E06F
:10A180000120687400202874384664E7FFB504464F
:10A1900083B00120254640350090287C00271E46CC
:10A1A00001280FD001202874FEF7ACFF0190687CD5
:10A1B000616801280DD0CA1FFD3A08D1A1680029A5
:10A1C00005D102E0022007B0F0BD042801D002272B
:10A1D000D0E0049800287AD005980028FBD0002E03
:10A1E000F9D0687C042801D00520687400206065DF
:10A1F0000599A163E687A68704992163E686A6866A
:10A200002064606420680168490603D40168402224
:10A21000114301600121E068C9028842606847D1AA
:10A22000002801D0012E3CD1206B21680088C86035
:10A23000206B801C2063E08E401EE08631E02068A9
:10A240008168890710D5E18E00290DD00099012978
:10A250000AD1216B0988C160206B801C2063E08ECD
:10A26000401EE0860020009020688168C9070DD05C
:10A27000E18F00290AD0C068A16B0880A06B801C08
:10A28000A063E08F401EE08701200090FEF73AFFB8
:10A290000199411A0C98814203D3401C01D0032735
:10A2A00066E0E08E0028CAD1E08F0028C7D148E0E0
:10A2B000002801D0012E3ED1206B21680078087360
:10A2C000206B401C2063E08E401EE08633E04DE0B2
:10A2D00020688168890710D5E18E00290DD000998A
:10A2E00001290AD1216B09780173206B401C20637E
:10A2F000E08E401EE0860020009020688168C9073B
:10A300000DD0E18F00290AD0C068A16B0870A06B46
:10A31000401CA063E08F401EE08701200090FEF704
:10A32000F1FE0199411A0C98814202D3401C02D0DF
:10A33000B5E70028B3D0E08E0028C9D1E08F00280F
:10A34000C6D12046019A0C9904F022F8002803D0C7
:10A350000127202060650DE0A068002803D1206857
:10A36000C16880680090606D002801D0012701E07D
:10A370000120687400202874384624E7094910B584
:10A38000401E884201D9012010BD074C60610321A5
:10A39000081F07F0A7F90020A06107202061002016
:10A3A00010BD0000FFFFFF0000E000E0F0B5024636
:10A3B0002032137E012B21D00125157602235376FE
:10A3C00006687468B3687027BC430F6827437760DA
:10A3D0000068AC07A04208D0094CA04205D0094C47
:10A3E000A04202D0084CA04204D180244968A34373
:10A3F00019438160557600201076F0BD0220F0BD33
:10A4000000040040000801400014014002462032D0
:10A41000137E012B06D0012313760068016500200E
:10A42000107670470220704710B586B0044614219C
:10A430006846FAF7E1FE0D492068884213D10C48BE
:10A44000C26A04210A43C262C06A084005904020E3
:10A45000009002210020019102900491039069462E
:10A460000448FEF765FD06B010BD00000004004082
:10A470000010024000080050F8B506460446203699
:10A48000307E00270D4601280ED001203076002AAC
:10A490000CD0042A1BD0082A2FD00C2A3ED001272A
:10A4A000002030763846F8BD0220F8BD206805F05F
:10A4B000AFFB2068816908221143816120688269AD
:10A4C00004218A43826120688169EA6812E0206879
:10A4D00005F0B6FB206882690121C9020A43826146
:10A4E000206881690122920291438161206881691B
:10A4F000EA68120211438161D2E7206805F0B9FBD6
:10A500002068C16908221143C1612068C269042121
:10A510008A43C2612068C169EA6812E0206805F0D8
:10A52000C3FB2068C1690122D2021143C1612068C6
:10A53000C269012189028A43C2612068C169EA684F
:10A5400012021143C161ABE770B5050005D02C467E
:10A550002034607E002802D006E0012070BD00207B
:10A560002076284600F010F802206076291D286821
:10A5700005F01AFB0120A077A076E07620776077BF
:10A580006076002070BD000000680449884204D154
:10A590000348816B0222114381637047000400402D
:10A5A000001002407047704770B504001BD0242093
:10A5B000E0672068016849084900016020680025BB
:10A5C00005602068456020688560204600F09EF99F
:10A5D000204680304560E567056025666566603425
:10A5E0002576002070BD012070BD10B506F062FD1B
:10A5F00010BD0000F8B502680446D0691168936880
:10A60000A44D06462E4025468035002E71D0A24F1F
:10A61000DE07F60F0F4037437ED0C70706D0CF05C1
:10A6200004D5012717626A683A436A60820708D531
:10A63000DA0706D0276802223A626A6804273A439A
:10A640006A60420708D5DA0706D0236804221A6236
:10A650006A6802231A436A60020709D520220A4069
:10A66000324305D0236808221A626B6813436B607B
:10A67000020509D54A0107D501222368D2021A62D0
:10A680006A6820231A436A606A68002A39D0800603
:10A6900006D5880604D5A16E002901D0204688473A
:10A6A000686821688968490602D4282108422DD0AB
:10A6B000204605F094FC21688868400622D5EFF317
:10A6C0001080012282F310888A6840239A438A60AE
:10A6D00080F31088606F002814D070498163606F28
:10A6E000FEF7A4F900280CD0606F816B08E000E051
:10A6F00012E0860610D58E060ED5A16EAFE020467C
:10A700008847F8BD2046FFF770FFF8BD2046FFF7E9
:10A710006CFF00206860F8BD266E012E7DD1C60654
:10A720007BD5CE0679D51023136222689068264621
:10A7300040064036002849DA616F08684068000426
:10A74000000CE8D0378B8742E5D970830868006831
:10A75000800634D4EFF31080012181F31088116852
:10A760001F01B943116080F31088EFF310800121BD
:10A7700081F3108821688A68520852008A6080F349
:10A780001088EFF31080012181F3108821688A6816
:10A790004027BA438A6080F3108820202860002078
:10A7A0002066EFF31080012181F3108821680A6888
:10A7B0009A430A6080F31088606FFEF715F9022053
:10A7C0006066308B718B401A81B234E0308B718BB4
:10A7D000401A81B2708B00289DD000299BD0EFF3E6
:10A7E0001080012686F310881668FF272137BE43A4
:10A7F000166080F31088EFF31080012282F3108836
:10A800002268966876087600966080F3108820208B
:10A81000286000202066A06600E010E0EFF31080C2
:10A82000012282F31088226815689D43156080F329
:10A830001088022060662046FFF7B4FEF8BDC5020E
:10A8400008D55B0206D50120000510622046FFF7FF
:10A85000AAFEF8BD030606D50B0604D5E16E002955
:10A8600000D04CE7F8BD4006FCD54806FAD5204696
:10A87000EFF31081012383F3108813684024A3436E
:10A88000136081F310882021C1670021C16600F0A8
:10A89000C7FAF8BD0F080000200100046DFE000893
:10A8A00010B5040003D0E06F002802D007E00120BB
:10A8B00010BD002178200155204600F073F82420B7
:10A8C000E06720680168490849000160204605F0FA
:10A8D0009FFC0128ECD0606A002802D0204605F0D9
:10A8E000FEF9206841680922D20291434160206844
:10A8F00081682A2291438160206801680122114306
:10A900000160204605F050FA10BD000010B5044665
:10A9100000681E4B05221E49120798420BD1486B56
:10A9200001239B0398434863032149021046FEF725
:10A930004FFA1B2012E0174B984212D1886B01236B
:10A940005B04984388630C211046FEF741FA606F60
:10A95000FEF792F8206FFEF78FF81C20FEF7F4FD4B
:10A9600010BD0D4A9042FBD1886B01221205904325
:10A97000886311120948FEF72BFA04210848FEF7F4
:10A9800027FA606FFEF778F80E20E7E700380140FD
:10A9900000100240004400400050004000080050F9
:10A9A000000C0050F0B587B0054614216846FAF750
:10A9B00023FC634B2A6863480227032100240426F2
:10A9C0009A421CD1426B33031A434263C26A012389
:10A9D0001A43C262C06A0391184005904802009071
:10A9E000052001970496029469460007FEF7A0FA35
:10A9F000002211461B20FEF7C3FD1B2051E0524BE5
:10AA00009A4252D1826B01235B041A438263C26A69
:10AA100001231A43C262C06A0426184005900C2024
:10AA2000009003910520019704960294694600075F
:10AA3000FEF77EFA464F4548BC60FC6041C7802661
:10AA4000FC60BE6020203C61786103200003B86197
:10AA50003F48083FFEF798F8002801D0FDF79FF81F
:10AA60006F67BD623B4F394839461438386004205F
:10AA700078601020083151C17C61BC610320000363
:10AA8000FC6138623846FEF77FF8002801D0FDF7F8
:10AA900086F82F67002211461C20BD62FEF770FD6C
:10AAA0001C20FEF761FD07B0F0BD2B4B9A42FAD196
:10AAB000826B01231B051A438263C26A3243C2625E
:10AAC000C26A32400592C36A08221343C362C06A55
:10AAD00001971040059050020090032003900294CB
:10AAE000694604971D48FEF723FA032003900620C9
:10AAF000049001970096029469461948FEF718FAE7
:10AB00001248184E3C383060B4600D20F46070601C
:10AB100074618020B461306120203462F06130467D
:10AB2000FEF732F8002801D0FDF739F86E670022F1
:10AB300011460E20B562FEF723FD0E20B1E700009E
:10AB4000003801400010024000440040580002401C
:10AB500074090020BC09002000500040000800508B
:10AB6000000C0050040A002070B580231B58202BD5
:10AB700001D0022070BD00290BD0002A09D0012489
:10AB800083682403A34206D10369002B03D1CB07BA
:10AB900001D0012070BD002303660B4B04689C426A
:10ABA0000ED063681B020BD5EFF31083012585F3EC
:10ABB000108825680126B6063543256083F3108882
:10ABC00005F030FC70BD00000048004070B58023E7
:10ABD0001B58202B01D0022070BD00290BD0002A69
:10ABE00009D0012483682403A34206D10369002B02
:10ABF00003D1CB0701D0012070BD002303660B4BAE
:10AC000004689C420ED063681B020BD5EFF31083DF
:10AC1000012585F3108825680126B6063543256091
:10AC200083F3108805F054FC70BD0000004800401C
:10AC300010B506F061FA10BD7047FFB50446C06F4D
:10AC400083B017460D46202802D0022007B0F0BD81
:10AC5000002D0BD0002F09D00120A16800038142F4
:10AC600006D12069002803D1E80701D00120EDE7D3
:10AC70000021842001512120E067FEF743FA264697
:10AC800040360190378277820120A168000381421B
:10AC900002D12069002802D02F46002511E00027AC
:10ACA0000FE000228021204605F0D2FC002815D1BB
:10ACB000002F17D02168387888627F1C708A401E68
:10ACC0007082708A019B002806980090E9D10022CA
:10ACD0004021204605F0BCFC00280AD02020E06777
:10ACE0000320B3E728882168C005C00D8862AD1C29
:10ACF000E4E72020E0670020A8E7000070B50446E4
:10AD0000C06F202801D0022070BD00290BD0002A7E
:10AD100009D00123A0681B03984206D120690028AE
:10AD200003D1C80701D0012070BD20464030E16446
:10AD30000282428200202546803568602121E16739
:10AD4000216F002918D0154BCB62236F144919636A
:10AD5000236F14495963216F134688632668E16C99
:10AD600032462832206FFDF757FF002804D010200C
:10AD700068602020E067D6E7216840200862EFF392
:10AD80001080012181F3108821688A6880231A438A
:10AD90008A6080F31088002070BD000089FF0008E1
:10ADA000D5FF000881FE000830B5C36F202B01D00D
:10ADB000022030BD00290BD0002A09D0012384686D
:10ADC0001B039C4206D10569002D03D1CD0701D09C
:10ADD000012030BDC164014640310A824A8200210F
:10ADE0008422C16611502121C1679C4202D10169B0
:10ADF00000290FD00849C166EFF31081012282F3C8
:10AE000010880068026880231A43026081F310886A
:10AE1000002030BD0149EEE7F7050108990501085A
:10AE200010B506F001FA10BD7047F0B585B00446C4
:10AE3000002500200390002602900027002C02D05D
:10AE40006068002801D105B0F0BDA068402800D995
:10AE5000F9E700252EE0204600F0E4F82E46002019
:10AE600003901FE0606A825D02AB2046039900F008
:10AE70007AF90746022F0DD1606A0090E06A0190CE
:10AE80006068029AD20080186A464168204600F045
:10AE9000A7F80AE0002F00D107E000BF761C039856
:10AEA000401C0390E06AB042DCD800BF022F00D102
:10AEB00003E06D1CE06AA842CDD800BF00BFC2E726
:10AEC0000FB438B504460D4607A80090E169A069A3
:10AED000009B069A06F0B4FB20620020009009480F
:10AEE0000078012803D1216AA06900F079FA294687
:10AEF0002046236AA26900F00FF838BC08BC04B0F1
:10AF0000184700007806002010B50446A06B01F039
:10AF100027FA002010BD0000F8B504460D4616467D
:10AF20001F463A46314620466369984700280AD1B1
:10AF30002046FFF7E9FF0094074B2A460021A06B4B
:10AF400001F0A6FA06E00094044B01220021A06B58
:10AF500001F09EFA0020F8BDA1B0000891B00008F1
:10AF600070B504460D468021204601F03DFB28685F
:10AF7000E06368686060A868A060E868E0602869CD
:10AF8000206168696061A869A061E869E0610020EA
:10AF90002062286A6062686AA0620020E062002184
:10AFA00030200155A86A60632046383001F0ECF982
:10AFB000002802D00020C04370BD204600F002F8F7
:10AFC000FAE700000146002901D1401E70470348FE
:10AFD00000680860014801600020F7E7740600205F
:10AFE00070B504460D461646022D06D0032D05D039
:10AFF000042D04D0052D07D102E000BF00BF00BF23
:10B000002046FFF781FF00E000BF00BF324629461F
:10B01000E06B00F0F5F970BD014800787047000062
:10B020007806002010B50446012240216018FAF786
:10B03000DCF810BD10B50024124804681FE020465B
:10B0400021698847002819D10F480078012810D1BC
:10B05000E16A606A01F038FB012803D1606A00F000
:10B060003FF906E0E16A606A00F086F907A000F0A7
:10B0700037F92046FFF7D9FE0020E0622468002C53
:10B08000DDD110BD74060020780600200D0A0000F6
:10B0900010B50446002205212046FFF7A1FF10BD90
:10B0A00010B50446002204212046FFF799FF10BD89
:10B0B00070B504460D46204600F02CF8012801D159
:10B0C000801E70BD2268501CE168FAF711F82160FB
:10B0D000236921685943A368C81829462269FAF7E9
:10B0E00072F80020EDE710B58160C26003610124B1
:10B0F00044600024046010BD10B504462268501C52
:10B10000E168F9F7F5FF6068814201D1012010BDC7
:10B110000020FCE710B504462268901CE168F9F7AE
:10B12000E7FF6068814201D1012010BD0020FCE7EB
:10B1300070B504460D462046FFF7DEFF012801D119
:10B14000801E70BD236960685843A368C1182846F3
:10B150002269FAF738F86268501CE168F9F7C8FF0D
:10B1600061600020EDE7F0B504460D4600260021A1
:10B170001DE020464030405C012817D1CF006068B8
:10B18000C059405D904204D0002027464037785493
:10B190000CE0761CCF006068C0596F1CC05D0028B1
:10B1A00004D1002B00D019600220F0BD491CA0681A
:10B1B0008842DED8002E01D10020F6E70120F4E716
:10B1C00070B504460D46002C01D1401E70BD00BF75
:10B1D0002068A842FCD32068401B20606268501998
:10B1E000E168F9F785FF61600020EFE770B504467C
:10B1F0000D46002C01D1401E70BD20684019206012
:10B2000000BFE16820688842FBD8A2685019E16855
:10B21000F9F76EFFA1600020EEE7FFB581B00446AC
:10B220000D4616460027002E06D00498002803D0AD
:10B23000E1682068884203D30020C04305B0F0BD18
:10B240002168E068401AA84202D20020C043F5E716
:10B25000A0684019E16888420BD9A168E068471AE4
:10B260002168E068401AE919884202D20020C043F0
:10B27000E4E7A268D019E168F9F73AFF316079197B
:10B28000049801600020D9E70146486870470146EC
:10B29000886870470246002A01D1401E704700208E
:10B2A000506090601060D16000BFF7E70146002950
:10B2B00001D1012070470868002801D10120F9E779
:10B2C0000020F7E70146002901D1012070470A68F4
:10B2D000C868904201D10120F8E70020F6E700009D
:10B2E0000FB400B50E48FFB0407882B0002805D0FA
:10B2F0007FB002B008BC002004B01847012183AB26
:10B3000049026846829A06F09BF90649024688423D
:10B3100000D90A466946002005F01AFFE8E7000058
:10B32000B4010020FF0100000FB400B51048FFB0C9
:10B33000407882B0002805D07FB002B008BC002061
:10B3400004B0184700226946104605F001FF0121AC
:10B3500083AB49026846829A06F072F905490246B3
:10B36000884200D90A466946002005F0F1FEE3E76D
:10B37000B4010020FF010000F0B5064616480C4657
:10B38000417891B0002923D10078012820D10127EC
:10B39000102C01D9102500E02546402101A8F9F71D
:10B3A0002BFF402301AA29463046009701F0CCF834
:10B3B0000AA101A8F9F72BFF01A8F9F752FF0246ED
:10B3C00001A9002005F0C4FE641B7619002CDFD112
:10B3D000002011B0F0BD0000B40100200D0A0000F3
:10B3E00010B5064A5278002A01D0002010BD0A4646
:10B3F0000146002005F0ACFE10BD0000B4010020A5
:10B40000F7B582B004460D46002700266088012863
:10B4100020D1206900280AD1606800680195009059
:10B4200019A200212046E368FCF79CFC12E0A90069
:10B430002069405800782D280CD0A9002069405878
:10B44000616809680091019017A200212046E36815
:10B45000FCF788FC6668F36829462046049A9847FA
:10B4600007460CE07068002808D07068C368294659
:10B470002046049A98470746766800E001E0012FCD
:10B48000F0D000BF05B0F0BD46534D3A252D3873BE
:10B490002053544154453A252D32387320455645A2
:10B4A0004E543A25750D0A0046534D3A252D3873F2
:10B4B0002053544154453A252D3238732045564582
:10B4C0004E543A25730D0A00FFB581B004460E466E
:10B4D00017460025002C01D105B0F0BD30212046D3
:10B4E000F9F78AFE0A98A060049820616660E76018
:10B4F0000021A16261620E48008820800B98608064
:10B500000C48006860610B48046009480088401CD2
:10B5100007490880656806E06560002211462046FC
:10B52000FFF76EFFAD68002DF6D100BFD4E7000035
:10B53000CC030020C80300200246002A01D1401E8F
:10B540007047D1620020FBE7FFB583B005460E4689
:10B550001C460C9F0020029020880004B9B20843CA
:10B5600002900298044B009031462846059A00F05C
:10B570008FFF07B0F0BD0000DD7D0008F7B596B085
:10B5800005460E466F680024002015903C462AE0D0
:10B590006C60002201212846FFF732FFA64205D148
:10B5A00000212846189AFFF72BFF1EE0502101A822
:10B5B000F9F722FE15AB01AA21463046FCF7EFFB56
:10B5C00000280FD10AE0159800686860002128461D
:10B5D000189AFFF715FF15984068159015980028E0
:10B5E000F1D102E06468002CD2D100BFB46806E05B
:10B5F0006C6000212846189AFFF702FFA468002C0F
:10B60000F6D119B0F0BD016E05E002467C324B1C4C
:10B61000D35C5354491CC26D8A42F6D8704710B5AA
:10B62000C26D511E05E002467C32545C4B1CD45462
:10B63000491E026E8A42F6DD10BD70B505460C4605
:10B64000A879002802D001282ED100E000BF432CA9
:10B650001BD004DC412C0CD0422C22D10FE0442C16
:10B6600019D07E2C1DD100220821284600F040FB75
:10B6700018E000220321284600F03AFB12E00022E5
:10B680000421284600F034FB0CE000220621284665
:10B6900000F02EFB06E000220521284600F028FBE2
:10B6A00000E000BF00BF2CE0432C1BD004DC412C89
:10B6B0000CD0422C22D10FE0442C19D07E2C1DD16D
:10B6C00000220821284600F081F818E0002203211A
:10B6D000284600F07BF812E000220421284600F002
:10B6E00075F80CE000220621284600F06FF806E00D
:10B6F00000220521284600F069F800E000BF00BFE5
:10B7000000BF00BF70BD70B504460D46432D46D046
:10B7100008DC1B2D0DD0332D25D0412D3DD0422DE1
:10B720004DD13BE0442D3BD05B2D11D07E2D46D139
:10B7300024E02079002802D0042804D100E000BFD2
:10B740000120207102E00020207100BF00BF39E01D
:10B750002079012802D10220207102E0002020710E
:10B7600000BF00BF2EE02079022802D10320207103
:10B7700002E00020207100BF00BF23E020790328F1
:10B7800006D129462046FFF758FF0420207102E029
:10B790000020207100BF00BF14E000BF00BF00BF49
:10B7A0002079022806D129462046FFF746FF0420CB
:10B7B000207102E00020207100BF00BF02E00020E5
:10B7C000207100BF00BF207970BD0000F7B50446AE
:10B7D0000D46092D02D00020A066E0662B0005F082
:10B7E00074FF0AFD0646CBFCFBFAF9F8F7FD607919
:10B7F000002802D0012837D100E000BFE06D6328A7
:10B800002FD20B20C001201881690298884720465A
:10B81000FFF705FF029821467C31226E8854206E86
:10B82000401C2066E06D401CE065266E002709E0A4
:10B8300022467C32905D0B22D201A2189169884782
:10B84000761C7F1CE06DB042F2D805E00B20C001F1
:10B85000201881690820884738467F1E0028F5D1C6
:10B8600000BF0020607100E000BF00BF3EE2E06D5D
:10B87000002806D10B20C00120184169FEA088478E
:10B8800034E26079002802D0012856D11FE000215F
:10B8900020467C30E26D81546422616F5143024640
:10B8A000C832881821467C31F9F7FDFC606F401CD6
:10B8B0006067606F0A2801DB00206067A06F401C92
:10B8C000A067A06F0A2801D30A20A06736E000BF56
:10B8D00000BF6422206F50432246FF324532811858
:10B8E0006422E6482018F9F76EFC266F11E00A2161
:10B8F000701CF9F7FDFB0F4664227A432346FF33A1
:10B900004533D11864227243D0186422F9F75BFCE6
:10B910003E46616F084609300A21F9F7FFFBB14244
:10B92000E5D1642171432246FF32453288186422F2
:10B93000D2496118F9F747FC00E000BF00BF0B20B7
:10B94000C00120184169CEA08847204600F002FDC2
:10B9500020467C3000F054FC002000F0FBFC00206E
:10B960002066E065606F0A3020670B20C001201858
:10B970004169C4A08847B9E16079002802D0012854
:10B9800055D100E000BFA06F002800D150E0A06FAB
:10B990000A2803D1616F206F88420CD1A06F0A285A
:10B9A00042D0616F0A31A26F881A0A21F9F7A0FB11
:10B9B000206F814238D0216F084609300A21F9F7FB
:10B9C00097FB21676422206F50432246FF3206E036
:10B9D0001CE1DBE096E084E076E02BE085E1453297
:10B9E000811820467C30F9F75EFC20467C30F9F760
:10B9F00038FCE065E06D20660B20C001201841692D
:10BA0000A1A088476423226F5A432346FF3345335E
:10BA1000D0180B22D201A218516988470B20C0010F
:10BA20002018416999A088470120607100E000BF9B
:10BA300000BF5BE16079002802D0012841D100E01D
:10BA400000BFA06F002800D13CE0616F08460930BC
:10BA50000A21F9F763FB206F81422FD0216F481C28
:10BA60000A21F9F745FB21676422206F50432246E3
:10BA7000FF324532811820467C30F9F714FC20460D
:10BA80007C30F9F7EEFBE065E06D20660B20C0012D
:10BA9000201841697CA088476423226F5A432346BB
:10BAA000FF334533D0180B22D201A21851698847C1
:10BAB0000B20C0012018416974A0884701206071E3
:10BAC00000E000BF00BF11E1206E002808DD206EFD
:10BAD000401E20660B20C00120188169082088477D
:10BAE00004E1E16D206E88420BD222467C32236E47
:10BAF000D05C0B22D201A21891698847206E401CAD
:10BB00002066F3E06079002802D001283BD100E0F4
:10BB100000BFE06D002833D0206E002830DD0B2000
:10BB2000C0012018816908208847266E012709E096
:10BB300022467C32905D0B22D201A218916988477F
:10BB4000761C7F1CE06DB042F2D80B20C00120189B
:10BB500081692020884705E00B20C00120188169F9
:10BB60000820884738467F1E0028F5D1206E401EE9
:10BB700020662046FFF747FDE06D401EE06500BFF0
:10BB80000020607100E000BF00BFAFE060790028D6
:10BB900002D0012837D100E000BFE06D00282FD08F
:10BBA000206E00282CDD216EE06D884228D0206EAA
:10BBB000461C012709E022467C32905D0B22D2010F
:10BBC000A21891698847761C7F1CE06DB042F2D8BC
:10BBD0000B20C001201881692020884705E00B2038
:10BBE000C001201881690820884738467F1E002838
:10BBF000F5D12046FFF707FDE06D401EE06500BF70
:10BC00000020607100E000BF00BF6FE06079002895
:10BC100002D0012866D100E000BFE06D00285ED0B0
:10BC2000E06E00280AD10120E06621467C312046E2
:10BC3000E030E26DF9F7C7FAE06D606642E0A06EB1
:10BC400000F026FB06462146E031626EF9F734FB30
:10BC5000002834D10B20C001201841690CA088476E
:10BC6000A06E00F015FB06460B20C00120184169AC
:10BC700030468847A06E0FE00D0A3E002C050000FC
:10BC80000D0A00003E0000000D3E00001B5B4A0054
:10BC90000D1B5B4A3E00000000F0FAFA06463146F2
:10BCA00020467C30F9F7FFFA20467C30F9F7D9FAC4
:10BCB000E065E06D2066A06E401CA06607E0A06E07
:10BCC000401CA06600F0DEFAA16E8842B7D800BF23
:10BCD00000F0D8FAA16E884201D80020A0660020AA
:10BCE000607100E000BF00BF00E000BF00BFFEBD0C
:10BCF000F7B504460E46330005F0E7FC09F2064EA0
:10BD0000F2F2B0BDD8F1F200E06D632843D2A07921
:10BD1000012806D10B20C001201881692A208847FC
:10BD200005E00B20C0012018816902988847204651
:10BD3000FFF775FC029821467C31226E8854206EF4
:10BD4000401C2066E06D401CE065256E002713E076
:10BD5000A079012806D10B20C001201881692A2072
:10BD6000884707E022467C32505D0B22D201A218A0
:10BD7000916988476D1C7F1CE06DA842E8D805E0FA
:10BD80000B20C001201881690820884738467F1E93
:10BD90000028F5D10DE10CE1E06D002809D1A07972
:10BDA000002806D10B20C0012018416982A08847D5
:10BDB000FFE0A079002802D001284CD117E0002133
:10BDC00020467C30E26D81540B20C001201841696F
:10BDD0007DA088470120A07100202066E0652246F2
:10BDE0007C32102120460C3000F07BFD34E0002135
:10BDF00020467C30E26D81540020E06522467C3292
:10BE0000402120461C3000F06CFD21461C312046AC
:10BE10000C3000F08BF900280CD10B20C001201849
:10BE200041696DA088470220A07100202066E0656E
:10BE300060710FE00B20C001201841696AA088479B
:10BE40000B20C001201841695BA088470020A07129
:10BE50002066E06500E000BF00BFAAE0206E002879
:10BE600008DD206E401E20660B20C001201881696D
:10BE7000082088479DE0E16D206E884215D2A079A8
:10BE8000012806D10B20C001201881692A2088478B
:10BE900008E022467C32236ED05C0B22D201A2182D
:10BEA00091698847206E401C206682E0E06D002882
:10BEB0003FD0206E00283CDD0B20C0012018816996
:10BEC00008208847256E012715E0A079012808D1B0
:10BED0000B20C001201881692A20884709E029E049
:10BEE00066E022467C32505D0B22D201A218916995
:10BEF00088476D1C7F1CE06DA842E6D80B20C0016E
:10BF0000201881692020884705E00B20C0012018F7
:10BF100081690820884738467F1E0028F5D1206EA9
:10BF2000401E20662046FFF76EFBE06D401EE06578
:10BF300000BF3EE0E06D002839D0206E002836DDDD
:10BF4000216EE06D884232D0206E451C012713E03F
:10BF5000A079012806D10B20C001201881692A2070
:10BF6000884707E022467C32505D0B22D201A2189E
:10BF7000916988476D1C7F1CE06DA842E8D80B20B2
:10BF8000C001201881692020884705E00B20C001EE
:10BF9000201881690820884738467F1E0028F5D17F
:10BFA0002046FFF730FBE06D401EE06500BF00E07B
:10BFB00000BF00BFFEBD00000D0A757365726E61A3
:10BFC0006D653A20000000000D0A70617373776F91
:10BFD00072643A20000000000D0A57656C636F6DB3
:10BFE00065210D0A3E0000000D0A5573657220762A
:10BFF0006572696679206661696C65642E0000006F
:10C0000038B5002000900024414804687CE072E0CC
:10C0100000F0EAF90546684601782046FFF773FB11
:10C02000002800D067E0A068281A3A49884205D95C
:10C03000A5600220A0710020E0652066A07900289C
:10C0400002D001282BD100E000BF684600780D28FF
:10C0500006D16846027802212046FFF749FE1DE01E
:10C06000684600780A2819D068460078082805D163
:10C07000002207212046FFF73BFE0FE068460078CC
:10C08000092805D1002209212046FFF731FE05E0ED
:10C090006846027801212046FFF72AFE29E068461B
:10C0A00000780D2806D16846027802212046FFF765
:10C0B0008DFB1DE0684600780A2819D06846007894
:10C0C000082805D1002207212046FFF77FFB0FE05B
:10C0D00068460078092805D1002209212046FFF78B
:10C0E00075FB05E06846027801212046FFF76EFBEC
:10C0F00000BF00BF00BF0B20C0012018C169684607
:10C100008847002884D02468002C80D138BD0000E6
:10C11000E803002040771B00034909680160022101
:10C120008171014908607047E80300200246002041
:10C130007047000000BFEFF30580002800D0704773
:10C1400007480068002804D1012080F3108800BF50
:10C1500000BF03480068401C0149086000BFEEE7CB
:10C16000D003002070B504460D4600F0A3F8002867
:10C170000FD000F09FF80B21C9014018006900287A
:10C1800007D000F097F80B22D2018018016902A0B5
:10C190008847002070BD00001B5B481B5B4A000005
:10C1A00070B502460C4600210023002A01D0002C65
:10C1B00002D10020C04370BD0021002316E0C8005A
:10C1C0000D4D2858002810D1D8001058CD000A4E27
:10C1D0007051D80080184068CD00AD1968600748DC
:10C1E0000068401C054D28605B1C491C502901D289
:10C1F000A342E4D30020DEE7F4030020F003002094
:10C20000F0B595B00446002600E0641C2078202894
:10C21000FBD02046F9F725F8002801D115B0F0BD74
:10C220002046F9F71EF80019461E02E00020307083
:10C23000761E30782028F9D0142301AA2021204628
:10C2400000F078FB0746002513E0E9000C4A50583F
:10C250002146F9F70DF800280AD1E80008494018EE
:10C2600001A9426838469047002800D105E004E063
:10C270006D1C00F007F8A842E7D800BF0020CDE70A
:10C28000F40300200148006870470000F00300201C
:10C29000014605480068814201D304A07047C800E8
:10C2A000034A1058FAE70000F003002000000000E5
:10C2B000F40300200148006870470000EC030020F0
:10C2C000F8B506460F46002536E0002418E0FFF7D3
:10C2D000F1FF002813D0FFF7EDFF0B21C901401833
:10C2E000006900280BD0FFF7E5FF0B23DB01C01826
:10C2F00002692819C000134B195813A09047641CF9
:10C30000052C04DAFFF7BEFF29198842DFD8FFF7B2
:10C31000D1FF00280FD0FFF7CDFF0B21C901401836
:10C320000069002807D0FFF7C5FF0B22D201801853
:10C33000016907A088476D1DFFF7A4FFA842C4D874
:10C340000020F8BDF4030020252D313673000000D5
:10C350000D0A00000149086070470000EC0300204E
:10C360000146202902D30020C04370470122182033
:10C370004843044B1A50002218204843C0188260DA
:10C380000020F2E7C43D002070B505460024002DD2
:10C3900001D1401E70BD00240CE0182060430C4900
:10C3A0000858002805D1012118206043084A11507F
:10C3B00002E0641C202CF0D300BF202C05D105A086
:10C3C000FEF78EFF0020C043E4E72C600020E1E789
:10C3D000C43D002074696D65722049442069732052
:10C3E00066756C6C0D0A000001480068704700001B
:10C3F000D803002010B5002400BF41E0182060439E
:10C400002149085802283AD1182060434018806812
:10C410001E490968091A182060431B4A8018C06821
:10C4200081422CD9182060431146401840690028E9
:10C4300020D01820604340180079002804D1012141
:10C440001820604311500AE00221182060430E4A70
:10C4500011500E480168182060438018816018222E
:10C460006243094BD218106918226243D2185169ED
:10C47000884704E0012118206043034A1150641CDE
:10C48000202CBBD310BD0000C43D0020D8030020E9
:10C49000F0B50446059D202C02D30020C043F0BD1A
:10C4A0000226182060430E4F3E50182060433E463F
:10C4B000801901710B48066818206043C019866016
:10C4C000182060433E468019C260182060438019DE
:10C4D000436118206043801905610020DFE70000F8
:10C4E000C43D0020D803002007480068401C0649CE
:10C4F00008600648026840680021521C4841034910
:10C500000A60486070470000D8030020E003002064
:10C5100000BFEFF30580002800D07047094800688D
:10C52000002804D007480068401E064908600548F6
:10C530000068002804D100BF80F3108800BF00BF4E
:10C5400000BFEAE7D0030020FFB581B005460C46E6
:10C550000026002300200090002D03D0002A01D0E7
:10C56000002C02D1002005B0F0BD0A98012801D1AD
:10C57000032000E002206043401C0499884201D956
:10C580000020F0E7002618E0A85D0090009908114F
:10C5900000F019F819465B1C505400990807000F69
:10C5A00000F011F819465B1C50540A98012803D179
:10C5B000202118465B1C1154761CA642E4D30020AF
:10C5C000D0541846CFE70146092903DC084630302D
:10C5D000C0B270470A2905DB0F2903DC0846373053
:10C5E000C0B2F6E73020F4E770B504460D462946A0
:10C5F0002046F8F701FE70BD0146302904DB3929D9
:10C6000002DC084630380EE0412904DB462902DC12
:10C610000846373807E0612904DB662902DC084652
:10C62000573800E00020C0B2704710B502460B46F4
:10C63000002406E01078FFF7DFFF21014418521CA8
:10C640005B1E002BF6D1204610BD00B5024600232C
:10C6500005E01078FFF7D0FF19014318521C10783D
:10C660000028F6D1184600BD70B588B005460C46C6
:10C67000002007900690059004902846F8F7F1FDF9
:10C68000064604A805A906AA07AB009201910290EC
:10C690000AA23146284600F031F8042803D00020D1
:10C6A000C04308B070BD0798207006986070059868
:10C6B000A0700498E0700020F3E7000025642E25A8
:10C6C000642E25642E25640002460B46002100BF1F
:10C6D00010E0505C202803DB505C7E2800DC08E082
:10C6E000505C0D2802D0505C0A2800D101E00020E7
:10C6F0007047491C9942ECD30120F9E70FB4F0B51B
:10C7000085B00446002004900022202003900020E1
:10C710000290002C02D00C98002805D1002005B012
:10C72000F0BC08BC04B018470DA80490CFE0002965
:10C7300008D10C980078252803D10C9840786528FA
:10C7400000D0C9E00C98007825286ED10C98401CC8
:10C750000C900C98007803900C98401C0C90039857
:10C76000652877D004DC2A2807D0642873D113E029
:10C77000702872D07828F9D13EE008E020780C9B30
:10C780001B78984202D0641C491E00E001E0002999
:10C79000F4D100BF521C88E00026019600960023C9
:10C7A00000252020049E20CE049618E02078009ECC
:10C7B000002E05D12D2803D10126019600960CE00C
:10C7C000302809DB392807DC012600960A265E435B
:10C7D0000746303FF31900E003E0641C491E0029BE
:10C7E000E4D100BF019E012E01D1DE43731C002D58
:10C7F00000D02B60521C58E000230025049E20CE60
:10C8000004961FE02078302806DB392804DC1E015E
:10C810000746303FF31913E0612807DB662805DC83
:10C820001F010646573EBB190AE043E0412806DBDC
:10C83000462804DC1F010646373EBB1900E003E032
:10C84000641C491E0029DDD100BF002D00D02B60E3
:10C85000521C2AE01BE024E0FFE7049E01CE049670
:10C8600000250023254609E026780C9F3F78BE422C
:10C8700001D05B1C00E003E0641C491E0029F3D1D9
:10C8800000BF002801D005604360521C0DE0049BEE
:10C8900001CB0493002800D00460521C01230293B2
:10C8A00003E001200290002200BF00BF029801288F
:10C8B0000DD111E020780C9B1B78984205D1641CA7
:10C8C0000C98401C0C90491E01E0002204E00C98DA
:10C8D0000078002800D02AE700BF0020049010460E
:10C8E0001DE70FB4F8B506460C46002509A80090D0
:10C8F00021463046009B089A04F0A2FE054600201F
:10C900000090A54200D3651E2846F8BC08BC04B0C0
:10C91000184710B502460B46002407E01078FFF7D1
:10C920006BFE0A2161434418521C5B1E002BF5D19B
:10C93000204610BDFFB504461D4621460023002DAC
:10C9400003D0002C01D0002A02D1002004B0F0BD99
:10C9500018465B1C800011500BE00E78019886424F
:10C9600006D100200870481C1E465B1CB600905182
:10C97000491C0878002801D0AB42EED31846E5E701
:10C9800070B506460025002478213046F8F75FFC94
:10C990000446002C04D158213046F8F758FC0446D0
:10C9A000002C0BD0641C05E02078FFF725FE290140
:10C9B0004518641C20780028F6D103E03046F8F7CB
:10C9C0008AFC0546284670BD10B503460C4600217A
:10C9D00000BF05E0585CA04201D1581810BD491CA9
:10C9E0009142F7D30020F9E770B504460D46002CBC
:10C9F00001D0002D02D10020C04370BD012120468E
:10CA00001030FEF7DDFB20462030A968FEF7D8FB8A
:10CA10000020F2E770B504460D46002C01D0002D31
:10CA200002D10020C04370BD012120461030FEF726
:10CA3000DDFB20462030A968FEF7D8FB0020F2E796
:10CA400010B50446002C00D110BD20461030FEF772
:10CA50002DFC012801D10020F6E720462030FEF70A
:10CA600025FC012801D10020EEE720461030FEF71A
:10CA70000BFC0C21484321684018E5E77CB50446CF
:10CA80000E460025002001900090002C00D17CBDB6
:10CA900020461030FEF716FC002801D00020F6E7F3
:10CAA0006B4601AA314620462030FEF7B6FB00282F
:10CAB00001D00020EBE720461030FEF7E8FB0C2108
:10CAC000484321684518A0680199401828606E60A5
:10CAD0000098A8602846DAE7FFB581B004460E4604
:10CAE0001D4600270C2068430399884202D3781E14
:10CAF00005B0F0BD0C202F46474326606760606894
:10CB00008019A0600398C11BE160294620461030BF
:10CB1000FEF7C0FB20462030E168FEF7BBFB00209B
:10CB2000E6E7FEE7F8B50F460546002412E0104898
:10CB30002E786100081832090EA16D1C009004F0D7
:10CB40006BFD00983207120F0AA1401C04F064FD2F
:10CB5000641CE4B2BC42EAD305480D227900425479
:10CB600008180A2242700248891C04F02BF9F8BD0B
:10CB7000103800202578000070B501240E4D6403A4
:10CB8000002221462846FCF7B6FA0022610028461A
:10CB9000FCF7B1FA0A2005F039FB012221462846AC
:10CBA000FCF7A9FA0A2005F031FB002221462846AD
:10CBB000FCF7A1FA70BD00000004005070B501241C
:10CBC0000E4D6403002221462846FCF794FA012208
:10CBD00091032846FCF78FFA0A2005F017FB012283
:10CBE00021462846FCF787FA0A2005F00FFB0022B1
:10CBF00021462846FCF77FFA70BD00000004005073
:10CC0000F1B500240126164F254676030022314651
:10CC10003846FCF770FA0A2005F0F8FA012231468E
:10CC20003846FCF768FA6006040E0121890338468D
:10CC3000FCF75CFA002801D0641CE4B2052005F082
:10CC4000E5FA6D1CEDB2082DE0D30098002803D062
:10CC5000FFF792FF2046F8BDFFF7B0FFFAE70000AC
:10CC600000040050F8B50126164F05467603002251
:10CC700031463846FCF73FFA0024E80901D001228A
:10CC800000E00022012189033846FCF734FA6806E7
:10CC9000050E0A2005F0BAFA012231463846FCF7A3
:10CCA0002AFA0A2005F0B2FA002231463846FCF78B
:10CCB00022FA0A2005F0AAFA641CE4B2082CDCD39C
:10CCC000F8BD00000004005070B501220C4D940323
:10CCD00021462846FCF70FFA012256033146284622
:10CCE000FCF709FA002221462846FCF704FA0A203C
:10CCF00005F08CFA002231462846FCF7FCF970BD9D
:10CD00000004005070B501240E4D6403002221463A
:10CD10002846FCF7F0F96600002231462846FCF769
:10CD2000EAF90A2005F072FA012221462846FCF7AA
:10CD3000E2F9012231462846FCF7DDF90A2005F028
:10CD400065FA70BD00040050F8B50122144D960339
:10CD5000002431462846FCF7CEF9062005F056FAA5
:10CD60000122570339462846FCF7C5F9062005F08D
:10CD70004DFA07E0641CE4B2FA2C03D9FFF7C2FFB6
:10CD80000120F8BD31462846FCF7B0F90028F1D162
:10CD9000002239462846FCF7AEF90020F8BD000015
:10CDA0000004005010B50A48018C012903D100216C
:10CDB0000184FCF7E9FB0648064A403801889142A5
:10CDC00002D1C088002801D1FCF7DEFB10BD0000B5
:10CDD00050360020AA55000010B5F9F73DFB002899
:10CDE00001D00020C04310BD10B5FAF78BFA10BD7A
:10CDF00010B500220F210248FEF702FB002010BDF3
:10CE00006010002010B5044603CC8EB00191009054
:10CE10001DA2102106A8083C04F0E4FB083403CC52
:10CE20000191009018A210210AA804F0DBFB0C224B
:10CE300006A91748F8F7C7F915492C200B39C8750A
:10CE400013480C220AA90D30F8F7BDF91048104B11
:10CE5000DD38817900200290039004900D480591FF
:10CE600001780D480B3B8088019100900BA2642152
:10CE70001846FFF736FD064902460B39002002F03E
:10CE80006BFD0EB010BD0000252E386C6600000052
:10CE9000E1020020010000201036002025732C2C18
:10CEA0002C2C2C302C30302C30302E302C2C2C2CA8
:10CEB0002C2C2A30302C25582C253032782C2578F3
:10CEC0002C25642C25642C2564250D0A0000000007
:10CED00010B5184800F032F81648401E41788170AD
:10CEE0003721202000F071F80321212000F06DF897
:10CEF0004021222000F069F80821232000F065F885
:10CF0000AA21302000F061F80B48008FC1B2322016
:10CF100000F05BF80121332000F057F85F2120205A
:10CF200000F053F8034800F009F80A2005F06EF904
:10CF300010BD0000910300201036002010B50146FE
:10CF40000F2000F021F8002800D0012010BD10B5FE
:10CF50000446FFF7B9FE3220FFF784FEFFF7F4FE28
:10CF6000E0B2FFF77FFEFFF7EFFEFFF7ADFE3320E5
:10CF7000FFF778FEFFF7E8FE0020FFF741FE0446CA
:10CF8000FFF7C0FE204610BD10B50C46FFF7DFFFCF
:10CF90002070012010BD70B50D460446FFF794FEC9
:10CFA0003220FFF75FFEFFF7CFFEE0B2FFF75AFE39
:10CFB000FFF7CAFE2846FFF755FEFFF7C5FEFFF74D
:10CFC000A1FE0A2005F022F970BD10B5FFF7E3FFBE
:10CFD000012010BD10B50248FCF78BF910BD000010
:10CFE000F0060020FEB504460027EFF31080029003
:10CFF000012080F31088344B2168CA1804D13348CB
:10D00000C76803208004074088680190C8680090C2
:10D0100048698E69002A08D12C4940398A6ACD04B2
:10D020002A438A628A6AAA438A62014631433CD013
:10D0300025492268CA4205D12449CB6803229204BB
:10D040009343CB6025462035002810D021680A691B
:10D0500001231A430A61216848610821204600F033
:10D0600037F8032800D1A873216808204860002EF3
:10D0700010D0206801690122114301612068866196
:10D080001021204600F024F8032800D1A87321685D
:10D09000102048600C482168C14206D10B48C16885
:10D0A0000322920491433943C16020680169490811
:10D0B0004900016121680198886021680098C86072
:10D0C000029880F31088FEBD0084FFBF401002402C
:10D0D00070B506460B480D46002409490068F8F76C
:10D0E00007F87D21C90048433168401E00D1032460
:10D0F0000B682A469A4301D00028F6D1204670BD1D
:10D10000204E0000A40000201CB50021184800910A
:10D11000164A01910260C1631205426081600722D4
:10D120008263012202610246C16020321170FF2336
:10D130005170C233436281621173016381610422C1
:10D1400041634261C161FBF7B1FA002801D072B6B8
:10D15000FEE7084800908013019069460448FBF7F9
:10D1600055FA002801D072B6FEE71CBD002401402C
:10D170008406002002000004F0B587B01421684640
:10D18000F8F73AF86A48C26A04210A43C262C26ADE
:10D190000A400592C16A01252943C162C16A29403A
:10D1A0000591C16A02263143C162C16A31400591CD
:10D1B000C26A08210A43C262C06A0122084005907F
:10D1C0000C215C48FBF797FF812105200022090113
:10D1D0000007FBF790FF002210215648FBF78BFF5A
:10D1E000002255495548FBF786FF01225449534810
:10D1F000FBF781FF11210520012209020007FBF73F
:10D200007AFF05200022E9030007FBF774FF1320D3
:10D21000400211273F0400240090694601970294C0
:10D220004448FBF785FE1C20009002946946019556
:10D2300003944048FBF77CFE0520694600070197F0
:10D2400000950294FBF774FE1020009005200294D4
:10D250006946019503940007FBF76AFE28020090D7
:10D26000052002946946019503940007FBF760FED0
:10D27000EF02052002946946000700970195039488
:10D28000FBF756FE2803009005200294694601959D
:10D2900003940007FBF74CFEE8030090052002947E
:10D2A0006946019503940007FBF742FE254800906C
:10D2B00002946946019503942048FBF739FE6946BC
:10D2C0001E48009602950194FBF732FE03204003AE
:10D2D0000090032003900195029469461748FBF7DC
:10D2E00027FE01946946134800970294FBF720FE3D
:10D2F000680200900194694602941048FBF718FEFA
:10D30000002202210520FCF73BF90520FCF72CF94F
:10D31000002211460720FCF733F90720FCF724F917
:10D320000520012210210007FBF7E5FE07B0F0BD44
:10D33000001002400008005081040000000400506A
:10D3400060E00000E184000010B50E480C49016067
:10D35000FF210531416000218160C16001614161AF
:10D36000C161012201625202416282618162072130
:10D37000C162FCF7D3FD002801D072B6FEE710BDF4
:10D38000003001404407002010B586B00024059409
:10D390001E4804940094019402941B490394016074
:10D3A0001F21846041600461F9214461C160FDF77F
:10D3B000CBF8002801D072B6FEE7049404A9134804
:10D3C0000594FCF7F3FF002801D072B6FEE7602059
:10D3D00000907D20019002940022694603940B483E
:10D3E000FDF74AF8002801D072B6FEE7042107488D
:10D3F000FDF70CF8002801D072B6FEE70348FDF7F0
:10D4000013F806B010BD0000000400409C07002087
:10D4100010B50C480A490160E12149024160002130
:10D420008160C16001618161C1610C220162426160
:10D430004162FDF735FA002801D072B6FEE710BD53
:10D4400000380140DC07002010B50C480A49016093
:10D450004B21C901416000218160C160016181618E
:10D46000C1610C22016242614162FDF719FA002894
:10D4700001D072B6FEE710BD0044004064080020F1
:10D4800010B50C480A490160E121490241600021C0
:10D490008160C16001618161C1610C2201624261F0
:10D4A0004162FDF7FDF9002801D072B6FEE710BD1C
:10D4B00000500040EC080020F8B5FFF773FC354839
:10D4C000FBF75CFE34480078052806D8FF210520CC
:10D4D000002201310007FBF70EFE012149022F480F
:10D4E000FBF704FE002806D000F0F6F9FAF7E2F99F
:10D4F000FFF758FCF8BD2A4FB878002801D0FCF798
:10D5000043F82848284C007800280DD002F07AFA19
:10D5100001210846FCF74EF820884B21090188427A
:10D52000E8D9FCF731F8F8BDFAF754FFFFF760FCD3
:10D53000FEF760FFFDF77EFD03F0B4FB1B4E0025F8
:10D540003078002813D020880028ECD0258003F004
:10D5500095FF174803F016FC30788100401813300F
:10D56000C1B20F480A30FFF7DDFA3570F8BD114837
:10D570002188008E8842F9D825807879002803D048
:10D580000B4803F0FFFBF8BD00210B4800F0DCF86E
:10D59000F8BD0000E006002001000020000400505B
:10D5A00004020020E80100201A0000205903002096
:10D5B000743800205036002005CE0008F8B5FCF77E
:10D5C000B7F9524C002120620F2005F06DF8054696
:10D5D00000214F4805F0E0F8680476D56D1C74D042
:10D5E0008122D20100210F2005F097F9002110209F
:10D5F00005F05AF8C1B221700022464805F08AF8B9
:10D60000444922464B78481C93748978D174017937
:10D61000217540793F4D60756A7A202A69D13E4B69
:10D620002A781B789A4264D1EA7822712A79627149
:10D63000EA79A271AA7AE2702175607529465200D2
:10D640000B313648F7F7BFFDE078420033485119F7
:10D6500032300B31F7F7B7FD0020E0713048007829
:10D66000002803D111202F4900020860A08AFAF790
:10D67000D1F82072607A28283BD22B480026006817
:10D68000E27825E071004B19DF7A69460F701B7B49
:10D690004B700988814219D13046F9F7F9FF1F49CB
:10D6A000700032310A5A207A1C4B4100DC335A5246
:10D6B000627950331A54627A90420BD1521C6272D2
:10D6C0001A46A08AA03A505204E00DE0761CF6B249
:10D6D0009642D7D3E07886420BD1217A627A914282
:10D6E00007D1F9F7D5FF04E0104A00210F2005F01B
:10D6F00014F904F005FF0121054805F04DF800205C
:10D7000005F066F8002005F016F8F8BD500300207B
:10D7100000D023243C39002094000020CC3A002083
:10D720000A0200201C000020900000200090272406
:10D7300000487047B010002000487047901000204B
:10D7400000487047A0100020034AD16110620120F8
:10D7500050700020704700006001002000487047B2
:10D76000E81000200249002248784A707047000003
:10D770006001002010B5074B04461A6A002A01D048
:10D78000D9699047182221460348F7F71CFD00206D
:10D7900010BD000060010020D010002002490023CD
:10D7A0000A5C0B54104670476901002002490023AF
:10D7B0000A5C0B54104670476C01002010B5044AF7
:10D7C000536A002B01D0926A9847002010BD0000D8
:10D7D00060010020034A012111540021D21C115480
:10D7E0000846704769010020034A012111540021B5
:10D7F000D21E1154084670476C01002010B5002855
:10D8000009D0064A01219170024680210448FFF7A1
:10D8100068F8002010BD0020C04310BD600100204A
:10D82000E81000200249002288788A7070470000C2
:10D83000600100200020704710B5192904D28A1E0B
:10D8400001460248F7F7BFFC002010BDB0100020D1
:10D8500010B5022902D20020C04310BD8C1E102C2E
:10D8600007D2014622460448F7F7ADFC02490020E2
:10D870000855002010BD00009010002010B50229AE
:10D8800002D20020C04310BD8C1E102C07D20146CE
:10D8900022460448F7F797FC02490020085500206B
:10D8A00010BD0000A01000200249002208780A7074
:10D8B000704700006001002070B5054C0546A26964
:10D8C000002A01D0616990470020256170BD0000E9
:10D8D00060010020FEE77047F8B5012149024E487B
:10D8E000FBF704FC4D4E4E4D0024002871D02878E3
:10D8F000317801270843002870D10320FAF796F801
:10D900002F706BE0474804804748FBF737FCF9F776
:10D91000D1FFFFF747FA4548464900786428444854
:10D92000086000D32F7144484449007809780246C2
:10D9300008431BD0002A0CD04148046002F096F83E
:10D9400001210846FBF736FE2879002801D0FBF7B5
:10D950001BFE3A480078002840D03948046002F0A5
:10D9600085F801210846FBF725FE37E0FFF740FA6E
:10D97000FEF740FDFDF75EFB03F094F9FAF72AFD90
:10D9800030480078002816D02F490888002825D074
:10D990000C8003F073FD2D4803F0F4F9294800785A
:10D9A000810040181330C1B21D480A30FFF7BAF8A1
:10D9B0002448047012E02648018E234802889142D0
:10D9C0000CD804806879002804D0204803F0DAF9E4
:10D9D00004E00EE000211F48FFF7B6FE01214902D6
:10D9E0000D48FBF783FB002803D0F9F72BFF032832
:10D9F00088D02C716C702878002803D00020FAF7AA
:10DA000015F82C70012149020348FBF76FFB002831
:10DA100000D13470F8BD000000040050B6010020B1
:10DA2000040200200C000020E0060020010000207D
:10DA30000011000028000020E6010020E70100207E
:10DA40001C000020590300201A0000207438002018
:10DA50005036002005CE000810B5012149020548C6
:10DA6000FBF744FB002803D1112003490002886220
:10DA700010BD00000004005000000020FEB505F0BD
:10DA8000A9F8334D0320688132496980EA88322A37
:10DA900001D2642103E07D21C9008A4200D9E980D6
:10DAA000298F0A2901D902212987E98E432901D921
:10DAB0004321E986A98A284A914201D10A21A982F3
:10DAC000A98C264A914201D90021A984204C244ADC
:10DAD0004034218E4B260F46B43F0123F600974277
:10DAE00002D3012932D026862386E18FB4399142B0
:10DAF00000D3E687E121C900E187698F782901D940
:10DB000078216987174AE98FD1711749087017483A
:10DB1000A988016016A003F055FD6888C2B2010A09
:10DB200017A003F04FFDE18DA08D00900191638D52
:10DB3000228DE18C1AA003F045FD218E20A003F078
:10DB400041FDE18F26A003F03DFDFEBD2386CBE71E
:10DB50001036002007030000FFFF00001027000020
:10DB60005D0D0000040200209400002090000020C1
:10DB7000C9E8B1B849443A202578202E0D0A0000A2
:10DB8000B9CCBCFEB0E6B1BE3A20CCFAD0ACB6A857
:10DB9000CEBB205625642E25642E200D0A000000E1
:10DBA000B7FECEF1C6F7B5D8D6B73A2025642E25F4
:10DBB000642E25642E25643A25642E0D0A0000008B
:10DBC000B5B1C7B0D4CBB6AFCAB1475053B9A4D7DB
:10DBD000F7BCE4B8F43A202564202E0D0A000000BA
:10DBE000B5B1C7B0B1BBB2F0CAB1475053B9A4D7B1
:10DBF000F7BCE4B8F43A202564202E0D0A0000009A
:10DC000000B5044980208862FF20F53005F0A6F8B1
:10DC100000BD000000040050112302461B0200B5A5
:10DC200019020D489A4202D100F0C0F800BD8A42A4
:10DC300002D100F057F809E0112A04D0824205D140
:10DC400000F002F900BD00F009F800BD002AFCD187
:10DC500000F07AF800BD00001111110000B500F0CD
:10DC60002FF800F02DF800F02BF800F029F800F064
:10DC700027F800F025F800F023F800F021F800F074
:10DC80001FF800F01DF800F01BF800F019F800F084
:10DC900017F800F015F800F013F800F011F800F094
:10DCA000B7F800F0B5F800F0B3F800F0B1F800F004
:10DCB000AFF800F0ADF800F0ABF800F0A9F800BD47
:10DCC00007488021816100BF00BF00BF00BF00BFC7
:10DCD00000BF816200BF00BF00BF00BF00BF704730
:10DCE0000004005000B500F093F800F091F800F047
:10DCF0008FF800F08DF800F08BF800F089F800F054
:10DD000087F800F085F8FFF7DBFFFFF7D9FFFFF793
:10DD1000D7FFFFF7D5FFFFF7D3FFFFF7D1FFFFF7DF
:10DD2000CFFFFFF7CDFFFFF7CBFFFFF7C9FFFFF7EF
:10DD3000C7FFFFF7C5FFFFF7C3FFFFF7C1FFFFF7FF
:10DD4000BFFFFFF7BDFF00BD00B5FFF7B9FFFFF74D
:10DD5000B7FFFFF7B5FFFFF7B3FFFFF7B1FFFFF71F
:10DD6000AFFFFFF7ADFFFFF7ABFFFFF7A9FFFFF72F
:10DD7000A7FFFFF7A5FFFFF7A3FFFFF7A1FFFFF73F
:10DD80009FFFFFF79DFFFFF79BFFFFF799FFFFF74F
:10DD900097FFFFF795FFFFF793FFFFF791FFFFF75F
:10DDA0008FFFFFF78DFFFFF78BFF00BD00B5FFF77B
:10DDB00087FFFFF785FFFFF783FFFFF781FFFFF77F
:10DDC0007FFFFFF77DFFFFF77BFFFFF779FF00F095
:10DDD0001FF800F01DF800F01BF800F019F800F033
:10DDE00017F800F015F800F013F800F011F8FFF73D
:10DDF00067FFFFF765FFFFF763FFFFF761FFFFF7BF
:10DE00005FFFFFF75DFFFFF75BFFFFF759FF00BD07
:10DE10000C488021816100BF00BF00BF00BF00BF70
:10DE200000BF00BF00BF00BF00BF00BF00BF00BFFA
:10DE300000BF00BF816200BF00BF00BF00BF00BFC6
:10DE4000704700000004005000B5FFF7E1FFFFF746
:10DE5000DFFFFFF7DDFFFFF7DBFFFFF7D9FFFFF77E
:10DE6000D7FFFFF7D5FFFFF7D3FFFFF7D1FFFFF78E
:10DE7000CFFFFFF7CDFFFFF7CBFFFFF7C9FFFFF79E
:10DE8000C7FFFFF7C5FFFFF7C3FFFFF7C1FFFFF7AE
:10DE9000BFFFFFF7BDFFFFF7BBFFFFF7B9FFFFF7BE
:10DEA000B7FFFFF7B5FFFFF7B3FF00BDF8B50446B6
:10DEB00000680025C168490619D4C1688022114351
:10DEC000C160FBF71FF927460646203709E0FBF73C
:10DED00019F9811B7D20C000814202D9042078708D
:10DEE00001252068C068400601D4002DEFD02846E7
:10DEF000F8BD70B5044600680025C16880229143D2
:10DF0000C16020688068800608D42046FBF7ECFFDB
:10DF1000002803D00420203460700125284670BDFD
:10DF200070B586B014216846F7F766F9642004F0EE
:10DF300066F90125104EED03002229463046FBF715
:10DF4000DAF80120002401900294694600950394B8
:10DF50003046FAF7EDFF642004F051F903200190F8
:10DF600002946946009503943046FAF7E1FF0220D7
:10DF700004F045F906B070BD0004005070B50546C8
:10DF800000F0F7F90024E443002819D1284600F0F6
:10DF900027F80022C721284600F07AF900282846F1
:10DFA00002D000F00FF80BE000F00CF8284600F06B
:10DFB000D1F9002804D1284600F078F9002800D0D3
:10DFC000204670BD28214843044910B540180189F6
:10DFD00040680122FBF78FF810BD00007825002073
:10DFE00028214843044910B540180189406800229F
:10DFF000FBF781F810BD000078250020FFB581B047
:10E000000C46019828214843174900254018406ACA
:10E010001F461646A0420DD9002E0BD0A1198142F1
:10E0200008D8B900114A00915158491E214201D126
:10E03000032F03D30020C04305B0F0BD002C0ED148
:10E04000B0420CD80198FFF799FF0AE061193A46EF
:10E05000019800F0D5F80549009808584519B542CF
:10E06000F4D30020E8E700007825002028320108DA
:10E0700038B504460322694600F09EF80025ED43BA
:10E08000002812D168460078FF2810D168464078F1
:10E09000FF280CD168468078FF2808D10322694602
:10E0A000204600F089F8002801D0284638BD68468F
:10E0B0008278282044430A48012189052018152A1E
:10E0C00005D0162A03D0172A04D0182A05D0416299
:10E0D000002038BD0121C905F9E701210906F6E74D
:10E0E00078250020FFB50E46C8B2FF2181B001316E
:10E0F00000250C1A0A9F9C4200D91C46019800F08A
:10E10000D5F8002842D1019800F033F900283DD11C
:10E110000198FFF765FF00220221019800F0B8F88E
:10E1200000281FD13002010E0022019800F0B0F843
:10E13000002817D13004010E0022019800F0A8F841
:10E1400000280FD1F1B20022019800F0A1F80028B8
:10E1500008D10CE003980022415D019800F098F886
:10E16000002803D00198FFF72DFF0FE06D1CA5429A
:10E17000F0D30198FFF726FF019800F0EBF8002894
:10E1800004D1019800F092F8002803D00020C04389
:10E1900005B0F0BD002F00D03C600020F8E7000083
:10E1A00010B528246043034CC90000194018426090
:10E1B000038110BD78250020F8B515460E460746A8
:10E1C0000024FFF70DFF00229F21384600F060F881
:10E1D000002807D10DE03219FF21384600F058F829
:10E1E000002805D03846FFF7EDFE0020C043F8BDFB
:10E1F000641CAC42EFD33846FFF7E4FE0020F8BDC4
:10E20000F8B5064615469000204A1058401E814336
:10E210000C46304600F0ADF80027FF43002833D10C
:10E220003046FFF7DDFE19480022001F415D3046F1
:10E2300000F02EF8002816D12002010E00223046F0
:10E2400000F026F800280ED12004010E00223046EE
:10E2500000F01EF8002806D1E1B20022304600F09E
:10E2600017F8002803D03046FFF7ACFE0CE030462C
:10E27000FFF7A8FE304600F06DF8002804D13046C4
:10E2800000F014F8002800D03846F8BD2832010804
:10E2900007B5114628225043034A0123105C01AA06
:10E2A00000F0A6F80EBD000078250020F8B5054660
:10E2B0000020694608706E462846FFF791FE00224E
:10E2C00005212846FFF7E4FF040005D13246FF216F
:10E2D0002846FFF7DDFF04462846FFF773FE2000BF
:10E2E00003D169460978C907E5D1F8BDFFB583B008
:10E2F000002001900D460398282148431449002727
:10E300004018406AFF431C461646A84214D9002E06
:10E3100012D0002C10D0411E2940401AA04201D238
:10E32000044610E001A8009023463246294603988F
:10E33000FFF7D8FE002802D0384607B0F0BD01989C
:10E340002D183618241A002CECD10020F5E7000017
:10E350007825002070B50546FFF742FE0022042113
:10E360002846FFF795FF04462846FFF72BFE204678
:10E3700070BD70B50546FFF733FE00220621284622
:10E38000FFF786FF04462846FFF71CFE204670BDB7
:10E39000F8B5044615480E46154613490068F6F7C9
:10E3A000A7FE7D21C900484300906068C11FFD3968
:10E3B0000ED13346002280212046009500F038F827
:10E3C00000280FD0606D2021084360650320F8BD50
:10E3D0000098002806D0401E009020688068C04346
:10E3E0000006F5D50020F8BD00366E01A40000201F
:10E3F00038B5144600291A460CD064256A430092A9
:10E40000064A800010580A469BB22146FBF7BEFE22
:10E41000002038BD214600F067F838BDC401002057
:10E42000024A80001150002070470000C401002003
:10E43000FFB581B01E4604460A9DFAF763FE401BF5
:10E44000351AFAF75FFE0746264800684001000DBE
:10E45000684339E0701C38D0FAF754FEC01BA8425C
:10E4600005D2002D03D0009800282BD02BE0206887
:10E470004168E022914341606068C11FFD390CD1C1
:10E480000121A068C903884202D04911884204D101
:10E49000206801684022914301600120A16A400385
:10E4A000814207D121680A6882430A6021680A68AC
:10E4B00002430A600120403460740020207403206D
:10E4C00005B0F0BD0025401E0090206881680298CC
:10E4D000884305D0002103988142BBD10020EFE79B
:10E4E0000121F8E7A400002010B56423534394B23F
:10E4F000034A800010582246FBF798FD002010BD0B
:10E50000C401002070470000F8B5044600206A46A8
:10E5100010801A4D55222A70AA226A700322AA700E
:10E52000661DEE702A716971154A49008918AC712F
:10E530002246E81DF6F747FE002007E029186A4644
:10E540008978128889186A461180401CB042F5DB30
:10E55000611DA81CF9F750F9014668460180291988
:10E560000078C8716846407808727D232246DB0037
:10E57000093202490348FCF760FBF8BD243D002046
:10E5800010360020DC070020F8B516460F4604467A
:10E590001D46012240210A48FAF7ADFDFFF730FB86
:10E5A0002846FFF739FB3046FFF736FB3846FFF7C2
:10E5B00033FB2046FFF730FBFFF722FBF8BD0000DE
:10E5C0000004005010B5002240210248FAF793FDE4
:10E5D00010BD00000004005010B5022813D0FDF754
:10E5E00069FE00280DD0FDF765FE0B24E40100193B
:10E5F0000069002805D0FDF75DFE0019016904A03F
:10E600008847002010BD4868FFF7F8F8F9E70000D8
:10E610004552524F520D0A000020704710B502209B
:10E62000FFF7D8F8FDF746FE00280DD0FDF742FEB3
:10E630000B24E40100190069002805D0FDF73AFE1B
:10E640000019016901A08847002010BD4F4B0D0A39
:10E650000000000070B50B24E4010D4602280FD025
:10E66000FDF728FE00280BD0FDF724FE00190069F5
:10E67000002805D0FDF71EFE001901692AA0884771
:10E680006868F6F728FE002815D0012826D0022851
:10E6900036D0FDF70FFE00280BD0FDF70BFE00195A
:10E6A0000069002805D0FDF705FE001901691FA0CB
:10E6B0008847002070BD0020F9F7B8F9FDF7FAFD92
:10E6C0000028F6D0FDF7F6FD001900690028F0D00B
:10E6D000FDF7F0FD0019016916A0E9E7FDF7EAFD75
:10E6E00000280BD0FDF7E6FD00190069002805D0D1
:10E6F000FDF7E0FD001901690EA08847012010E038
:10E70000FDF7D8FD00280BD0FDF7D4FD00190069F6
:10E71000002805D0FDF7CEFD0019016905A0884746
:10E720000220F9F783F9C4E7417267204552524F3E
:10E73000520D0A004F4B0D0A0000000070B54868EA
:10E74000F6F7C9FD7D210446C900F6F7D1FC0503A3
:10E7500064212046F6F7CCFC0A21F6F7C9FC080232
:10E760002D180A212046F6F7C3FC0C460A21F6F7BD
:10E77000BFFC0801281800190D4980B288800D4996
:10E78000086004F0CBFAFDF795FD00280DD0FDF7E9
:10E7900091FD0B24E40100190069002805D0FDF764
:10E7A00089FD0019016904A08847002070BD0000A0
:10E7B00010360020900000204F4B0D0A0000000092
:10E7C00010B5022814DAFDF775FD00280DD0FDF70D
:10E7D00071FD0B24E40100190069002805D0FDF744
:10E7E00069FD0019016903A088470020C04310BDDE
:10E7F000002010BD64656275675F6F666620666C99
:10E8000061670D0A0000000010B5022814DAFDF758
:10E8100051FD00280DD0FDF74DFD0B24E40100193A
:10E820000069002805D0FDF745FD0019016903A026
:10E8300088470020C04310BD002010BD646562758C
:10E84000675F6F6E20666C61670D0A0070B50B25FF
:10E85000ED010C4602280FD0FDF72CFD00280BD04F
:10E86000FDF728FD40190069002805D0FDF722FDBD
:10E870004019016911A088476068F6F72CFD04462D
:10E8800000021149000C48828C8204F047FA2146AC
:10E89000022002F0A3FBFDF70DFD00280BD0FDF7D1
:10E8A00009FD40190069002805D0FDF703FD401956
:10E8B000016906A08847002070BD000041726720F2
:10E8C0004552524F520D0A00503600204F4B0D0A50
:10E8D0000000000070B5FDF7EDFC0B24E4010028FA
:10E8E0000CD0FDF7E7FC00190069002806D0FDF701
:10E8F000E1FC0019026920A122A09047FDF7DAFC93
:10E9000000280FD0FDF7D6FC00190069002809D0B7
:10E91000FEF712FF0546FDF7CDFC001902692946F6
:10E920001EA09047FDF7C6FC00280FD0FDF7C2FCE3
:10E9300000190069002809D0FEF7FAFE0546FDF728
:10E94000B9FC0019026929461AA09047FDF7B2FCEC
:10E9500000280FD0FDF7AEFC00190069002809D08F
:10E96000FEF7EEFE0546FDF7A5FC001902692946F3
:10E9700016A09047002070BD56323032313035310C
:10E980003030300056657273696F6E3A2020202057
:10E99000202020202025730D0A000000494D454904
:10E9A0003A20202020202020202020202025730D08
:10E9B0000A000000434349443A2020202020202020
:10E9C000202020202025730D0A000000494D5349C6
:10E9D0003A20202020202020202020202025730DD8
:10E9E0000A00000010B527210248FDF7D9FB0020DE
:10E9F00010BD00003432010810B50B24E4010228D8
:10EA000012D0FDF757FC00280BD0FDF753FC00197E
:10EA10000069002805D0FDF74DFC001901690BA025
:10EA200088470020C04310BDFDF744FC00280BD0F0
:10EA3000FDF740FC00190069002805D0FDF73AFCFD
:10EA40000019016906A08847002010BD7573616731
:10EA5000653A206C6F6720737472696E670D0A00E7
:10EA60004F4B0D0A0000000010B5FDF723FC0028F5
:10EA70000DD0FDF71FFC0B24E401001900690028EC
:10EA800005D0FDF717FC0019016902A08847002096
:10EA900010BD00004F4B0D0A0000000010B5032808
:10EAA00014D0FDF707FC00280DD0FDF703FC0B2464
:10EAB000E40100190069002805D0FDF7FBFB0019EF
:10EAC000016903A088470020C04310BD002010BD8D
:10EAD00075736167653A206C6F675F7072696E74F9
:10EAE000206173635B302D315D20636E740D0A000D
:10EAF000002070477047000010B50220FEF774FE3A
:10EB0000FDF7D8FB00280DD0FDF7D4FB0B24E40162
:10EB100000190069002805D0FDF7CCFB0019016938
:10EB200001A08847002010BD4F4B0D0A00000000D7
:10EB300010B50020FEF74EFEFDF7BCFB00280DD0FF
:10EB4000FDF7B8FB0B24E40100190069002805D08B
:10EB5000FDF7B0FB0019016901A08847002010BD36
:10EB60004F4B0D0A0000000010B50020FEF73CFEE0
:10EB7000FDF7A0FB00280DD0FDF79CFB0B24E40162
:10EB800000190069002805D0FDF794FB0019016900
:10EB900001A08847002010BD4F4B0D0A0000000067
:10EBA00010B50B24E401022812D0FDF783FB0028E6
:10EBB0000BD0FDF77FFB00190069002805D0FDF799
:10EBC00079FB001901690BA088470020C04310BDE4
:10EBD000FDF770FB00280BD0FDF76CFB00190069F6
:10EBE000002805D0FDF766FB0019016908A08847D9
:10EBF000002010BD75736167653A207274635F739E
:10EC000065745F616C61726D207365630D0A00004D
:10EC10004F4B0D0A000000000020704710B5072878
:10EC200014D0FDF747FB00280DD0FDF743FB0B2464
:10EC3000E40100190069002805D0FDF73BFB00192D
:10EC4000016903A088470020C04310BD002010BD0B
:10EC500075736167653A207274635F7365742079B8
:10EC6000797979206D6D206464206868206D6D204D
:10EC700073730D0A0000000010B5FAF785FC002040
:10EC800010BD000070B50B24E4010E4603280FD020
:10EC9000FDF710FB00280BD0FDF70CFB00190069F5
:10ECA000002805D0FDF706FB0019016920A0884760
:10ECB0007068F6F710FB0546B068F6F70CFB0146E6
:10ECC000681E132821D832291FDC002D1DDD1B4EA4
:10ECD0007D203586C000F6F721FA31464039C880DC
:10ECE00004F01CF8FDF7E6FA00280BD0FDF7E2FA75
:10ECF00000190069002805D0FDF7DCFA0019016948
:10ED00000FA08847012030840FE0FDF7D3FA0028D8
:10ED10000BD0FDF7CFFA00190069002805D0FDF7E8
:10ED2000C9FA0019016902A08847002070BD0000DF
:10ED3000417267204552524F520D0A005036002052
:10ED40004F4B0D0A0000000070B50B24E4010D4686
:10ED500002280FD0FDF7AEFA00280BD0FDF7AAFA73
:10ED600000190069002805D0FDF7A4FA001901690F
:10ED70000DA088476868F6F7AEFA0E49488303F09D
:10ED8000CDFFFDF797FA00280BD0FDF793FA001995
:10ED90000069002805D0FDF78DFA0019016906A069
:10EDA0008847002070BD0000417267204552524FD5
:10EDB000520D0A00503600204F4B0D0A0000000093
:10EDC00010B50B24E401062812DAFDF773FA0028C7
:10EDD0000BD0FDF76FFA00190069002805D0FDF788
:10EDE00069FA001901690EA088470020C04310BDD0
:10EDF00003F094FFFDF75EFA00280BD0FDF75AFAF6
:10EE000000190069002805D0FDF754FA00190169BE
:10EE100005A08847064801210184002010BD00009C
:10EE20004552524F520D0A004F4B0D0A0000000090
:10EE30005036002010B50B24E401052812DAFDF746
:10EE400039FA00280BD0FDF735FA001900690028BF
:10EE500005D0FDF72FFA001901690EA088470020A0
:10EE6000C04310BD03F05AFFFDF724FA00280BD071
:10EE7000FDF720FA00190069002805D0FDF71AFAFD
:10EE80000019016905A08847064801210184002076
:10EE900010BD00004552524F520D0A004F4B0D0A53
:10EEA0000000000050360020F8B50B26F6010D4694
:10EEB000022812DAFDF7FEF900280BD0FDF7FAF967
:10EEC00080190069002805D0FDF7F4F9801901695F
:10EED00014A088470020C043F8BD69466868FDF764
:10EEE000C3FB6868FDF74CFD104CE18A884203D0F3
:10EEF0006868FDF745FDE08203F010FFFDF7DAF9E1
:10EF000000280BD0FDF7D6F980190069002805D03C
:10EF1000FDF7D0F98019016905A0884701202084F8
:10EF20000020F8BD4552524F520D0A0050360020C5
:10EF30004F4B0D0A00000000F8B50B26F6010D46F8
:10EF4000032812DAFDF7B6F900280BD0FDF7B2F965
:10EF500080190069002805D0FDF7ACF98019016916
:10EF600023A088470020C043F8BD69466868FDF7C4
:10EF70007BFB214C68460078618E88420ED1694641
:10EF80004978A28E914209D169468978E28E9142F0
:10EF900004D16946C978228F914209D060866846BB
:10EFA0004078A08668468078E0866846C0782087EA
:10EFB000A868FDF7E5FC618F884203D0A868FDF7DB
:10EFC000DFFC608703F0AAFEFDF774F900280BD080
:10EFD000FDF770F980190069002805D0FDF76AF97E
:10EFE0008019016905A08847012020840020F8BD10
:10EFF0004552524F520D0A00503600204F4B0D0A19
:10F0000000000000F8B50B26F6010D46032812DAC1
:10F01000FDF750F900280BD0FDF74CF98019006975
:10F02000002805D0FDF746F98019016923A088471B
:10F030000020C043F8BD69466868FDF715FB214C08
:10F0400068460078E18C88420ED169464978228D65
:10F05000914209D169468978628D914204D169460D
:10F06000C978A28D914209D0E08468464078208515
:10F070006846807860856846C078A085A868FDF7F6
:10F080007FFCE18D884203D0A868FDF779FCE0851C
:10F0900003F044FEFDF70EF900280BD0FDF70AF946
:10F0A00080190069002805D0FDF704F9801901696D
:10F0B00005A08847012020840020F8BD4552524F0A
:10F0C000520D0A00503600204F4B0D0A0000000080
:10F0D000F8B50B26F6010D46022812DAFDF7EAF81C
:10F0E00000280BD0FDF7E6F880190069002805D04C
:10F0F000FDF7E0F88019016914A088470020C0439B
:10F10000F8BD69466868FDF7AFFA6868FDF738FC36
:10F11000104C218B884203D06868FDF731FC2083B6
:10F1200003F0FCFDFDF7C6F800280BD0FDF7C2F890
:10F1300080190069002805D0FDF7BCF88019016925
:10F1400005A08847012020840020F8BD4552524F79
:10F15000520D0A00503600204F4B0D0A00000000EF
:10F1600070B54868F6F7B7F80C4CE08703F0D6FDA9
:10F17000FDF7A0F800280DD0FDF79CF80B25ED0158
:10F1800040190069002805D0FDF794F8401901697D
:10F1900003A0884701202084002070BD5036002045
:10F1A0004F4B0D0A0000000070B54868F6F793F861
:10F1B0000C4C208603F0B2FDFDF77CF800280DD042
:10F1C000FDF778F80B25ED0140190069002805D0FE
:10F1D000FDF770F84019016903A0884701202084D9
:10F1E000002070BD503600204F4B0D0A000000007B
:10F1F0000020704710B502A0FCF772F810BD0000A7
:10F200004576656E743A25750D0A000070B50B24BD
:10F21000E4010D4602280FD0FDF74CF800280BD072
:10F22000FDF748F800190069002805D0FDF742F8FD
:10F230000019016915A088476868F6F74CF800F0D6
:10F2400075F9002811D0FDF735F800280BD0FDF72F
:10F2500031F800190069002805D0FDF72BF80019D6
:10F2600001690BA08847002070BDFDF723F8002836
:10F27000F9D0FDF71FF8001900690028F3D0FDF759
:10F2800019F80019016904A0ECE700004172672039
:10F290004552524F520D0A004F4B0D0A000000001C
:10F2A000F8B50B24E4010D4604280FD0FDF702F851
:10F2B00000280BD0FCF7FEFF00190069002805D0DC
:10F2C000FCF7F8FF0019016919A088476868F6F78C
:10F2D00002F80746AE68E868F5F7FDFF82B23146EE
:10F2E000384600F05DF9002811D0FCF7E3FF002854
:10F2F0000BD0FCF7DFFF00190069002805D0FCF7F0
:10F30000D9FF001901690BA088470020F8BDFCF760
:10F31000D1FF0028F9D0FCF7CDFF001900690028C3
:10F32000F3D0FCF7C7FF0019016904A0ECE7000067
:10F33000417267204552524F520D0A004F4B0D0A41
:10F340000000000038B50020034600901D4A01214E
:10F35000684600F045F90B24E401002811D0FCF7C1
:10F36000A9FF00280BD0FCF7A5FF001900690028B1
:10F3700005D0FCF79FFF0019016913A08847002002
:10F3800038BDFCF797FF00280CD0FCF793FF00195D
:10F390000069002806D0FCF78DFF001902690CA057
:10F3A00000999047FCF786FF0028E8D0FCF782FF21
:10F3B000001900690028E2D0FCF77CFF0019016900
:10F3C00006A0DBE7F5F100084552524F520D0A0046
:10F3D000536F636B49443A25750D0A004F4B0D0A74
:10F3E0000000000070B50B24E4010D4603280FD087
:10F3F000FCF760FF00280BD0FCF75CFF00190069E8
:10F40000002805D0FCF756FF0019016919A08847AC
:10F410006868F5F760FFAD6806462846F5F721FFF6
:10F4200002462946304600F097FA002811D0FCF732
:10F4300041FF00280BD0FCF73DFF001900690028B0
:10F4400005D0FCF737FF001901690BA088470020A1
:10F4500070BDFCF72FFF0028F9D0FCF72BFF001937
:10F4600000690028F3D0FCF725FF0019016904A00A
:10F47000ECE70000417267204552524F520D0A00DE
:10F480004F4B0D0A0000000000207047002070471D
:10F4900038B5144869460880FCF70CFF00280DD0E9
:10F4A000FCF708FF0B24E40100190069002805D0CF
:10F4B000FCF700FF001901690BA088471124002305
:10F4C0002403022221461846FEF798FD02236A46CD
:10F4D00021460020FEF70AFF064801210184002092
:10F4E00038BD0000AAAA0000757064617465204FE1
:10F4F0004B0D0A00503600200948418F0948828987
:10F50000914208D208490978002904D0012181706C
:10F51000C18A491C01E000218170C182704700004E
:10F5200010360020000000200B02002009490A4A82
:10F530004143891803280AD2002908D008780028F6
:10F5400003D0012801D0052008700020704700205A
:10F55000C0437047C404000068110020F8B50024BF
:10F560000D4D264601270D486043401901780329B7
:10F5700003D0042901D0062908D18670077083685A
:10F58000002B03D0C268022120469847641C032C3C
:10F59000E9DB0020F8BD000068110020C404000071
:10F5A00070B515460B4A0C4B4243D41803280DD2B4
:10F5B000002C0BD00B46204608A22A211030FDF764
:10F5C00090F9658703202070002070BD0020C043A3
:10F5D00070BD0000C4040000681100202573000005
:10F5E000FFB51F4881B01F460E4600251D496943DF
:10F5F0000C1802D02178002906D06D1C032DF5DBF4
:10F600000020C04305B0F0BD16492046FCF7ECFFD2
:10F6100065606670022020700398E7601023A06088
:10F620005F01214620463A46C4313C30FDF754FA8A
:10F63000B1208000012E0AD02118204610233A461E
:10F640006C30FDF749FA019805600020DAE72118CF
:10F65000204601233A46B030FBF745FDF3E70000B2
:10F6600068110020C40400000649074A4143891874
:10F67000032804D2002902D000200870704700201F
:10F68000C0437047C404000068110020032805DA55
:10F6900003494843034940181030704702A070479F
:10F6A000C40400006811002000000000032805DAEF
:10F6B0000349484303494018408F70470020704772
:10F6C000C404000068110020032805DA03494843F8
:10F6D000034940183C30704700207047C4040000C4
:10F6E00068110020032804DA034948430349085CF1
:10F6F0007047002070470000C4040000681100201B
:10F70000032805DA03494843034940184078704705
:10F7100000207047C4040000681100200C490D4A05
:10F7200041438918002210B5D24303280ED2002984
:10F730000CD00B78042B09D001220A708B68002BA7
:10F7400002D0CA6802219847002010BD104610BDA3
:10F75000C4040000681100200A490B4A414310B557
:10F76000891803280BD2002909D007220A708B6858
:10F77000002B02D0CA6800219847002010BD00204D
:10F78000C04310BDC40400006811002070B50546D8
:10F790001A481B4968434418032D25D2002C23D056
:10F7A0000620207010235E01214620463246C431D7
:10F7B0003C30FDF791F91149114BB1206943627852
:10F7C0008000C9180918012A11D02046102332469A
:10F7D0006C30FDF781F9A368002B03D00121284686
:10F7E000E2689847002070BD0020C04370BD2046ED
:10F7F00001233246B030FBF776FCECE7C40400008E
:10F800006811002009490A4A414310B589180328A4
:10F8100009D2002907D08B68002B02D0CA680321C7
:10F820009847002010BD0020C04310BDC404000054
:10F8300068110020FFB5014617461F481F4A0024E3
:10F840004843E443801881B01E4603291AD2002899
:10F8500018D0002E16D04178012916D06C300090B7
:10F86000FDF7EEF805000DD06A68BA4206D22968A5
:10F870000298F5F7A8FC68680024306029460098D3
:10F88000FDF7B2F8204605B0F0BD0024B0302546A3
:10F8900000900BE0029801190098FBF749FC002842
:10F8A00002D000203560EEE7641C6D1CBC42F1D331
:10F8B00000243560E6E70000C40400006811002061
:10F8C000F7B505461A481B49684300244018671ECF
:10F8D0001646032D1FD200281DD04178012910D0D3
:10F8E0006C3007461146FDF7C9F8040019D03246BE
:10F8F00020680199F5F767FC38462146FDF78AF83C
:10F9000013E00546B03509E0019801192846FBF7D8
:10F91000CFFB002801D03846FEBD641CB442F3D3AF
:10F9200003E0294604A0FBF7DBFC0020FEBD00003D
:10F93000C404000068110020536F636B65745B257D
:10F94000755D205265637620427566666572204655
:10F95000756C6C0D0A000000F7B505461348144994
:10F96000684300274018FF4382B01646032D16D285
:10F97000002814D0002E12D03C3011460090FDF724
:10F980007DF804000DD0324620680399F5F71BFC82
:10F9900021460098FDF73EF8002005B0F0BD38463E
:10F9A000FBE7294603A0FBF79BFCF8E7C404000033
:10F9B00068110020736F636B65745B25645D207351
:10F9C000656E64206275662066756C6C0D0A0000B9
:10F9D000032805DA044A5043044A115400207047B2
:10F9E0000020C04370470000C404000068110020DC
:10F9F000034A1168382389B2994301431160704763
:10FA00000030014000B5154885B0C178002922D1E9
:10FA10000121C170F8F7EEFC1148FAF7C5FD142179
:10FA20006846F5F7E9FB10200090112001900020B6
:10FA30000290039069460B48F9F77AFA01210022F7
:10FA400089020948F9F757FBFF200721413002F0EE
:10FA50002BFD02F03DFD05B000BD000004020020BA
:10FA600064080020000800500004005000B515484C
:10FA700085B08178002922D101218170F8F7BAFC84
:10FA80001148FAF791FD14216846F5F7B5FB1020EF
:10FA900000901120019000200290039069460B48CD
:10FAA000F9F746FA0121002289020948F9F723FBF8
:10FAB000FF200721413002F0F7FC02F009FD05B0FC
:10FAC00000BD00000402002064080020000800506F
:10FAD0000004005010B5FCF707FDF9F757FB10BD07
:10FAE00010B59AB034216846F5F786FB142115A8A5
:10FAF000F5F782FB20210DA8F5F77EFB244801686D
:10FB00000324E402A143C21489180160F9F74AFDF5
:10FB100020480169A14301610E200090FF200130BF
:10FB200002901020049002200990400401210B90C3
:10FB30000001059100240C9003910A946846F9F79E
:10FB400053FF002801D072B6FEE70F201590032066
:10FB50001690179418940121199415A8F9F71AFE14
:10FB6000002801D072B6FEE7A3200D9001204004CA
:10FB70000E9003200F948004149010940DA8F9F7B0
:10FB80004BFD002801D072B6FEE71AB010BD000090
:10FB900000700040401002400249014888607047F0
:10FBA0000050000800ED00E0F0B502680124A40751
:10FBB000144D154E154FA04205D0A84203D0B042B7
:10FBC00001D0B84204D11346702293434A681A43C5
:10FBD000A04205D0A84203D0B04201D0B84204D11F
:10FBE00003231B029A43CB681A4380239A430B6971
:10FBF0001A4302608A68C262096881620121416118
:10FC0000F0BD000000040040000801400014014065
:10FC100030B5026A520852000262026A456883697E
:10FC20007024A3439C080B68A40023430224A2432E
:10FC30008C6845601443836149684163046230BD48
:10FC400030B5026A10239A430262036A45688269EA
:10FC500073242402A2430C682402144320229343F9
:10FC60008A68456012011A438461496881630262AF
:10FC700030BD30B5026AFF2301339A430262026A43
:10FC80004568C3697024A3439C080B68A400234300
:10FC900001246402A2438C68456024021443C361BA
:10FCA0004968C163046230BD30B5026A01231B0399
:10FCB0009A430262036A4568C26973242402A2431C
:10FCC0000C68240214430122520393438A6845605E
:10FCD00012031A43C46149680164026230BD10B561
:10FCE000818CC90707D001684A6801235B049A43E5
:10FCF000836A1A434A60818C890707D501684A687C
:10FD000001231B049A43C36A1A434A60818C490742
:10FD100007D501684A6801239B049A43036B1A4381
:10FD20004A60818C090707D501684A680123DB0313
:10FD30009A43436B1A434A60818CC90607D502680F
:10FD4000916801231B039943836B19439160818C54
:10FD5000890607D501688A6801235B039A43C36B50
:10FD60001A438A60818C490612D503685A680121BA
:10FD70000905046C8A4322435A60026C8A4207D107
:10FD80000268516803235B059943436C1943516032
:10FD9000818C090607D501684A680123DB04806C61
:10FDA0009A4302434A6010BDFEB5074600258037DE
:10FDB00004467D60F9F7A6F90190206800682646A0
:10FDC00000076036002819DA274800900121002238
:10FDD00049052046019B00F03BFC00280ED0EFF3C4
:10FDE0001080012181F3108821680A6880239A43DA
:10FDF0000A6080F310882020E06729E0206800680E
:10FE0000400728D518480090012100228905204686
:10FE1000019B00F01DFC00281DD0EFF31080012194
:10FE200081F3108821680A68FF2321339A430A600E
:10FE300080F31088EFF31080012181F3108821688E
:10FE40008A68520852008A6080F310882020386047
:10FE500035760320FEBD2020E067386025666566A4
:10FE600035760020FEBD0000FFFFFF0110B5806A5F
:10FE70000022014640314A834A82FAF7B6FB10BDA0
:10FE8000F8B5846AE06F254680352E682168896858
:10FE900000270906002906DA212804D15220075339
:10FEA000204600F0CCF820688068400606D5222E57
:10FEB00004D15A200753204600F091F868681021B9
:10FEC000084368602046FAF790FBF8BD70B501461C
:10FED0000968806A096800228906002938DB5A21EE
:10FEE0000A52EFF31081012383F3108803681C6822
:10FEF000FF250135AC431C6081F31088EFF31081BE
:10FF0000012383F3108803689C68640864009C6084
:10FF100081F31088EFF31081012383F310880368C5
:10FF20009C684025AC439C6081F31088202380218D
:10FF30000B50016E01290BD1EFF31081012383F3E4
:10FF4000108803681C681025AC431C6081F310887E
:10FF50004266016E012902D0FAF76AFE70BD58218F
:10FF6000095AFAF71FFB70BD10B5806A012141667E
:10FF7000016E012902D0FAF75FFE10BD5821095A1F
:10FF80004908FAF70FFB10BD10B501460968806AF1
:10FF9000096889061BD4002252210A52EFF310810E
:10FFA000012282F31088026893688024A34393603F
:10FFB00081F31088EFF31081012282F3108800682A
:10FFC000026840231A43026081F3108810BDFAF7DB
:10FFD00027FF10BD10B5806AFAF726FF10BD10B5D7
:10FFE000EFF31081012282F3108802681368FF2466
:10FFF0002134A343136081F31088EFF310810122B1
:020000040801F1
:1000000082F31088026893685B085B00936081F359
:100010001088016E01290BD1EFF31081012282F3C8
:100020001088026813681024A343136081F31088BA
:10003000202280210A5000210166816610BD10B582
:10004000EFF31081012282F3108802681368C02444
:10005000A343136081F310882021C16710BD000005
:1000600070B501464031034680338C8B1D680268B1
:10007000222D04D0906908210843906170BD526A16
:10008000456D22402A80426D921C42654A8B521E69
:100090004A834A8B002AF1D1EFF31082012484F3C2
:1000A000108804682568FF262136B543256082F351
:1000B0001088EFF31082012484F310880468A56887
:1000C0006D086D00A56082F3108820221A6000235D
:1000D00083664366174A046894420ED0626812022F
:1000E0000BD5EFF31082012585F3108825680126D2
:1000F000B606B543256082F31088026E012A02D04D
:10010000FAF796FD70BD0366EFF31082012383F3C7
:1001100010880468256810239D43256082F31088A9
:100120000268D469E443E40600D41362098BFAF749
:1001300039FA70BD0048004070B5014640310346B1
:1001400080338C8B1D680268222D04D090690821B1
:100150000843906170BD526A2240446D2270426D26
:10016000521C42654A8B521E4A834A8B002AF1D1A7
:10017000EFF31082012484F3108804682568FF26B9
:100180002136B543256082F31088EFF310820124F5
:1001900084F310880468A5686D086D00A56082F37B
:1001A000108820221A60002383664366174A046879
:1001B00094420ED0626812020BD5EFF31082012533
:1001C00085F3108825680126B606B543256082F3BD
:1001D0001088026E012A02D0FAF72AFD70BD03666C
:1001E000EFF31082012383F310880468256810233D
:1001F0009D43256082F310880268D469E443E406D5
:1002000000D41362098BFAF7CDF970BD00480040A5
:10021000F8B50446016880682269E669104362699E
:10022000002532431043754B0A68754E3240024335
:100230000A6020684168032212039143E268114377
:1002400041602168A069994201D0226A10438A68FE
:100250000B263602B24302438A606A4922686A4822
:100260008A420CD1C0688007800F06D001283FD099
:1002700002283BD0032827D124E0012725E0634949
:100280008A420AD1C0680C2108402DD004282FD002
:1002900008282BD00C2817D114E05D498A4223D0BE
:1002A0005C498A4220D09A420ED1C1680320800264
:1002B000014019D001208002091A19D0091A15D05D
:1002C000814201D1082700E010274F4952484039A8
:1002D00086009A4234D1002F0CD0022F0DD0042F6B
:1002E00010D0082F7ED128E00027EEE70227ECE7A8
:1002F0000427EAE7F9F71CFB06E00968C90605D4FC
:10030000304603E0F9F734FB002872D062685100F0
:100310005118814266D81103814263D3010E06024F
:100320005008002330185941F4F70CFF032109024B
:100330003A4A411A91425AD954E00120C003E5E7F4
:100340000122E369D20393422AD13B0001F0BDF9B7
:100350000906090C4A114A4A4A264A00F9F7E8FAFE
:1003600009E0F9F7F5FA06E00968C90605D4304650
:1003700003E0F9F7FDFA00283BD0616840004A0825
:100380008018F4F7B5FE0146254A1039914229D864
:10039000511C01400007400F084328E01046ECE7DD
:1003A0003B0001F092F90906090C1F111F1F1F21C4
:1003B0001F00F9F7BDFA09E0F9F7CAFA06E0096883
:1003C000C90605D4304603E0F9F7D2FA002810D068
:1003D00061684A081018F4F78BFE02461049103A7B
:1003E0008A4203D9012504E01046F1E780B2216872
:1003F000C8600020A066E0662846F8BD00480040BE
:10040000F369FFEF00380140401002400044004013
:10041000004C00400050004000093D00FFFC0F0070
:10042000EFFF000070B504464165403002830020B4
:1004300025468035686022212960616F002919D026
:10044000204BCB62636F20491963636F1F49596367
:10045000616F13468863666D216832462431606F90
:10046000F8F7DAFB002805D010206860202028600B
:10047000012070BD206900280CD0EFF3108001210D
:1004800081F3108821680A68FF2301331A430A6048
:1004900080F31088EFF31080012181F31088226827
:1004A00093680B43936080F31088EFF3108081F31F
:1004B000108821688A6840231A438A6080F3108874
:1004C000002070BDCDFE000869FF000881FE000815
:1004D00070B54165014640310A834A830023836633
:1004E000012284681203FF25944204D10469002C80
:1004F00013D1264C0AE07F26002C09D001252D07B8
:10050000AC420CD10469002C05D03F248C8307E059
:100510000469002C01D08E8302E08D8300E08B8380
:10052000014680314B6022230B60EFF310810123E1
:1005300083F3108803689C6801252C439C6081F339
:1005400010888168914202D1016900290ED01049BA
:100550008166016900290BD0EFF31081012282F33B
:10056000108800680268FF23213309E00949816689
:10057000EFF31081012282F31088006802682023C3
:100580001A43026081F31088002070BDFF01000053
:10059000390101086100010810B5C16F212910D18E
:1005A000014640314A8A002A0CD0C26C0368128886
:1005B000D205D20D9A62C26C921CC264488A401E57
:1005C000488210BDEFF31081012282F31088026887
:1005D00013688024A343136081F31088EFF3108124
:1005E000012282F310880068026840231A430260E7
:1005F00081F3108810BD10B5C16F21290ED10146BD
:1006000040314A8A002A0AD0C26C036812789A6282
:10061000C26C521CC264488A401E488210BDEFF36F
:100620001081012282F31088026813688024A3439A
:10063000136081F31088EFF31081012282F3108898
:100640000068026840231A43026081F3108810BDDD
:10065000FFB5064681B080360546044660350A9FE0
:100660002EE0781C2CD0F8F74DFD0499401AB842C2
:1006700014D8002F12D020680168490720D5C1691D
:10068000C94309070CD4082707622046FFF7A7FCD7
:10069000776000202876012005B0F0BD0320FBE73D
:1006A000C069C04300050BD401202168C002086264
:1006B0002046FFF794FC2020706000202876EDE7AC
:1006C0002068C1690298884305D0002103988142BF
:1006D000C7D00020E0E70121F8E70000F3B5FFB044
:1006E0008CB0F849F8A0FAF7FBFD0722F8A18B9827
:1006F000F4F7E2FDF94D01272C46F74E403400286F
:100700003FD00E22F6A18B98F4F7D6FD00286CD0CE
:100710000922F7A18B98F4F7CFFD00287ED008229C
:10072000F6A18B98F4F7C8FD002878D00822F6A12E
:100730008B98F4F7C1FD002872D00922F5A18B989F
:10074000F4F7BAFD00286CD00A22F5A18B98F4F7D3
:10075000B3FD002814D00922F4A18B98F4F7ACFD66
:10076000002872D00922F4A18B98F4F7A5FD002887
:100770006CD00A22F3A18B98F4F79EFD00287DD05F
:100780009EE10C2301AA2C218B98FCF7D3F80528B5
:1007900075D30298FBF759FFA9888842F0D100254C
:1007A0000398FCF7EDF8218E814235D0208632E0A7
:1007B0006946C978A28D91420CD0E08468464078A1
:1007C00020856846807860856846C0780125A085C8
:1007D000002030700598FCF7D3F8E18D884236D0C0
:1007E0000598FCF7CDF8E08510E10C2301AA2C2137
:1007F0008B98FCF79FF80528CAD30298FBF725FFD2
:10080000A9888842BCD100250398FCF7B9F8E18F8C
:10081000814201D0E0870125694603E01AE03DE00E
:100820007AE085E00498FBF71FFF68460078E18CCA
:100830008842C2D169464978228D9142BDD169462C
:100840008978628D9142B8D1B2E7A2E0BEE0002D76
:10085000CAD135E10C2301AA2C218B98FCF76AF848
:10086000032895D30298FBF7F0FEA988884287D128
:100870000398FBF7EAFE012803D101E0CCE0DBE0BE
:10088000B7700398FBF7E1FE022800D1F7700398D8
:10089000FBF7DBFE0328DCD1377111E10C2301AA41
:1008A0002C218B98FCF746F80428A5D30298FBF777
:1008B000CCFEA9888842CCD1A5A10498F4F7D8FC35
:1008C0000028C6DDA54869460880A5A0FAF708FDFE
:1008D000112400232403022221461846FDF78EFB33
:1008E00002236A4621460020FDF700FD092400236B
:1008F000FF226403013221461846FDF77FFB03986F
:10090000F4F7AFFC431C21460020039AFDF7EEFCF0
:100910000A20F8F7B5F9D3E00C2301AA2C218B9813
:10092000FCF708F803289CD30298FBF78EFEC7E07B
:100930000C2301AA2C218B98FBF7FCFF03287BD307
:100940000298FBF782FEA9888842A6D18AA1039863
:10095000F4F78EFC002803D10498FCF711F83081DD
:1009600087A10398F4F784FC002896D185490420D8
:1009700088610402AB8884A221465248FBF7B1FF8C
:1009800002465049F068FEF7E7FFAB887EA2214699
:1009900016E00FA800900DAB80A28C998B98FBF706
:1009A000ADFE022835D10E9A0D99002088540D987D
:1009B000FBF74BFEAB8898422BD1012172A2890232
:1009C0004048FBF78EFF02463E4976E00C2301AA21
:1009D0002C218B98FBF7AEFF00900298FBF735FEB9
:1009E0003E49898888426BD10098022824D3039815
:1009F000FBF7C6FF85B20498FBF7C2FF80B2102D4B
:100A000008D0FF2D02D835496A00885202F086F9D5
:100A1000278455E0308153E00C2301AA2C218B98C8
:100A2000FBF788FF04460298FBF70FFE2B498988E5
:100A3000884245D1022C04D20020C0437FB00EB0C2
:100A4000F0BD0398FBF79CFF84B20498FBF798FF76
:100A500087B257A10DA800F0DFFD85B21F4857A14E
:100A600082880DA8401900F0D7FD281885B23F19DB
:100A70000BE01A486100425A0DA8401950A100F03D
:100A8000CBFD2818641C85B2A4B2A742F1D8652119
:100A90000DA841556D1CA9B26E224254491C89B261
:100AA00064224254491C89B20D224254491C89B225
:100AB0000A224254491C8AB20146F068FEF74CFFF4
:100AC0000020BBE71032002025730D0A0000000053
:100AD000244750535F532C00E401002010360020BF
:100AE00024434841494348554750535F532C000025
:100AF00024726563656976652C0000002475706456
:100B00006174652C00000000246765746C6F672CAD
:100B10000000000024636F6E74726F6C2C00000084
:100B20002475736572646174612C000024736574AC
:100B3000746F6E652C0000002473657470617261BF
:100B40002C0000002472656164706172612C0000E9
:100B5000563230323130353130303000CCCC0000BC
:100B6000676F746F204F5441204170706C696361EE
:100B700074696F6E0D0A0000626565706572000031
:100B800054545300000C0050245265636569766527
:100B9000766F6963652C25580D0A0000247365740F
:100BA000746F6E652C25702C25700D0A00000000F6
:100BB000247265706C79706172612C0025782C004C
:100BC00025642C0030B51D4C89B02078022832D124
:100BD000FCF7AEFD1A4B1B4A1B49A5791B7812780E
:100BE0000978089505AD0EC5184963794A880390C0
:100BF000D5B2120A0192164802950493007800902B
:100C00008B88012113A289021D48FBF76AFE054665
:100C1000A0792A46401CA0711949E068FEF79CFEA5
:100C20007D23AAB2DB0016491648FAF706F82946D2
:100C30001348F4F7E1FA002009B030BDE4010020C8
:100C4000020000200A0200200700002010360020C9
:100C500001000020245854422C25582C2530327590
:100C600025252C25642E25642C25732C25642C31F8
:100C70002E2C25642C25642C25642C256400000072
:100C800010320020DC07002010B50023034A0221A7
:100C90000348FEF7A5FC002010BD0000310D01083F
:100CA000F00100203EB5FCF79FF800251849194CCB
:100CB000012803D00D60257000203EBD11200002E8
:100CC0000860207800280ED00228F5D1FBF78CFBB5
:100CD0002169114A411A9142EED365702061FFF7F4
:100CE00071FF6571E8E701200C4D2070288DAA8DF9
:100CF000698D6B4607C30121EB8C09A289020B4861
:100D0000FBF7EFFDEA8D0949E068FEF749FCD3E700
:100D100024000020E4010020881300005036002049
:100D200025752E25752E25752E257500103200206F
:100D300038B5114800240278002914D0012916D0B2
:100D4000022912D003290DD100946B460B4A0C499D
:100D5000C068FEF76FFD002804D10948009944548B
:100D6000FFF7BCFC38BD012AFCD1047038BD012A54
:100D7000FCD10221017038BDE4010020FF03000016
:100D80001032002070B5FBF72FFB0B4D6969401A3C
:100D9000C8280ED3FBF728FB084C68612278084965
:100DA000E868FEF7D9FD21780548F4F725FA002018
:100DB0002070002070BD0000E4010020A20100208E
:100DC0007824002070B5114C0D46217802291AD1E3
:100DD0000F49A2698B1801462A461846F4F7F3F921
:100DE000A0694019A061FBF7FFFAE169401AC82821
:100DF00009D3FBF7F9FAE0610549A269E068FEF75B
:100E0000ABFD0020A061002070BD0000E4010020C7
:100E1000102E002010B50248F9F7ECFB10BD0000C1
:100E2000DC07002010B50248F9F7E4FB10BD000014
:100E30006408002010B50248F9F7DCFB10BD000083
:100E4000EC080020F8B51D4D0E0034D0042832D235
:100E5000742148431A494418A078002802D0012878
:100E600022D028E0E168A068421860680090406FD6
:100E7000006840682769101A0818C01BF4F738F991
:100E8000012905D817D100980068C069800612D4DE
:100E90003878307061692069884201D1A06800E02B
:100EA000401C2061002506E0204618303146FAF744
:100EB0003FF90028F6D02846F8BD0000FFFFFFFFED
:100EC000402C0020002901D0042802D30020C04378
:100ED000704774225043034A80184068086000201D
:100EE00070470000402C002070B50C00064601D071
:100EF000042E02D30020C04370BD74214843214911
:100F00000E54227845186A706078A8706068A860EE
:100F1000A168E9606278002A02D0012A05D00BE0BE
:100F200028614018401E686106E0284618300123F9
:100F3000A2686168FAF7D7F8E068E8622069286378
:100F4000A0692867606968632078002801D00128BB
:100F500006D121460C310EC928463830FBF7BCFDBE
:100F60006078002804D0012806D0022804D006E0CA
:100F7000304600F009F802E0304600F021F8002089
:100F800070BD0000402C002038B50C49742250433D
:100F900042185068016804E04C6A6B461C801C884B
:100FA0001C80CB691B07F7D491681161D368CC18FA
:100FB000641E54619AB2F9F7D7FD38BD402C002069
:100FC00074214843044910B540180146683140680F
:100FD0000122F9F7FBFD10BD402C002070B50E4634
:100FE000044674200A49604345186868F9F7DCFA3A
:100FF000686846606868F9F753FC002802D0002052
:10100000C04370BD204600F005F8002070BD000010
:10101000402C002070B5054674201A4968434418D6
:10102000A078002802D0012807D00DE0A068206138
:10103000E1684018401E606106E020461830012338
:10104000E268A168FAF74FF86078002801D001281B
:1010500006D121462C310EC920463830FBF73CFD25
:10106000A078002804D0012806D0022804D006E089
:101070002846FFF789FF02E02846FFF7A1FF00207E
:1010800070BD0000402C002070B50D0001D0042878
:1010900002D30020C04370BD742148430449441862
:1010A00074212046FBF7A0FA0020656070BD0000A7
:1010B000402C002010B502460E4900207423434303
:1010C0005B185B6893420FD17422424351188978B0
:1010D000002906D0012901D0022901D1FFF770FFB4
:1010E00010BDFFF751FF10BD401CC0B20428E5D36E
:1010F00010BD0000402C002038B5014613480024E4
:1011000074226243121852688A4219D174216143D1
:101110000818817801290BD0022908D1016F002914
:1011200002D0806EC0B288472046FFF749FF38BD25
:10113000816E6A46117069461830F9F7B9FFF3E716
:10114000641CE4B2042CDBD338BD0000402C00202A
:10115000F7B582B00021009103991546002903D00C
:10116000002D01D0042803D30020C04305B0F0BDFA
:10117000742148432B494618707834463834002887
:1011800004D0012820D0022842D049E0FAF7D2FF4B
:1011900020462946FBF772FC070033D0204639462B
:1011A000FBF738FC2A4638680399F4F70CF8204618
:1011B000FBF746FC0446FBF7ABF9A088216882B236
:1011C0007068F9F79BFD2BE0FAF7B4FF204629463B
:1011D000FBF754FC070015D020463946FBF71AFCF4
:1011E0002A4638680399F3F7EEFF2046FBF728FC00
:1011F0000446FBF78DF9A088216882B27068F9F780
:10120000D3FD0DE0FBF784F90020C043009007E018
:10121000134664204343AAB270680399F9F70DFDA1
:101220000098A3E7402C002070B51F4A00217423CA
:101230004B439B185B68834231D1742041438C1827
:101240006078002816D0012813D120463830054692
:10125000FBF7F6FB01462846FBF7C6FB2846FBF7E3
:10126000EFFB002805D081888AB201686068F9F731
:101270009BFD70BD204638300546FBF7E1FB01467B
:101280002846FBF7B1FB2846FBF7DAFB0028F0D035
:1012900081888AB201686068F9F730FD70BD491C29
:1012A000C9B20429C3D370BD402C0020F8B5002575
:1012B000184C194F64280CD0622826D0602807D11A
:1012C000258401F02BFD6420F6F7E0FB1348C7608E
:1012D000F8BD13486946088072B680211148F6F7B8
:1012E00077FC064607E080210E48F6F771FC0646BB
:1012F000C820F6F7CBFB002EF5D00222694609483C
:10130000F6F710FD62B6A584DBE702486584403835
:101310000580D6E7503600200400FA0500ED00E015
:10132000CCCC0000384A0008F8B5414C00232178A5
:10133000404A1D46082910D007294ED0062957D00B
:10134000052959D004295AD003295BD000295DD042
:1013500001295FD0022961D062E0A17800264A1FEE
:1013600004E0344FBF5DFB189BB2761C9642F8DB5D
:10137000627927799B185B18E1785E186378F61814
:10138000F6198019C00723D0012A1DD0022A1FD1C7
:1013900028480078012802D10846FFF787FF264831
:1013A000E178627840182349F3F70DFF01F0B6FCAD
:1013B0006420F6F76BFBBFF34F8F21491F48C860CD
:1013C000BFF34F8F00BFFDE749081846FDF79CF8B3
:1013D0002570E570A570A571F8BDA1795054491C20
:1013E000C8B2A071A178491F8842F5D1082001E058
:1013F000607007202070F8BDE0700620FAE7607189
:101400000520F7E7A070E5700420F3E7552807D121
:101410000120EFE7AA2803D10220EBE7032803D03D
:101420002570E570A570F8BD032020702071F8BD0F
:1014300088030020C03C0020103600200400FA057C
:1014400000ED00E010B5084C04212046F7F74EFEF1
:10145000002807D1012204212046F7F74CFE03A003
:1014600000F0B0F810BD0000000800504C4F524191
:101470005F63735F6572726F720D0A00F0B5484862
:101480000023027885B0551E31E00020D41A641E76
:1014900029E0444F41007E5ACF19BE467F88BC46A2
:1014A00066451ED9404F7F5A0296404E0097365CE3
:1014B00003963D4E8E19019677883B4E7752394FF1
:1014C00066467E52394909188C464E7837490E5483
:1014D000019F009E7E807146029E4E806146039E63
:1014E0004E70401C80B28442D3DC5B1C9BB2AB428A
:1014F000CBDB2F492A4D887903012E480078400024
:101500000343082A01D908202870294C12200A34E4
:10151000A0702A78284E900010180F30E0702448F0
:101520003688C6810889A071060AE671401C0881C8
:101530002248007820726372214B1888888200202C
:10154000188020736073A073E073227420465200E9
:1015500015491130F3F737FE287812494200101967
:101560001130F3F730FE2A7810499000001911303D
:10157000F3F729FE287881004118A01C0F31F6F7F7
:101580003BF96946088028788100401869460019AF
:101590000978417469464978817405B0F0BD00004E
:1015A00059030020A83B0020583B0020F83B0020B6
:1015B000040200200900002090000020010000200B
:1015C0009E0300200FB410B503A9044B044A0298EF
:1015D00000F054FA10BC08BC04B01847E129010817
:1015E0007C0600200FB41CB50246002007AC002981
:1015F0000BD0491E01910092064B6A46214606987F
:1016000000F03CFA009A002111701CBC08BC04B028
:1016100018470000B52101080FB410B504A9074B05
:1016200002AA039800F02AFA044602A9002000F05A
:10163000CCFD204610BC08BC04B01847CB210108E3
:101640007CB51546024600201C4600290BD0491ED9
:1016500000920191044B6A462146284600F00EFA9A
:10166000009A002111707CBDB52101082021020CD7
:1016700001D010211046020A01D010460839020993
:1016800001D01046091F820801D01046891E420869
:1016900001D0881E7047081A7047F8B5040C8BB249
:1016A000264682B25E430D0C1046370C5843360472
:1016B00080190021794116466E43370C3604801993
:1016C000794126466E438919F8BD30B47446641ECC
:1016D0002578641CAB4200D21D46635D5B00E318B5
:1016E00030BC18478307FF22DB0E9A408907090E9A
:1016F0009940002808DB830809489B001B181868DC
:1017000090430843186070470007000F08388308AB
:1017100004489B001B18D86990430843D861704760
:1017200000E400E000ED00E0004870478006002083
:1017300001480068704700008006002002E008C8E9
:10174000121F08C1002AFAD170477047002001E03B
:1017500001C1121F002AFBD1704700000149086037
:10176000704700008006002008B50021684601701F
:101770006B46012202212C2001F0DEF8022168468E
:1017800001706B4601222C2001F0D6F808BD000044
:1017900038B504466D20694608706B46012207493A
:1017A0002E2001F0C9F80649002C01D0054A00E0BE
:1017B000054A2E2001F0A6F838BD000006080000FA
:1017C00006180000070600000716000038B504469A
:1017D0006B4602220021362000F080FFB321230057
:1017E000FFF773FF0E0F08153A3A3A3A1C273A3AB8
:1017F0002F34483A0021684601704078410849007A
:1018000014E06946087880088000401C04E06946BE
:10181000087880088000801C08701DE06846027807
:101820000A40483202704178802001436846417086
:1018300012E0684602780A40027040784106490E7C
:10184000F4E7694648780221084303E0694648788E
:10185000FD210840694648706B4601220021362070
:1018600001F06AF8012200AB11463620013301F085
:1018700063F838BD69460878CF21084069462030B2
:10188000CAE708B5032168464170012101706B4623
:1018900002220021362001F04FF80122D203062156
:1018A0002D2001F02FF8012000F0A9FC0120FFF706
:1018B0008DFF08BD08B5020A69464A7008706B467C
:1018C000022204212D2001F037F803206946087018
:1018D0006B46012206212D2001F02EF800206946DA
:1018E00008706B46012206212D2001F025F80A21FF
:1018F0002D2000F0D9FE08BDF0B51FB486B00998C0
:10190000089A030D0021024314D05148514A181877
:10191000504305141198012810981AD0281A401C19
:1019200000264D4F4D49009601910490002812DA8F
:10193000444211E01198012449A3012801D11098D3
:10194000C1430698119A84600360C26041600BB085
:10195000F0BD4042E4E70446210500203F4A001C58
:1019600051410391029012E0E00707D032463B4616
:1019700001990098F3F7ACFD0191009032463B4687
:1019800010461946F3F7A4FD06460F466410002CD6
:10199000EAD10498039B0028029A0999089806DA6C
:1019A000F3F796FD019B009AF3F792FD05E0F3F73C
:1019B000F7FD019B009AF3F7F3FD04460E46002263
:1019C000284BF3F7C1FE03D80020C043014607E0CF
:1019D0000022254B20463146F3F7C8FCF4F762F8A5
:1019E000102409E0002C0ADB0A220023F3F7AAFBEB
:1019F000079B30321A55641E02460A43F2D1112267
:101A0000641C079B121B1C19119B012B03D0012383
:101A100008430ED10AE0084304D0112010900020A2
:101A2000119077E71098151A6D1E0BE010988242FE
:101A300002DD00236D1C03E0824201DA00236D1EEB
:101A4000002BEED0069811998260C16030C07EE70D
:101A500001FCFFFF104D0000000014400000F03FAB
:101A6000300000000000F0430000E03F30380A285A
:101A700001D201207047002070470000FFB597B0E9
:101A80000646002518E2252877D100242746FD497F
:101A9000049400E00443761C32780120203A904000
:101AA0000842F7D130782A280ED002223078014639
:101AB0003039092916D804990A2359433039401876
:101AC0001443761C0490F1E7189802C8049118900A
:101AD000002904DA01204003044348420490022014
:101AE0000443761C30782E2814D1042004437078E7
:101AF000761C2A2809D11898761C80C8189009E00D
:101B00000A214F43303FC719761C307801463039DF
:101B10000929F5D930786C2810D006DC4C281AD069
:101B200068280ED06A2817D104E0742813D07A28C8
:101B300012D110E00120400504430CE00121090509
:101B400001E0032109050C437178814203D1012092
:101B500000052418761C761C3078119066280BD06E
:101B600013DC58287DD009DC00287BD04528F6D02E
:101B70004628F4D047281AD1A5E118E0632835D0CB
:101B8000642870D0652812D19DE170286CD008DCE3
:101B90006728F1D069287BD06E280DD06F2806D138
:101BA000BAE073282ED0752871D0782859D01A9AA7
:101BB000199990476D1C7EE16002400F022809D000
:101BC00003280DD00428189801680DD00D60001D61
:101BD000189070E11898EA1701680D604A60F6E7FE
:101BE000189801680D80F2E70D70F0E718986A46C2
:101BF00001781172001D18900020507202A8009008
:101C0000012005E0189802C8189000200091C043F8
:101C100061070DD5002101E00199491C0191B942EC
:101C200012DA8142F8DB009A515C0029F4D10BE012
:101C3000002101E00199491C01918142FADB019ADE
:101C40000099895C0029F5D1019904981A9B471ADB
:101C500021463846199A00F097FA0199401945181B
:101C60000BE04FE02CE113E04EE000980099007883
:101C7000491C00911A9A199990470198401E0190A9
:101C8000401CF2D1214638461A9B199A10E137E0E0
:101C90000A200021009001916002410F022907D023
:101CA000189A01CA1892C2179446032908D00AE06C
:101CB0001898C01DC108C90005C91891944607E0CD
:101CC00000B2C2179446042902D140B2C1178C4613
:101CD00000226146944506DA0A46002140429141BD
:101CE0008C462D2102E0210504D52B216A46117373
:101CF000012103E0E10701D02021F7E7029155E03F
:101D00000A200AE0102008E01020009000210420A2
:101D100004430191082703E008200021019100906D
:101D20006002410F022907D0189A01CA18920022B6
:101D30009446032908D008E01898C01DC108C900BE
:101D400005C91891944603E080B2042900D1C0B2BD
:101D500000210291210729D51199702906D0009AF6
:101D60001021019B4A401A4305D00EE040216A46EB
:101D70001173012108E06146014306D030216A4613
:101D800011731199517302210291009A0821019B4C
:101D90004A401A430AD16146014301D1610705D582
:101DA00030216A46117301217F1E02911199582931
:101DB00004D035A10E910DA90D910DE037A1F9E7E1
:101DC0006146019B009AF3F7BDF90E9B8C469B5C24
:101DD0000D9A521E0D92137061460143F0D10D9879
:101DE00005A9081A20300190600703D501200004DE
:101DF000844300E001270198874201DD381A00E0A2
:101E00000020019900904118029809180498401A7E
:101E10000490E00306D421461A9B199A049800F016
:101E2000B3F94519002706E003A81A9AC05D19996D
:101E300090476D1C7F1C02988742F5DBE0030CD5B0
:101E400021461A9B199A049800F09EF9451904E05E
:101E50001A9A3020199990476D1C0099481E0090DD
:101E60000029F5DC08E00D980D990078491C0D91CA
:101E70001A9A199990476D1C0199481E01900029E2
:101E8000F1DC63E109280100303132333435363773
:101E900038396162636465660000000030313233B6
:101EA0003435363738394142434445460000000056
:101EB00000F05AF94519761C3078002800D0E2E588
:101EC00028461BB0F0BD600700D406271898C01D37
:101ED000C108C90048680A680831C30FDB071891B8
:101EE000190001D09CA108E0210501D59BA104E0C7
:101EF000E10701D09AA100E09AA1430011985B0884
:101F0000109165280CD006DC452809D046281DD044
:101F1000472841D141E0662818D067283CD13CE0F1
:101F20000021112F01DB112000E0781C01910090AD
:101F300008A911A8FFF7E0FC139905910021119A57
:101F400015927F1C12980197009150E00120C00764
:101F500003900120019008A9009711A8FFF7CCFC7D
:101F6000139A149905920022119B009212981593CE
:101F7000059A0192002901D0104602E0791C401810
:101F80000190381A01D5019804E04042401E0090AB
:101F9000781C0190C01B029043E0012F00DA01275A
:101FA0000021112F01DD112000E038460191009041
:101FB00008A911A8FFF7A0FC13990591119A002117
:101FC000129815920091019721070CD40599B942F6
:101FD00001DB019900E00191012904DD159A491EF8
:101FE000515C302906D0B84201DA011D05DA012121
:101FF000029115E00199491EEDE7002805DC0099E2
:10200000411800910199091A03E0019A411C91427B
:1020100000DD01910099401A401C02900120C00788
:102020000390200706D402990198814202DB002028
:10203000C043029000206946C87707AF012103988A
:102040000337C907884224D0022011902B20129018
:10205000039800280CDA404203902D20129007E0EC
:102060000A210398F3F744F830317F1E039039704A
:102070001199481E11900029F2DC03980028EFD135
:10208000791E129808703078202108404530BF1E14
:10209000387006A8C01BC01D039010980078002857
:1020A00000D00120019941180298C017091803981F
:1020B00009180498401A401E0490E00306D42146F3
:1020C0001A9B199A049800F05FF845191098007847
:1020D000002803D01A9A199990476D1CE00324D563
:1020E00021461A9B199A049800F04EF845191CE0F5
:1020F0000098002807DB00990598884203DD1598B1
:10210000405C199901E0199930201A9A904700987B
:102110006D1C401C00900298401E0290002804D1C3
:102120001A9A2E20199990476D1C0199481E01900A
:102130000029DDDC05E038781A9A7F1C1999904750
:102140006D1C0399481E03900029F4DC21461A9B5C
:10215000199A0498ACE600002D0000002B00000046
:102160002000000000000000F8B5044600251E46CF
:102170001746880404D405E039462020B0476D1C7A
:10218000641EF9D52846F8BDFFB50446002581B088
:102190001E46C80301D5302700E02027880404D557
:1021A00005E038460399B0476D1C641EF9D52846F2
:1021B00005B0F0BD4A68002A06D00A68531C0B60BF
:1021C00010704868401E486070470A68531C0B60D6
:1021D0001070704730B583B00446FFF7A9FA054682
:1021E000002000900246019021466846F3F74BFB21
:1021F0002846FFF7B3FA0199009803B030BD7D215E
:1022000010B5C9004843F5F748FC10BD002140E077
:1022100000BF00BF00BF00BF00BF00BF00BF00BFC6
:1022200000BF00BF00BF00BF00BF00BF00BF00BFB6
:1022300000BF00BF00BF00BF00BF00BF00BF00BFA6
:1022400000BF00BF00BF00BF00BF00BF00BF00BF96
:1022500000BF00BF00BF00BF00BF00BF00BF00BF86
:1022600000BF00BF00BF00BF00BF00BF00BF00BF76
:1022700000BF00BF00BF00BF00BF00BF00BF00BF66
:1022800000BF00BF00BF00BF00BF00BF00BF00BF56
:10229000491C8142BCD37047FEB504460020019022
:1022A00000906079734940000E5A61782578491E84
:1022B0007148CFB20163042D77D0072D75D000216E
:1022C0000291217801736C49E379012292058969B1
:1022D000002B6CD0914381616748217A4173217A48
:1022E00082698907890B0A4382610021042000F07A
:1022F00014FB324661492E2000F004FB3846FFF7FC
:1023000047FA5F4E0522705D810040185D49431811
:1023100007212B2000F010FB5B49029801220B18CB
:102320000B21282000F008FB705D584980000A58F6
:102330000C21282000F0F1FAE0795549800040187E
:10234000A1794900425A0221272000F0DBFA5148C6
:102350007E00825B0421272000F0D4FAE079002877
:1023600029D0A07804282CD0282069460872202281
:102370000621272000F0C6FA02AB012226212720E1
:1023800000F0DAFA444938014018E17889004258EF
:102390000821272000F0C1FAA17A601C627A0902A4
:1023A000114313D016E000E001E0012188E711435A
:1023B000F608816190E764220621272000F0A2FA46
:1023C000E0E71020694608720246D1E733490172FE
:1023D000090A4172417A007A0A0202432021272029
:1023E00000F090FA2E4F0C2123203A6800F095FA65
:1023F000F01982880421232000F084FAA0790028B3
:102400000BD0E0792749012243180021212000F058
:1024100093FA03200190012000902A07120F100167
:102420000243607800218007000B024301980005F9
:1024300002430098400402432079C0064009024349
:102440006079C00602431F2000F067FAA078617827
:102450000123084302040848DB030261E1794903D0
:1024600019430A4302610021082000F056FA0020B7
:10247000FEBD0000C4330108883D00200428000090
:102480006C330108A3030020C1030020743301084A
:1024900094330108A0330108A4330108411000005F
:1024A0008C330108C303002038B50C4607498A8BDA
:1024B000002102432C2000F025FA684604706B4688
:1024C000012206212C2000F037FA38BD883D00207B
:1024D00010B5FFF749F910BD10B5044604213620A8
:1024E00000F0E2F80121C902002C01D0084300E00D
:1024F000884302460421362000F00FFA10BD000088
:1025000038B540206946087000210E2000F0CCF854
:102510000446002211460E2000F0FFF96B4601220E
:1025200000210D2000F008FA074A00210F2000F0DA
:10253000F4F900F0CDF9224600210E2000F0EDF96B
:1025400002480021017338BDF8FF2724A83D002070
:102550007CB50646042069460870434C002060752F
:1025600021462031206348710873A0836063A06313
:1025700000F0AEF83D4D206002E000F0A9F82060C8
:10258000A842FAD10020FFF721F939484321017010
:10259000384A00211E2000F0C0F96B4601220021BC
:1025A000242000F0C9F91E20FFF784F985B2280A1B
:1025B000A0730420FFF77EF90006000E0DD0022064
:1025C0006946087101AB012212212D2000F0B4F9F7
:1025D000A08B012109030843A08300F079F8206053
:1025E0000620FFF767F960600720FFF763F9A06036
:1025F000E806C00E207501D110202075C0B200F091
:10260000D7F9F00707D0FFF73CF9A08B0121C902E9
:102610000843A0830AE00521362000F02FF8164970
:10262000084002460521362000F06CF90120FFF732
:10263000CDF80021042000F037F8A0610021262009
:1026400000F032F8152189030843024600212620B4
:1026500000F063F900222621362000F053F900F043
:1026600037F8206000207CBD883D00203001CADEA4
:10267000A20300201F1F1F1FFFFD000038B5094CDB
:1026800089B280B26B46022200F028F8002806D1F9
:1026900068464078010268460078081884B22046EF
:1026A00038BD0000FFFF000038B50024E44389B2C4
:1026B00080B26B46042200F011F8002806D10321F5
:1026C0006846435C2202D418491EFAD5204638BD1C
:1026D00010B500210846FFF7E7FF10BD38B5002907
:1026E00009D0402420436C462070C8B27F2906D808
:1026F000607002200AE069460870012006E080242C
:1027000020436C466070C809A0700320694600F041
:10271000C9FA38BD10B5144603460A4621461120B1
:10272000FFF7DCFF10BD10B5034605220021152080
:10273000FFF7D4FF10BD38B5054600206946087084
:1027400000F0C6F8FF2401342246002D01D00322F8
:10275000120200210D2000F0D5F8002D13D06B4699
:10276000012203210F20FFF7B9FF68460078000718
:1027700009D5FFF7C5FE224600210D2000F0C2F862
:102780000020C04338BD002038BD10B502460121ED
:102790000A2000F0C2F810BD70B50D4604460021B5
:1027A0000E20FFF781FF002D01D0204300E0A04361
:1027B000024600210E2000F0B0F870BD10B50246B0
:1027C00002492E2000F09EF810BD00000418000001
:1027D000F8B505466B46012203210420FFF77EFF72
:1027E0000126114C3607002D0DD02A4600210C2061
:1027F00000F088F869460878102108436946087097
:10280000A069304307E069460878EF21084069462F
:102810000870A069B0430B46A06101220321042087
:1028200000F08AF8F8BD0000883D002010B502468F
:102830000021182000F066F810BD0000F8B507462A
:10284000002568460570B807204C2E4600280ADA95
:102850008020694608706B46012200210D2000F09F
:102860006BF801202073F8076946087821D006210B
:102870000843694608706B46012200210D2000F0D4
:102880005BF803210F20FFF7F9FE8121C900084200
:1028900019D04020694608706B46012200210D20A6
:1028A00000F04AF80020FFF717FE00252673ED43DD
:1028B00009E002210843694608706B4601220021A5
:1028C0000D2000F039F82846F8BD0000A83D002092
:1028D0001CB56B46012203210F20FFF7FFFE68465F
:1028E00000784022C1091040C9014000814208D04F
:1028F000012069460871024601AB03210D2000F05A
:102900001BF81CBD08B56B461A70120A5A7089B2C2
:1029100080B2022200F010F808BD38B500236C46E2
:10292000E254120A5B1C042BFADB89B280B2234604
:10293000042200F001F838BD38B58024002909D000
:10294000C02528436D462870C8B27F2907D8687013
:10295000022009E0204369460870012004E020437A
:102960006870C809A8700320694600F0FDF938BDF9
:1029700010B51446012312189B029A4202D9002076
:10298000C04310BD0B46821E21460920FFF7D4FF2D
:10299000002010BD10B5054A8905126901430A439C
:1029A00000210820FFF7B9FF002010BD883D00205E
:1029B00038B504466B4601220E212B20FFF78EFE10
:1029C00068460078E10640094001C90E01436846A7
:1029D00001706B4601220E212B20FFF7ADFF38BDA1
:1029E00013B501231A4669460248F8F726F90098FC
:1029F0001CBD0000DC07002008B5F6F7CFFBFDF793
:102A00006FF8694867490160062141606749C16004
:102A10008160F6F77DFB002801D072B6FEE7FAF779
:102A2000ABFB6348016B012211430163006B104053
:102A30000022009011460A20F6F7A2FD0A20F6F7C0
:102A400093FD002211460B20F6F79AFD0B20F6F7B6
:102A50008BFD554857494030002412C07F2101604A
:102A60008460C4600461FF21446141600838F7F765
:102A7000D5F9002801D072B6FEE7FAF701FDFAF7A2
:102A8000E3FCFAF761FCFAF73FFB47484A4910308C
:102A900012C004608461C46148490462C16008389E
:102AA000F6F78CFC002801D072B6FEE7FAF7B0FC0E
:102AB000FAF76AFC3C490020FC31FEF7E5FA404990
:102AC0000320FEF7E1FA3E4902208839FEF7DCFADE
:102AD000354900206431FBF7A3FC3A4C01229202F5
:102AE00021460020F3F73EFD012221460220F3F7A4
:102AF00039FD354D0122520329460120F3F732FDFD
:102B0000102229460020F5F75DFC002120232246F3
:102B10000846FBF745FB0020FBF7AAFAF4F798FEFE
:102B2000FBF760FFFAF7AAFFF5F708FAFAF754F98E
:102B3000FEF7AAF801220520D1030007F6F7DBFA19
:102B4000F4F7F2FF0721A015FFF7AEFCFAF7C0F982
:102B5000FF24F5342046F6F793F8134800221B496A
:102B60001030F6F79FFC002801D072B6FEE7112066
:102B7000000403461A461146FBF706FD2046F6F709
:102B80007FF8FBF71FFD2046F6F77AF8F5F79AF97C
:102B90002046F6F775F8F5F7ADFC0D494870FAF7E1
:102BA0008BFCFCE700300040E0060020FF0F000037
:102BB0000010024000280040007C0040FFFF0000A1
:102BC000EC0800200004005000080050FF7F0000C7
:102BD00000000020F8B5012252022B492B48F5F7DE
:102BE00017F829482A490288044600257926212712
:102BF00040348A4237D00180264981807D21C90036
:102C0000C1800A2101811E214581C94381810121A1
:102C1000C18185836183022202877822428781876E
:102C2000C187E58225846584A584C583A580272185
:102C3000E1846A212185D22161850D21A185164972
:102C4000E1856686A786E221E1862A21218713494C
:102C500061874B21C9002186E121C900E187052157
:102C6000818200F05BF86584A5842584608E0C4920
:102C7000884207D16686A786E220E0862A20208740
:102C800006486087F8BD00001036002000F80108F3
:102C9000AA55000072180000581B00004F230000C6
:102CA000FFFF0000FFB581B01D4616460746002411
:102CB000FEF7C8FB102105231B0799620E4808E0A8
:102CC000029A125DC2608268D207FCD0C2682A7084
:102CD000641CBC42F4DB0022174606E0C76084682F
:102CE000E407FCD0C468AC54521CB242F6D39961DC
:102CF000002005B0F0BD000000300140F8B51546D9
:102D00001E4607460024E20028463146F2F74AFAFA
:102D10003855641C042CF6DBF8BD000070B572B6A3
:102D200001250C4E6D0229463046F4F751FF04464A
:102D300007E029463046F4F74BFF0446C820F4F775
:102D4000A5FE002CF5D02A4603493046F4F7EAFFE9
:102D500062B670BD00F8010810360020002100E0C6
:102D6000491C8142FCD37047FFB581B015460F4620
:102D700006460024FEF766FB102205231B079A6215
:102D80000D4906E0385DC8608868C007FCD0C86897
:102D9000641CB442F6DB002007E0049C245CCC6099
:102DA0008C68E407FCD0CC68401CA842F5D39A613B
:102DB000002005B0F0BD0000003001400000000020
:102DC00000000000010203040607080903040608C6
:102DD0000C10182030000000000102030400000065
:102DE0006C390108020000002439010802000000CB
:102DF000C436010803000000783A0108030000000F
:102E0000503601080700000058360108080000008D
:102E10001037010809000000B43601080A0000005C
:102E2000CC3501080B000000A03601080C000000A2
:102E300030370108100000006C3601081100000056
:102E4000BC360108120000001C39010818000000FF
:102E500070390108190000008836010816000000CA
:102E6000A434010814000000903401081A00000086
:102E70000436010817000000103601081B0000008E
:102E8000243B01081C000000FC3601081D00000066
:102E90007C3601081E000000F03601081F0000000B
:102EA0000437010820000000F0350108210000006F
:102EB000183601082200000028360108230000000F
:102EC000D8350108240000007436010825000000F0
:102ED000B0350108260000007C34010827000000FE
:102EE000943601082800000044360108290000003B
:102EF000A83601082A000000E43501082B00000074
:102F0000C03501082C000000D03601082D0000005B
:102F1000243701082E000000183701082F00000098
:102F20006036010830000000E4360108310000007E
:102F3000FC350108150000001C3C010832000000AF
:102F4000DC36010833000000383601083400000088
:102F5000B434010835000000D43401083600000004
:102F6000EC34010837000000043501083800000087
:102F70001C35010839000000343501083A00000012
:102F80004C3501083B000000643501083C0000009E
:102F90007C3501083D000000943501083E0000002A
:102FA000AC3501083F000000203C0108443B01080B
:102FB00058390108643A0108AC3B0108483A010855
:102FC00044390108B4380108C83801087C3B0108BD
:102FD000343A0108183A0108EC390108903B01081D
:102FE000F43B010894390108F4380108983A0108C3
:102FF000803A01086C37010850370108F83701089A
:10300000D83901080C3801082C3901087C3901082D
:1030100088380108E43701080C3B0108503B0108DF
:10302000A83901082C3B0108643B0108CC37010892
:10303000203801083C3801089C370108083901088C
:1030400034370108F43A0108C03901087038010822
:10305000003A0108B437010884370108B03A010882
:10306000DC3B0108C43B0108DC380108DC3A0108FC
:10307000083C0108C83A0108583801089C38010882
:10308000C0340108D8340108F034010808350108BB
:103090002035010838350108503501086835010828
:1030A0008035010898350108A83C0108000000009F
:1030B000D8300108A96B0008383D0108A830010884
:1030C000D8300108C1680008CC3C0108A8300108CC
:1030D00000000000A56A0008FC3C0108B8300108A7
:1030E00000000000F56A0008683D0108B8300108DA
:1030F00000000000056200089C3D0108B83001088E
:1031000000000000FD710008543D0108B8300108BE
:1031100000000000C1600008C03C0108A8300108A0
:1031200000000000A56800087C3D0108A8300108E7
:10313000E4310108156C0008443D010828310108FC
:1031400000000000316600088C3D010828310108AC
:10315000583101082D680008EC3C0108483101088D
:1031600000000000F1670008DC3C0108483101085C
:1031700000000000B1650008843C010888130000CD
:1031800001000000703C01088813000001000000ED
:10319000643C010888130000010000007C3C010829
:1031A0008813000001000000443C0108881300005F
:1031B00001000000543C01088813000001000000D9
:1031C0002C3C010860EA000003000000903C01086C
:1031D00060EA0000030000009C3C0108E8030000D6
:1031E00005000000B43D010828310108000000007E
:1031F0007D6C0008F83D010848310108000000001E
:103200008D6E0008E43D010848310108000000000F
:10321000C96D0008CC3D01084831010800000000DC
:10322000297000082052D800001000000080000023
:1032300000000100DC3F01088DF40008D43F0108C4
:1032400079EC0008C03F01081DEC0008103F0108A0
:10325000A1EB0008B83F010819EC0008583F01082D
:10326000F1F10008503F0108D5E80008443E01088C
:10327000D9E500082C3F010809E80008E83E0108EC
:10328000C1E700088C3F01081DE600089C3F0108CB
:10329000F9EA0008383F010869EB0008F43E01082C
:1032A00031EB0008B43E010891F40008BC3E01086F
:1032B00045F30008AC3F0108A1F200084C3E0108AC
:1032C000E5F30008A83E01080DF20008583E010889
:1032D00055E60008C83E01084DE80008D83E010840
:1032E00085EC0008383E01083DE70008443F01082E
:1032F00005F000086C3F0108A9F10008783F0108BB
:1033000061F10008043F010839EF0008843E01081C
:1033100049ED0008F03F010835EE0008643E010861
:10332000A9EE0008743E0108D1F00008603F0108D2
:10333000C1ED0008283E0108F5EA00082C3E01080E
:10334000F1EA0008003F0108F9E90008203F010800
:1033500069EA0008C83F01089DEA0008983E010894
:1033600019E60008E43F010889F4000800000102A2
:1033700003040005405C0000A05C0400C06C080071
:10338000805C0400E03F1E00E07D1E0007A90225CE
:1033900070889B880A0016000100060001000200E8
:1033A00087008D002D001A3152001A339A001A3509
:1033B0001D011A376B003B31BE003B335E013B35CC
:1033C00096023B37000099599959EB518F421E459F
:1033D000142E0080EB51F5283333E13A703DE13A89
:1033E000C235852BC2353333C235C235AE47E13ADB
:1033F0005138A330513800404040404040404040A8
:1034000041414141414040404040404040404040B7
:1034100040404040404040050202020202020202D7
:10342000020202020202022020202020202020206E
:1034300020020202020202029090909090901010DE
:10344000101010101010101010101010101010107C
:103450001010020202020202888888888888080800
:1034600008080808080808080808080808080808DC
:103470000808020202024000F73301082B514955A7
:1034800052433A20227064706465616374220000C4
:103490002B51495552433A2022636C6F7365642265
:1034A0002C0000002B51495552433A20227265638B
:1034B00076222C002B524543454956452C000000EE
:1034C000414952373830455F4556454E545F4E5559
:1034D0004D5F300030000000414952373830455FC1
:1034E0004556454E545F4E554D5F3100310000004A
:1034F000414952373830455F4556454E545F4E5529
:103500004D5F320032000000414952373830455F8C
:103510004556454E545F4E554D5F33003300000015
:10352000414952373830455F4556454E545F4E55F8
:103530004D5F340034000000414952373830455F58
:103540004556454E545F4E554D5F350035000000E1
:10355000414952373830455F4556454E545F4E55C8
:103560004D5F360036000000414952373830455F24
:103570004556454E545F4E554D5F370037000000AD
:10358000414952373830455F4556454E545F4E5598
:103590004D5F380038000000414952373830455FF0
:1035A0004556454E545F4E554D5F39003900000079
:1035B0002B5147505358545241444154413A000012
:1035C0002B514D545355423A000000002B434950B3
:1035D00047534D4C4F433A002B514750534C4F43A8
:1035E0003A0000002B514D54444953433A00000027
:1035F0002B5148545450524541443A002B434349BF
:10360000443A00002B514953454E443A0000000013
:103610002B514952443A00002B51485454505245C2
:10362000414446494C453A002B5148545450504F60
:10363000535446494C453A002B514C544F4E453A51
:10364000000000002B514D54434C4F53453A0000AD
:103650002B435245473A00002B43475245473A0017
:103660002B514D5450494E473A0000002B434D54C6
:10367000493A00002B43434C4B3A00002B51464F34
:1036800050454E3A000000002B51494F50454E3AEC
:10369000000000002B514D544F50454E3A000000A1
:1036A0002B4350494E3A00002B514D54434F4E4E40
:1036B0003A0000002B4353513A0000002B434D4782
:1036C000523A00002B434D45204552524F523A008A
:1036D0002B514D54554E533A000000002B43545487
:1036E000533A00002B514D54535441543A000000BA
:1036F0002B51485454504745543A00002B51464CE6
:1037000053543A002B5148545450504F53543A009C
:103710002B43474154543A002B514D545245435684
:103720003A0000002B514D5450554245583A000084
:103730003E000000414952373830455F4556454EFE
:10374000545F514750535854524144415441000032
:10375000414952373830455F4556454E545F4E45D6
:10376000575F49505F44415441000000414952377E
:103770003830455F4556454E545F534D535F444185
:1037800054410000414952373830455F4556454E57
:10379000545F514D54535542000000004149523787
:1037A0003830455F4556454E545F514750534C4F56
:1037B00043000000414952373830455F4556454E79
:1037C000545F514D5444495343000000414952371E
:1037D0003830455F4556454E545F51485454505219
:1037E00045414400414952373830455F4556454EC2
:1037F000545F524541440000414952373830455FDB
:103800004556454E545F43434944000041495237B1
:103810003830455F4556454E545F53454E44000091
:10382000414952373830455F4556454E545F5148FF
:103830005454505245414446494C45004149523741
:103840003830455F4556454E545F514854545050AA
:103850004F535446494C4500414952373830455F33
:103860004556454E545F514C544F4E4500000000A4
:10387000414952373830455F4556454E545F514DAA
:1038800054434C4F53450000414952373830455F4F
:103890004556454E545F434C4F53450041495237BE
:1038A0003830455F4556454E545F5245434549566D
:1038B00045000000414952373830455F4556454E76
:1038C000545F435245470000414952373830455F05
:1038D0004556454E545F434752454700414952378C
:1038E0003830455F4556454E545F514D5450494E12
:1038F00047000000414952373830455F4556454E34
:10390000545F41434B000000414952373830455F16
:103910004556454E545F43434C4B000053454E447F
:10392000204F4B0053485554204F4B0041495237CC
:103930003830455F4556454E545F53454E445F4FC2
:103940004B000000414952373830455F4556454EDF
:10395000545F4F4B000000004849444F5F41545FA3
:103960004556454E545F4F4B000000004F4B000042
:1039700053454E44204641494C00000041495237CE
:103980003830455F4556454E545F53454E445F467B
:1039900041494C002D414952373830455F45564525
:1039A0004E545F504F4C4C00414952373830455FC0
:1039B0004556454E545F51464F50454E000000005D
:1039C000414952373830455F4556454E545F514D59
:1039D000544F50454E000000414952373830455F42
:1039E0004556454E545F4F50454E000041495237B1
:1039F0003830455F4556454E545F4350494E0000B0
:103A0000414952373830455F4556454E545F514D18
:103A100054434F4E4E000000414952373830455F05
:103A20004556454E545F4C42535F4C4F43415449B9
:103A30004F4E0000414952373830455F4556454E9C
:103A4000545F4353510000004849444F5F41545F65
:103A50004556454E545F53454E445F4552524F5272
:103A6000000000004849444F5F41545F4556454EB1
:103A7000545F4552524F52004552524F520000007F
:103A8000414952373830455F4556454E545F52459F
:103A900041445F534D530000414952373830455F30
:103AA0004556454E545F4E45575F534D53000000F9
:103AB000414952373830455F4556454E545F514D68
:103AC00054554E5300000000414952373830455F8D
:103AD0004556454E545F51545453000041495237A6
:103AE0003830455F4556454E545F514D545354410F
:103AF00054000000414952373830455F4556454E25
:103B0000545F5044504445414354000041495237AA
:103B10003830455F4556454E545F434F4E4E454302
:103B200054000000434F4E4E454354004149523724
:103B30003830455F4556454E545F514854545047C0
:103B4000455400004556454E545F455849540000C1
:103B5000414952373830455F4556454E545F5146CE
:103B60004C535400414952373830455F4556454E15
:103B7000545F5148545450504F53540041495237A8
:103B80003830455F4556454E545F434741545400D5
:103B9000414952373830455F4556454E545F494E8E
:103BA00049545F54494D454F555400004849444FCE
:103BB0005F41545F4556454E545F54494D454F55FE
:103BC00054000000414952373830455F4556454E54
:103BD000545F514D545245435600000041495237FD
:103BE0003830455F4556454E545F514D545055420F
:103BF00045580000414952373830455F4556454EDB
:103C0000545F44454C415900414952373830455F73
:103C10004556454E545F52445900000052445900E5
:103C20004556454E545F454E5452590041542B431E
:103C30005354543D222573222C22222C22220D0A79
:103C40000000000041542B4349505258463D310D6D
:103C50000A00000041542B4349504D55583D310D49
:103C60000A00000041542B434349440D0A00000060
:103C700041542B43494D490D0A0000004154490D60
:103C80000A00000041542B4347534E0D0A00000028
:103C900041542B43494943520D0A000041542B43E0
:103CA000494653520D0A0000414952373830450009
:103CB0004149523738304552756E4154436D640066
:103CC0004149523738304549646C650041495237A3
:103CD000383045506F7765724F66660041495237FC
:103CE0003830454950436865636B0000414952379D
:103CF0003830454950506F6C6C00000041495237D4
:103D0000383045506F7765724F6E00004149523729
:103D1000383045436C6F7365576972656C657373B2
:103D200000000000414952373830454F70656E57EA
:103D30006972656C65737300414952373830454983
:103D40006E697400414952373830454950496E69AF
:103D500074000000414952373830454154436D6486
:103D6000496E6974000000004149523738304541BE
:103D700054436D6454657374000000004149523728
:103D8000383045526561647900000000414952377E
:103D900038304549505265616479000041495237D5
:103DA0003830455761697453696D43617264526577
:103DB0006164790041495237383045536561726317
:103DC00068696E674E6574776F726B004149523750
:103DD000383045536F636B657453656E644461742A
:103DE0006100000041495237383045536F636B65BD
:103DF00074436C6F73650000414952373830455346
:103E00006F636B6574436F6E6E65637400000000D2
:103E100041495237383045435351000041495237E8
:103E20003830454C6F6300006F7461006C6F675FE2
:103E300075706C6F616400006465766963655F69C5
:103E40006400000061745F636D6400007463705F00
:103E500073656E64000000006462675F6D6F646587
:103E6000000000007365745F7274636D6D6F64654C
:103E7000000000007365745F757762656E61626C47
:103E8000650000007365745F6770737570646174BA
:103E90006574696D65000000617564696F5F766FB8
:103EA0006C756D65000000007463705F636C6F7308
:103EB0006500000075706461746500007463705F74
:103EC00063726561746500006770735F6261756439
:103ED0005F726174650000007365745F6461746192
:103EE000726174650000000064656275675F6F66EB
:103EF0006600000034675F706F7765726F666600FA
:103F00006C6F67007365745F7274636D000000000E
:103F10007274635F7365745F616C61726D00000041
:103F20006C6F675F636C65616E000000646562754D
:103F3000675F6F6E0000000034675F706F776572B7
:103F40006F6E00007365727665725F696E666F00F2
:103F5000696E666F00000000736C6565700000009C
:103F60007365745F6E747269700000007365745FCE
:103F70006770735F730000007365745F63686169E5
:103F80006368756770735F7300000000636C6F7324
:103F9000655F776972656C65737300006F70656E3D
:103FA0005F776972656C6573730000007463705F9E
:103FB000636F6E6E656374007274635F676574002F
:103FC0007274635F736574006C6F675F7072696EA3
:103FD000740000007265626F6F7400007465737422
:103FE000000000007474735F706C61790000000061
:103FF0007365745F7178777A00000000636C6561A7
:10400000720000006C7300002840010800000020CE
:1040100084060000D45F00080041010884060020E7
:10402000444200004C170108022B0A581524434350
:104030004D53472C524D432C312C302C2A30340D0B
:104040000A145C475341149A44144A56148B314164
:10405000145B4C4C147A46145C5458543C7B300D21
:104060008F32019204025D2085B03C010813256C5B
:104070008C080C3D1013E9639B08241013516A79D6
:104080000C01148B103E2C1A213C01309A1C400B61
:1040900014E568400217017A01194BC84204013047
:1040A00003C655AA000C5F24474E4747412C4C429B
:1040B000532C140502041509090102024341E201CF
:1040C00062FF1A0762380C1E0805400826091040D6
:1040D00008560A131D043B08BE05062AD8BC40102A
:1040E00008320217FC3F010865C1100808044001AE
:1040F00008C1C209293E01FF01FF014CB2010000C5
:04000005080050C1DE
:00000001FF
